:04000C00A8600000E8
:10001000E06000001861000050610000886100008D
:040048000062000052
:040054003063000015
:04007800C061000063
:0400A00032640000C6
:100400003220EF00C3202000008041001040BA00DD
:100410000160EF00000006000A0D0000416C0000C2
:100420006C20000044650000636F000064650000FC
:1004300072730000206C00006F61000064650000B2
:10044000640A00000D000000CF0278003220EF00A7
:1004500023232000008041001040BA000160EF001B
:10046000000006000A0D0000496E000070750000D3
:1004700074200000257500003A20000020000000D4
:10048000CF0278003220EF00E324200000804100FA
:100490001040BA000160EF0000000600313000009B
:1004A000383000007020000028350000392E000090
:1004B000393400002920000044650000636F00000B
:1004C0006465000072200000436F00006E6600004B
:1004D00069670000204400006F6E0000650A00009C
:1004E0000D000000CF0278003220EF00032820002A
:1004F000008041001040BA000160EF0000000600DB
:100500003130000038300000702000002835000035
:100510003029000020440000656300006F64000083
:1005200065720000204300006F6E000066690000E5
:1005300067200000446F00006E6500000A0D000097
:1005400000000000CF0278003220EF00032B2000D3
:10055000008041001040BA000160EF00000006007A
:1005600031300000383000006920000028350000DC
:10057000392E0000393400002920000044650000B5
:10058000636F00006465000072200000436F00008C
:100590006E66000069670000204400006F6E000076
:1005A000650A00000D000000CF0278003220EF0045
:1005B000232E2000008041001040BA000160EF00AF
:1005C00000000600313000003830000069200000D3
:1005D0002835000030290000204400006563000039
:1005E0006F64000065720000204300006F6E000021
:1005F0006669000067200000446F00006E6500001F
:100600000A0D000000000000CF0278003220EF0049
:1006100023312000008041001040BA000160EF004B
:10062000000006003732000030700000283500005E
:10063000392E0000393400002920000044650000F4
:10064000636F00006465000072200000436F0000CB
:100650006E66000069670000204400006F6E0000B5
:10066000650A00000D000000CF0278003220EF0084
:1006700023342000008041001040BA000160EF00E8
:1006800000000600373200003070000028350000FE
:100690003029000020440000656300006F64000002
:1006A00065720000204300006F6E00006669000064
:1006B00067200000446F00006E6500000A0D000016
:1006C00000000000CF0278003220EF000337200046
:1006D000008041001040BA000160EF0000000600F9
:1006E000363400003020000078200000343800004C
:1006F000302800003630000029200000456E000040
:10070000636F00006465000072200000436F00000A
:100710006E66000069670000204400006F6E0000F4
:10072000650A00000D000000CF0278003220EF00C3
:10073000233A2000008041001040BA000160EF0021
:100740000000060038300000302000007820000053
:10075000363000003028000036300000292000002C
:1007600044650000636F00006465000072200000B3
:10077000436F00006E6600006967000020440000BF
:100780006F6E0000650A00000D000000CF027800C7
:100790003220EF00433D2000008041001040BA00AD
:1007A0000160EF000000060031300000323400002C
:1007B000207800002037000036380000283600007E
:1007C0003029000020440000656300006F640000D1
:1007D00065720000204300006F6E00006669000033
:1007E00067200000446F00006E6500000A0D0000E5
:0807F00000000000CF027800B8
:10180000FE460400020000003220EF0003C1200069
:10181000008041001040BA000160EF0000000600A7
:101820003132000038300000207800002031000004
:10183000303200003428000036300000292000003B
:1018400044650000636F00006465000072200000C2
:10185000436F00006E6600006967000020440000CE
:101860006F6E0000650A00000D000000CF027800D6
:101870003220EF0043C42000008041001040BA0035
:101880000160EF0000000600313200003830000037
:10189000207800002037000036380000283600008D
:1018A0003029000020440000656300006F640000E0
:1018B00065720000204300006F6E00006669000042
:1018C00067200000446F00006E6500000A0D0000F4
:1018D00000000000CF0278003220EF0083C7200014
:1018E000008041001040BA000160EF0000000600D7
:1018F0003133000036360000207800002037000029
:10190000363800002836000030290000204400004E
:10191000656300006F6400006572000020430000F2
:101920006F6E00006669000067200000446F0000D1
:101930006E6500000A0D000000000000CF02780074
:101940003220EF00C3CA2000008041001040BA00DE
:101950000160EF000000060031340000303000006C
:1019600020780000203100003035000030280000D1
:10197000363000002920000044650000636F00003D
:101980006465000072200000436F00006E66000076
:1019900069670000204400006F6E0000650A0000C7
:1019A0000D000000CF0278003220EF0003CE2000AF
:1019B000008041001040BA000160EF000000060006
:1019C0003136000030300000207800002031000067
:1019D000323000003028000036300000292000009E
:1019E00044650000636F0000646500007220000021
:1019F000436F00006E66000069670000204400002D
:101A00006F6E0000650A00000D000000CF02780034
:101A10003220EF0043D12000008041001040BA0086
:101A20000160EF000000060053440000204E00005B
:101A3000545300004320000028200000532D0000D4
:101A400056690000646500006F2900002044000012
:101A5000656300006F6400006572000020430000B1
:101A60006F6E00006669000067200000446F000090
:101A70006E6500000A0D000000000000CF02780033
:101A80003220EF00C3D42000008041001040BA0093
:101A90000160EF00000006005344000020500000E9
:101AA000414C000020200000285300002D5600006B
:101AB00069640000656F0000292000004465000093
:101AC000636F00006465000072200000436F000037
:101AD0006E66000069670000204400006F6E000021
:101AE000650A00000D000000CF0278003220EF00F0
:101AF000E3012000830150000500310023D92000BC
:101B0000008041001040BA000160EF0000000600B4
:101B100020D9200083814100808141001380BA00D8
:101B2000000006005344430020206F004E546E0016
:101B30005343660020286900204367006F6D200032
:101B4000706F440073696F0074656E002920650032
:101B500044650A00636F0D00646500007220000098
:101B6000CF0278003220EF00C30120008301500033
:101B700005003100E3DC2000008041001040BA0085
:101B80000160EF0000000600E0DC200083814100DE
:101B9000808141001380BA000000060053444300D6
:101BA00020506F00414C6E002028660020436900E1
:101BB0006F6D6700706F20007369440074656F007B
:101BC00029206E0044656500636F0A0064650D009E
:101BD00072200000CF0278003220EF0083DF200067
:101BE000008041001040BA000160EF0000000600D4
:101BF0003139000032300000207800002031000030
:101C0000323000003020000028360000304800004C
:101C10007A2900002D2000004E4F000054200000C3
:101C200073750000707000006F7200007465000032
:101C3000640A00000D000000CF0278003220EF009F
:101C4000A3E22000008041001040BA000160EF00D4
:101C500000000600556E00006B6E00006F770000FC
:101C60006E0A00000D000000CF0278003220EF0065
:101C700023E42000008041001040BA000160EF0022
:101C8000000006000A0D0000456E0000636F0000B2
:101C900064650000722000006C6F00006164000049
:101CA000656400000A0D000000000000CF0278000B
:101CB0003220EF0043E62000008041001040BA00CF
:101CC0000160EF00000006000A0D000056580000F9
:101CD000503A000020000000CF0278003220EF00D0
:101CE000A3E72000008041001040BA000160EF002F
:101CF0000000060031300000383000007020000085
:101D000028350000392E0000393400002920000059
:101D1000456E0000636F00006465000072200000E3
:101D2000436F00006E6600006967000020440000F9
:101D30006F6E0000650A00000D000000CF02780001
:101D40003220EF00C3EA2000008041001040BA00BA
:101D50000160EF0000000600313000003830000064
:101D600070200000283500003029000020450000C8
:101D70006E6300006F640000657200002043000085
:101D80006F6E00006669000067200000446F00006D
:101D90006E6500000A0D000000000000CF02780010
:101DA0003220EF00C3ED2000008041001040BA0057
:101DB0000160EF0000000600313000003830000004
:101DC0006920000028350000392E00003934000059
:101DD00029200000456E0000636F0000646500006C
:101DE00072200000436F00006E660000696700000B
:101DF000204400006F6E0000650A00000D00000026
:101E0000CF0278003220EF00E3F020000080410094
:101E10001040BA000160EF00000006003130000001
:101E2000383000006920000028350000302900000B
:101E3000204500006E6300006F64000065720000C2
:101E4000204300006F6E00006669000067200000FC
:101E5000446F00006E6500000A0D000000000000E5
:101E6000CF0278003220EF00E3F320000080410031
:101E70001040BA000160EF00000006003732000099
:101E80003070000028350000392E00003934000081
:101E900029200000456E0000636F000064650000AB
:101EA00072200000436F00006E660000696700004A
:101EB000204400006F6E0000650A00000D00000065
:101EC000CF0278003220EF00E3F6200000804100CE
:101ED0001040BA000160EF00000006003732000039
:101EE0003070000028350000302900002045000037
:101EF0006E6300006F640000657200002043000004
:101F00006F6E00006669000067200000446F0000EB
:101F10006E6500000A0D000000000000CF0278008E
:101F20003220EF00C3F92000008041001040BA00C9
:101F30000160EF0000000600383000003020000093
:101F400078200000363000003028000036300000D5
:101F500029200000456E0000636F000064650000EA
:101F600072200000436F00006E6600006967000089
:101F7000204400006F6E0000650A00000D000000A4
:101F8000CF0278003220EF00E3FC20000080410007
:101F90001040BA000160EF00000006003130000080
:101FA000323400002078000020370000363800006E
:101FB0002836000030290000204500006E63000034
:101FC0006F64000065720000204300006F6E000027
:101FD0006669000067200000446F00006E65000025
:101FE0000A0D000000000000CF0278003220EF0050
:101FF00023002100008041001040BA000160EF0082
:102000000000060031320000383000002078000067
:102010002037000036380000283600003029000044
:10202000204500006E6300006F64000065720000D0
:10203000204300006F6E000066690000672000000A
:10204000446F00006E6500000A0D000000000000F3
:10205000CF0278003220EF006303210000804100AE
:102060001040BA000160EF000000060031320000AD
:1020700038300000207800002031000030320000AD
:10208000342800003630000029200000456E000092
:10209000636F00006465000072200000436F000061
:1020A0006E66000069670000204400006F6E00004B
:1020B000650A00000D000000CF0278003220EF001A
:1020C000A3062100008041001040BA000160EF002B
:1020D0000000060031330000363600002078000092
:1020E0002037000036380000283600003029000074
:1020F000204500006E6300006F6400006572000000
:10210000204300006F6E0000666900006720000039
:10211000446F00006E6500000A0D00000000000022
:10212000CF0278003220EF00E30921000080410057
:102130001040BA000160EF000000060031340000DA
:1021400030300000207800002031000030350000E1
:10215000302800003630000029200000456E0000C5
:10216000636F00006465000072200000436F000090
:102170006E66000069670000204400006F6E00007A
:10218000650A00000D000000CF0278003220EF0049
:10219000230D2100008041001040BA000160EF00D3
:1021A00000000600313600003030000020780000CA
:1021B00020310000323000003028000036300000AE
:1021C00029200000456E0000636F00006465000078
:1021D00072200000436F00006E6600006967000017
:1021E000204400006F6E0000650A00000D00000032
:1021F000CF0278003220EF00631021000080410000
:102200001040BA000160EF00000006003139000004
:102210003230000020780000203100003230000011
:10222000302800003630000029200000456E0000F4
:10223000636F00006465000072200000436F0000BF
:102240006E66000069670000204400006F6E0000A9
:10225000650A00000D000000CF0278003220EF0078
:10226000E30120008301500005003100A314210088
:10227000008041001040BA000160EF00000006003D
:10228000A014210083814100808141001380BA00A5
:102290000000060053444300202D6F0020376E00DD
:1022A0003230660020786900203467003830200022
:1022B000202844004E546F0053436E0029206500CF
:1022C000456E0A00636F0D00646500007220000017
:1022D000CF0278003220EF00631721000080410018
:1022E0001040BA000160EF000000060053440000F7
:1022F000203700003638000020780000203500002C
:102300003736000020280000504100004C29000012
:10231000204500006E6300006F64000065720000DD
:10232000204300006F6E0000666900006720000017
:10233000446F00006E6500000A0D00000000000000
:10234000CF0278003220EF0003022000830150000A
:1023500005003100E31B2100008041001040BA005D
:102360000160EF0000000600E01B210083814100B6
:10237000808141001380BA00000006005344200011
:10238000202D430020286F0034386E00306966002D
:1023900020796900506267005072200029204400B3
:1023A000284E6F0054536E004329650020450A00F3
:1023B0006E630D006F64000065720000CF0278004C
:1023C0003220EF00E30120008301500005003100BE
:1023D000C31F2100008041001040BA000160EF00DF
:1023E00000000600C01F2100838141008081410060
:1023F0001380BA00000006005344430020286F00F9
:1024000035376E00366966002079690050626700D2
:10241000507220002920440028506F00414C6E006B
:1024200029206500456E0A00636F0D006465000099
:1024300072200000CF0278003220EF0083222100BA
:10244000008041001040BA000160EF00000006006B
:102450000A0D000056580000502800007277000056
:10246000293A000000000000CF0278003220EF007F
:1024700023242100008041001040BA000160EF00D9
:10248000000006000A0D0000565800005028000009
:10249000772900003A20000000000000CF027800F9
:1024A0003220EF00C3252100008041001040BA0017
:1024B0000160EF00000006000A0D00005658000001
:1024C00050280000722900003A200000000000009F
:1024D000CF0278003220EF00632721000080410006
:1024E0001040BA000160EF000000060057720000C3
:1024F0006974000065200000254C0000580A0000A7
:102500000D000000CF0278003220EF0003292100E7
:10251000008041001040BA000160EF00000006009A
:10252000577200006974000065200000254C00000F
:10253000582C00002052000065610000642000005B
:10254000254C0000580A00000D000000CF02780062
:102550003220EF00432B2100008041001040BA00E0
:102560000160EF00000006004D6400000000000064
:10257000CF0278003220EF00632C21000080410060
:102580001040BA000160EF00000006004C67000038
:1025900000000000CF0278003220EF00832D2100E0
:1025A000008041001040BA000160EF00000006000A
:1025B000536D000000000000CF0278003220EF00D1
:1025C000A32E2100008041001040BA000160EF00FE
:1025D000000006005552000000000000CF02780005
:1025E0003220EF00C32F2100008041001040BA00CC
:1025F0000160EF00000006004C52000000000000E7
:10260000CF0278003220EF00E3302100008041004B
:102610001040BA000160EF00000006004C4D0000C1
:1026200000000000CF0278003220EF0003322100CA
:10263000008041001040BA000160EF000000060079
:102640004C4C000000000000CF0278003220EF0068
:1026500023332100008041001040BA000160EF00E8
:1026600000000600554C000000000000CF0278007A
:102670003220EF0043342100008041001040BA00B6
:102680000160EF000000060050490000503A0000D1
:1026900020250000732C00004C2000002573000052
:1026A00000000000CF0278003220EF00030320007A
:1026B00083015000050031000337210000804100F4
:1026C0001040BA000160EF00000006000037210052
:1026D00083814100808141001380BA000000060020
:1026E0000D0A2C000D0A450052656E0061646400FD
:1026F00044754300616C680055616100727472003A
:10270000506F3D00727425002C5032006F727800BB
:10271000743D2C00257557002C42610075666900D8
:1027200066657400723D3D00254C2500582C6C00F8
:10273000536975007A650A003D250D003278000066
:10274000CF0278003220EF00E33A21000080410000
:102750001040BA000160EF00000006000D0A000002
:10276000526500006164000044750000616C000067
:102770005561000072740000506F00007274000018
:1027800028250000752900003A2000000000000004
:10279000CF0278003220EF00633D2100008041002D
:1027A0001040BA000160EF00000006002D2000007C
:1027B000546900006D6500006F750000742800000A
:1027C000256C0000782900000A0D000000000000C0
:1027D000CF0278003220EF00633F210000804100EB
:1027E0001040BA000160EF00000006002D2000003C
:1027F00045720000726F000072280000256C000016
:10280000782900000A0D000000000000CF027800C7
:102810003220EF00E3012000830150000500310069
:1028200043422100008041001040BA000160EF00E7
:102830000000060040422100838141008081410068
:102840001380BA00000006000D0A780028552C00FD
:102850003229440045726100726F7400725B61003E
:1028600042493A002C202500504532002C207800A7
:10287000464529005D280A004C530D00523A0000DD
:1028800025320000CF0278003220EF0003452100FE
:10289000008041001040BA000160EF000000060017
:1028A0000D0A000028550000322900004572000082
:1028B000726F0000725B00004F76000065720000CE
:1028C000727500006E5D0000284C0000535200003D
:1028D0003A250000327800002C44000061740000AA
:1028E000613A000025320000782900000A0D00003E
:1028F00000000000CF0278003220EF00E30120004A
:10290000830150000500310083492100008041000F
:102910001040BA000160EF0000000600804921006D
:1029200083814100808141001380BA0000000600CD
:102930000D0A780028552C003129440045726100A9
:10294000726F7400725B610042493A002C202500CE
:10295000504532002C207800464529005D280A00A9
:102960004C530D00523A000025320000CF0278008F
:102970003220EF00434C2100008041001040BA009B
:102980000160EF00000006000D0A0000285500005D
:102990003129000045720000726F0000725B000078
:1029A0004F76000065720000727500006E5D0000D9
:1029B000284C0000535200003A25000032780000F5
:1029C0002C44000061740000613A000025320000D0
:1029D000782900000A0D000000000000CF027800F6
:1029E0003220EF00C34F2100008041001040BA00A8
:1029F0000160EF000000060045720000726F0000E9
:102A0000723A0000204900006E760000616C000000
:102A100069640000204D00006573000073610000D0
:102A2000676500002825000032780000290A0000B0
:102A30000D000000CF0278003220EF008352210009
:102A4000008041001040BA000160EF000000060065
:102A5000284D00004C4E00004B5F00004254000027
:102A60004E290000436F0000646500003D25000012
:102A7000327800002C20000025320000782C000065
:102A800020250000327800002C20000025320000B4
:102A9000780D00000A000000CF0278003220EF001D
:102AA000A3552100008041001040BA000160EF00F2
:102AB00000000600286400006566000061750000E3
:102AC0006C7400003A290000436F00006465000048
:102AD0003D250000327800002C2000002532000047
:102AE000782C000020250000327800002C20000007
:102AF00025320000780D00000A000000CF027800A7
:102B00003220EF00C3582100008041001040BA007D
:102B10000160EF00000006000A0D00004275000091
:102B20006666000065720000204F000076650000B8
:102B3000724C0000617000002045000072720000BD
:102B40006F7200000D0A000000000000CF02780044
:102B50003220EF00435B2100008041001040BA00AA
:102B60000160EF0000000600205000004343000019
:102B700020500000726F000067720000616D00005D
:102B8000204D00006F640000652000002000000060
:102B9000CF0278003220EF00635D21000080410009
:102BA0001040BA000160EF00000006002020000085
:102BB0002020000020200000202000002020000015
:102BC0002020000020200000202000002020000005
:102BD00020000000CF0278003220EF00835F210048
:102BE000008041001040BA000160EF0000000600C4
:102BF000202000005570000064610000746900002E
:102C00006E67000020430000616D000065720000E7
:102C10006120000020000000CF0278003220EF0089
:102C2000A3612100008041001040BA000160EF0064
:102C3000000006005072000065730000657400001B
:102C40002025000075200000506100006E6100002A
:102C5000736F00006E69000063200000436F000086
:102C60006D7000006C650000746500000A0D0000C6
:102C700000000000CF0278003220EF0083642100C2
:102C8000008041001040BA000160EF000000060023
:102C90002050000072650000736500007420000081
:102CA00025330000750A00000D000000CF027800F7
:102CB0003220EF0043662100008041001040BA003E
:102CC0000160EF0000000600507200006573000014
:102CD000657400002025000075200000536F00007F
:102CE0006E7900002F430000616E00006F6E0000DF
:102CF000204300006F6D0000706C000065740000E0
:102D0000650A00000D000000CF0278003220EF00BD
:102D100023692100008041001040BA000160EF00EB
:102D2000000006005072000065730000657400002A
:102D3000202500007520000054720000616E000024
:102D400073690000746900006F6E00000A0D0000D6
:102D500000000000CF0278003220EF00836B2100DA
:102D6000008041001040BA000160EF000000060042
:102D7000507200006573000065740000202500009B
:102D80007520000054720000616E0000736900003D
:102D9000746900006F6E000028730000290A0000AB
:102DA0000D000000CF0278003220EF00036E2100FA
:102DB000008041001040BA000160EF0000000600F2
:102DC000507200006573000065740000202500004B
:102DD0007520000054720000616E000073690000ED
:102DE000746900006F6E000028670000290A000067
:102DF0000D000000CF0278003220EF008370210028
:102E0000008041001040BA000160EF0000000600A1
:102E100020500000726500007365000074200000FF
:102E200025330000752000004C6F00006164000035
:102E30006564000000000000CF0278003220EF003F
:102E4000A3722100008041001040BA000160EF0031
:102E50000000060020500000434300002050000006
:102E600072650000736500007420000025330000C7
:102E7000752000004C6F0000616400006564000074
:102E800000000000CF0278003220EF00037521001F
:102E9000008041001040BA000160EF000000060011
:102EA0002020000020200000202000002020000022
:102EB0002020000020200000202000002020000012
:102EC0002020000000000000CF0278003220EF0038
:102ED00023772100008041001040BA000160EF001C
:102EE00000000600536500006C20000049520000FD
:102EF0002D50000072650000736500007420000012
:102F0000312000002020000000000000CF027800E7
:102F10003220EF0043792100008041001040BA00C8
:102F20000160EF0000000600536500006C20000007
:102F3000495200002D5000007265000073650000CA
:102F4000742000003020000020200000000000005D
:102F5000CF0278003220EF00637B21000080410027
:102F60001040BA000160EF00000006005365000049
:102F70006C200000495200002D50000072650000D6
:102F800073650000742000003125000063200000FC
:102F900000000000CF0278003220EF00837D210086
:102FA000008041001040BA000160EF000000060000
:102FB000536500006C200000495200002D500000B5
:102FC0007265000073650000742000003025000069
:102FD0006320000000000000CF0278003220EF00E4
:102FE000A37F2100008041001040BA000160EF0083
:102FF00000000600536500006C20000049520000EC
:103000002D50000072650000736500007420000000
:10301000253300007520000000000000CF0278007A
:103020003220EF00C3812100008041001040BA002F
:103030000160EF0000000600507200006F630000A6
:10304000657300007320000050720000657300007B
:10305000657400003D250000750A00000D000000A9
:10306000CF0278003220EF000302200083015000DD
:1030700005003100E3842100008041001040BA00C7
:103080000160EF0000000600E08421008381410020
:10309000808141001380BA00000006004275500094
:1030A000696C7200644D6500756C7300746965002D
:1030B000205074007265320073652800742025006A
:1030C00050723200657375006574290028310A005A
:1030D000293D0D0025320000752C0000CF0278003C
:1030E0003220EF00C3872100008041001040BA0069
:1030F0000160EF00000006004669000072730000E6
:1031000074200000507200006573000065740000B8
:1031100020500000726500007365000074280000F4
:10312000312900003D250000750A00000D00000057
:10313000CF0278003220EF00638A21000080410036
:103140001040BA000160EF00000006005365000067
:103150006C200000495200002D50000072650000F4
:103160007365000074200000253200007520000007
:1031700000000000CF0278003220EF00838C210095
:10318000008041001040BA000160EF00000006001E
:103190000A0D000052650000616400002043000039
:1031A0006F6E00006669000067280000257500004A
:1031B000293A000020000000CF0278003220EF0002
:1031C000A38E2100008041001040BA000160EF0092
:1031D000000006002043000068650000636B0000EB
:1031E000737500006D3D000025320000782000005E
:1031F000536100006D6500000A0D00000000000032
:10320000CF0278003220EF00E3012000830150005C
:1032100005003100E3912100008041001040BA0018
:103220000160EF0000000600E09121008381410071
:10323000808141001380BA00000006002043200076
:1032400068654400636B6900737566006D286600ED
:1032500025326500782972003D436500616C6E007F
:10326000637574006C610A0074650D0064280A00BF
:1032700025320D0078290000CF0278003220EF00BF
:10328000A3942100008041001040BA000160EF00CB
:103290000000060043680000656300006B730000D7
:1032A000756D000020520000656100006420000080
:1032B00025320000782C000020430000616C0000E3
:1032C000637500006C6100007465000064200000FC
:1032D00025320000780A00000D000000CF027800BF
:1032E0003220EF00C3972100008041001040BA0057
:1032F0000160EF0000000600436F00006E660000F2
:1033000069670000205300006176000065640000DA
:103310000A0D000000000000CF0278003220EF000C
:10332000A3992100008041001040BA000160EF0025
:1033300000000600526500006164000020450000A6
:1033400045500000726F00006D20000046610000D3
:10335000696C0000656400002D20000052650000CB
:103360006C6F00006164000020440000656600008E
:10337000617500006C740000730A00000D0000000D
:10338000CF0278003220EF00C301200083015000FB
:1033900005003100E39D2100008041001040BA008B
:1033A0000160EF0000000600E09D210083814100E4
:1033B000808141001380BA000000060028445000BC
:1033C0006F53720061766F0065446D006566200082
:1033D000617546006C7461007329690053616C006B
:1033E00076656500436F64006E660A0069670D00CC
:1033F00045450000CF0278003220EF0083A0210075
:10340000008041001040BA000160EF00000006009B
:103410004C6F000063200000254C0000782C000059
:1034200020500000726500007365000074200000E9
:10343000256400000A0D000000000000CF027800A3
:103440003220EF00C3A22100008041001040BA00EA
:103450000160EF000000060052650000616400009A
:10346000204C00006F630000202500004C78000015
:103470002C200000436100006D65000072610000B7
:10348000202500006420000050430000432000007D
:103490005072000065730000657400002025000074
:1034A000640A00000D000000CF0278003220EF0017
:1034B00023A62100008041001040BA000160EF0007
:1034C00000000600436100006D65000072610000AD
:1034D000204E0000756D0000626500007220000043
:1034E00025750000206E00006F740000204D000064
:1034F000617400006368000020250000750A000068
:103500000D000000CF0278003220EF00E301200020
:10351000830150000500310003AA21000080410012
:103520001040BA000160EF000000060000AA210070
:1035300083814100808141001380BA0000000600B1
:103540005072200065734D0065746100204E740058
:10355000756D630062656800722020004368250075
:10356000656332006B735800756D0A0020250D00ED
:1035700032780000206E00006F740000CF027800E7
:103580003220EF00C3AC2100008041001040BA009F
:103590000160EF0000000600536100007665000046
:1035A000204C00006F630000202500004C780000D4
:1035B0002C200000436100006D6500007261000076
:1035C000202500006420000050430000432000003C
:1035D0005072000065730000657400002025000033
:1035E000640A00000D000000CF0278003220EF00D6
:1035F00023B02100008041001040BA000160EF00BC
:1036000000000600536F00006E79000020450000A6
:10361000564900002D4400003330000020200000F7
:10362000202000002020000020000000CF027800B1
:103630003220EF0043B22100008041001040BA0068
:103640000160EF0000000600536F00006E7900007B
:1036500020450000564900002D4400003330000092
:103660002F44000033310000202000002000000023
:10367000CF0278003220EF0063B4210000804100C7
:103680001040BA000160EF00000006005661000023
:1036900064640000696F0000204100006464000061
:1036A0002D6100002D430000616D0000202000000E
:1036B00020000000CF0278003220EF0083B6210006
:1036C000008041001040BA000160EF0000000600D9
:1036D000536F00006E79000020450000564900003D
:1036E0002D44000031300000302000002020000078
:1036F0002020000020000000CF0278003220EF00E0
:10370000A3B82100008041001040BA000160EF0022
:10371000000006005641000044440000494F0000EC
:1037200020480000442D0000313800002020000017
:10373000202000002020000020000000CF027800A0
:103740003220EF00C3BA2100008041001040BA00CF
:103750000160EF0000000600536F00006E7900006A
:1037600020450000564900002D440000373000007D
:103770002020000020200000202000002000000069
:10378000CF0278003220EF00E3BC2100008041002E
:103790001040BA000160EF0000000600536F000007
:1037A0006E79000020420000524300002D330000DB
:1037B00030300000202000002020000020200000E9
:1037C00020000000CF0278003220EF0003BF21006C
:1037D000008041001040BA000160EF0000000600C8
:1037E000536F00006E790000204200005243000039
:1037F0002D4800003730000030200000202000005D
:103800002020000020000000CF0278003220EF00CE
:1038100023C12100008041001040BA000160EF0088
:1038200000000600536F00006E7900002042000087
:10383000524300002D5A00003730000030200000B5
:10384000202000002020000020000000CF0278008F
:103850003220EF0043C32100008041001040BA0035
:103860000160EF0000000600536F00006E79000059
:1038700020420000524300002D5A00003333000064
:103880003020000020200000202000002000000048
:10389000CF0278003220EF0063C521000080410094
:1038A0001040BA000160EF0000000600536F0000F6
:1038B0006E79000020450000564900002D480000A8
:1038C00044310000202000002020000020200000C3
:1038D00020000000CF0278003220EF0083C72100D3
:1038E000008041001040BA000160EF0000000600B7
:1038F000506100006E610000736F00006E6900008F
:1039000063200000415700002D48000045310000B1
:103910003030000020000000CF0278003220EF009D
:10392000A3C92100008041001040BA000160EF00EF
:103930000000060043650000696C0000696E00002D
:103940006756000049450000572000002020000075
:10395000202000002020000020000000CF0278007E
:103960003220EF00C3CB2100008041001040BA009C
:103970000160EF0000000600436100006E6E000071
:103980006F6E000020560000432D000043350000FC
:10399000306900002F72000020200000200000008D
:1039A000CF0278003220EF00E3CD210000804100FB
:1039B0001040BA000160EF00000006004361000003
:1039C0006E6E00006F6E000020420000552D00005A
:1039D0003435000048200000202000002020000096
:1039E00020000000CF0278003220EF0003D0210039
:1039F000008041001040BA000160EF0000000600A6
:103A0000436100006E6E00006F6E000020420000F7
:103A1000552D000035300000482000002020000017
:103A20002020000020000000CF0278003220EF00AC
:103A300023D22100008041001040BA000160EF0055
:103A400000000600556E00006B6E00006F770000EE
:103A50006E200000436100006D650000726100008F
:103A6000202000002020000020000000CF0278006D
:103A70003220EF0043D42100008041001040BA0002
:103A80000160EF000000060000000000CF02780097
:103A90003220EF0043D52100008041001040BA00E1
:103AA0000160EF0000000600486F00007374000022
:103AB0002053000065720000696100006C20000066
:103AC000496E000070750000743A00002045000047
:103AD0006E610000626C0000656400000000000080
:103AE000CF0278003220EF00E3D7210000804100B0
:103AF0001040BA000160EF0000000600486F0000AF
:103B000073740000205300006572000069610000BA
:103B10006C200000496E000070750000743A0000CF
:103B20002044000069730000616200006C650000C1
:103B300064000000CF0278003220EF0083DA210019
:103B4000008041001040BA000160EF000000060054
:103B50005365000072690000616C000020450000A0
:103B6000636800006F3A0000204500006E610000AD
:103B7000626C00006564000000000000CF02780065
:103B80003220EF00C3DC2100008041001040BA0069
:103B90000160EF000000060053650000726900003C
:103BA000616C000020450000636800006F3A00006F
:103BB0002044000069730000616200006C65000031
:103BC00064000000CF0278003220EF0003DF210004
:103BD000008041001040BA000160EF0000000600C4
:103BE0005365000072690000616C0000204900000C
:103BF0006E6600006F3A0000204F00006E0000006B
:103C0000CF0278003220EF00E3E021000080410085
:103C10001040BA000160EF0000000600536500008C
:103C200072690000616C0000204900006E660000AF
:103C30006F3A0000204F00006666000000000000A0
:103C4000CF0278003220EF00E3E221000080410043
:103C50001040BA000160EF0000000600546100004F
:103C60006C6C0000792000004C6500007665000057
:103C70006C3A000020410000637400006976000087
:103C8000652000004C6F000077000000CF02780034
:103C90003220EF0043E52100008041001040BA00CF
:103CA0000160EF0000000600546100006C6C000031
:103CB000792000004C650000766500006C3A000039
:103CC0002041000063740000697600006520000058
:103CD000486900006768000000000000CF0278001B
:103CE0003220EF00C3E72100008041001040BA00FD
:103CF0000160EF00000006004469000061670000F9
:103D00006E6F00007374000069630000204D0000B6
:103D10006F640000653A0000204F00006E00000054
:103D2000CF0278003220EF00E3E92100008041005B
:103D30001040BA000160EF00000006004469000076
:103D4000616700006E6F000073740000696300001B
:103D5000204D00006F640000653A0000204F000015
:103D60006666000000000000CF0278003220EF00FD
:103D700023EC2100008041001040BA000160EF00F8
:103D8000000006005365000072690000616C0000CD
:103D90002044000069610000672000004D6F0000B2
:103DA000646500003A2000004F6E00000000000033
:103DB000CF0278003220EF0063EE21000080410046
:103DC0001040BA000160EF000000060053650000DB
:103DD00072690000616C000020440000696100000D
:103DE000672000004D6F0000646500003A2000006D
:103DF0004F66000066000000CF0278003220EF001E
:103E0000A3F02100008041001040BA000160EF00E3
:103E1000000006004578000074650000726E000026
:103E2000616C0000205400007269000067670000A8
:103E30006572000073200000496E00006974000084
:103E4000696100006C6900007A6500006400000090
:103E5000CF0278003220EF0063F3210000804100A0
:103E60001040BA000160EF00000006004578000035
:103E700074650000726E0000616C00002054000048
:103E8000726900006767000065720000732000001F
:103E90006E6F000074200000496E0000697400001D
:103EA000696100006C6900007A6500006400000030
:103EB000CF0278003220EF0063F62100008041003D
:103EC0001040BA000160EF000000060054720000CC
:103ED000616E000073690000746900006F6E00007D
:103EE000204D00006F640000653A0000204D000086
:103EF0006978000000000000CF0278003220EF0057
:103F0000A3F82100008041001040BA000160EF00DA
:103F10000000060054720000616E0000736900002A
:103F2000746900006F6E0000204D00006F64000097
:103F3000653A000020430000757400000000000096
:103F4000CF0278003220EF00E3FA21000080410028
:103F50001040BA000160EF0000000600547200003B
:103F6000616E000073690000746900006F6E0000EC
:103F7000204D00006F640000653A000020570000EB
:103F80006970000065000000CF0278003220EF0069
:103F900023FD2100008041001040BA000160EF00C5
:103FA0000000060057690000706500002052000004
:103FB0006967000068740000202D00003E200000AA
:103FC0004C6500006674000000000000CF0278001D
:103FD0003220EF0043FF2100008041001040BA0072
:103FE0000160EF00000006005769000070650000E6
:103FF000204C000065660000742000002D3E00008B
:104000002052000069670000687400000000000092
:10401000CF0278003220EF006301220000804100CF
:104020001040BA000160EF000000060020200000F0
:104030005769000070650000205400006F70000098
:10404000202D00003E200000426F00007420000080
:1040500000000000CF0278003220EF00830322002E
:10406000008041001040BA000160EF00000006002F
:104070002020000057690000706500002042000009
:104080006F740000202D00003E200000546F0000DF
:104090007020000000000000CF0278003220EF0006
:1040A000A3052200008041001040BA000160EF002B
:1040B000000006002020000020570000697000006A
:1040C000652000004C520000202D00003E20000022
:1040D000554C00002020000000000000CF027800B6
:1040E0003220EF00C3072200008041001040BA00D8
:1040F0000160EF00000006002020000020570000B3
:1041000069700000652000004C4C0000202D00006C
:104110003E2000005552000020200000000000005A
:10412000CF0278003220EF00E30922000080410036
:104130001040BA000160EF000000060020200000DF
:1041400020570000697000006520000055520000F3
:10415000202D00003E2000004C4C000020200000DC
:1041600000000000CF0278003220EF00030C220094
:10417000008041001040BA000160EF00000006001E
:10418000202000002057000069700000652000001A
:10419000554C0000202D00003E2000004C52000035
:1041A0002020000000000000CF0278003220EF0045
:1041B000230E2200008041001040BA000160EF0091
:1041C0000000060020200000576900007065000014
:1041D000205400006F200000436500006E74000052
:1041E000657200002020000000000000CF0278006F
:1041F0003220EF0043102200008041001040BA003E
:104200000160EF00000006005769000070650000C3
:10421000204C0000203E0000436500006E7400004A
:10422000657200003C2000005220000000000000E9
:10423000CF0278003220EF0063122200008041009C
:104240001040BA000160EF0000000600576900004E
:104250007065000020540000203E0000436500000F
:104260006E740000657200003C20000042200000D7
:1042700000000000CF0278003220EF0083142200FB
:10428000008041001040BA000160EF00000006000D
:10429000202000002020000020200000204E0000F0
:1042A0006F6E00006520000020200000202000002C
:1042B0002020000000000000CF0278003220EF0034
:1042C000A3162200008041001040BA000160EF00F8
:1042D000000006004D65000064690000756D000077
:1042E00000000000CF0278003220EF000318220007
:1042F000008041001040BA000160EF00000006009D
:104300004C6100007267000065000000CF02780079
:104310003220EF0043192200008041001040BA0013
:104320000160EF0000000600536D0000616C0000AA
:104330006C000000CF0278003220EF00831A2200C8
:10434000008041001040BA000160EF00000006004C
:104350005570000070650000722000005269000076
:1043600067680000742D0000257300000000000045
:10437000CF0278003220EF00631C22000080410051
:104380001040BA000160EF00000006004C6F000012
:104390007765000072200000526900006768000025
:1043A000742D00002573000000000000CF0278008B
:1043B0003220EF00431E2200008041001040BA006E
:1043C0000160EF00000006004C6F00007765000000
:1043D000722000004D690000646400006C650000FC
:1043E0002D25000073000000CF0278003220EF007E
:1043F00023202200008041001040BA000160EF003D
:10440000000006004C6F000077650000722000007D
:104410004C650000667400002D250000730000004C
:10442000CF0278003220EF00E3212200008041001B
:104430001040BA000160EF00000006005570000057
:1044400070650000722000004C650000667400007A
:104450002D25000073000000CF0278003220EF000D
:10446000A3232200008041001040BA000160EF0049
:1044700000000600205000004950000020530000BA
:10448000697A0000653A0000204D00006564000074
:10449000697500006D20000000000000CF02780068
:1044A0003220EF00C3252200008041001040BA00F6
:1044B0000160EF000000060020500000495000009D
:1044C00020530000697A0000653A0000204C00008B
:1044D00061720000676500002020000000000000FD
:1044E000CF0278003220EF00E32722000080410055
:1044F0001040BA000160EF000000060020500000EC
:104500004950000020530000697A0000653A00001D
:10451000205300006D6100006C6C00002020000042
:1045200000000000CF0278003220EF00032A2200B2
:10453000008041001040BA000160EF00000006005A
:104540002050000049500000204C00006F63000024
:1045500061740000696F00006E200000313A0000B5
:104560005552000000000000CF0278003220EF001A
:10457000232C2200008041001040BA000160EF00AF
:10458000000006002050000049500000204C0000B0
:104590006F63000061740000696F00006E2000000E
:1045A000323A00004C52000000000000CF027800B8
:1045B0003220EF00432E2200008041001040BA005C
:1045C0000160EF000000060020500000495000008C
:1045D000204C00006F63000061740000696F0000F0
:1045E0006E200000333A00004C4D00000000000037
:1045F000CF0278003220EF006330220000804100BB
:104600001040BA000160EF000000060020500000DA
:1046100049500000204C00006F63000061740000EE
:10462000696F00006E200000343A00004C4C00001E
:1046300000000000CF0278003220EF008332220019
:10464000008041001040BA000160EF000000060049
:104650002050000049500000204C00006F63000013
:1046600061740000696F00006E200000353A0000A0
:10467000554C000000000000CF0278003220EF000F
:10468000A3342200008041001040BA000160EF0016
:1046900000000600466F00007265000067720000AF
:1046A0006F7500006E64000000000000CF0278000B
:1046B0003220EF0043362200008041001040BA0053
:1046C0000160EF000000060042610000636B000023
:1046D000677200006F7500006E640000000000004B
:1046E000CF0278003220EF00E33722000080410043
:1046F0001040BA000160EF000000060050610000A9
:1047000073730000204F00006E20000053740000FF
:1047100061740000757300003A20000041630000DE
:10472000746900007665000000000000CF02780088
:104730003220EF00433A2200008041001040BA00CE
:104740000160EF000000060050610000737300007C
:10475000204F00006E2000005374000061740000C0
:10476000757300003A200000496E0000616300008C
:10477000746900007665000000000000CF02780038
:104780003220EF00C33C2200008041001040BA00FC
:104790000160EF000000060050610000737300002C
:1047A0002052000065730000706F00006E730000FF
:1047B00065200000537400006174000075730000F0
:1047C0003A200000506500006E640000696E000031
:1047D00067000000CF0278003220EF00833F220004
:1047E000008041001040BA000160EF0000000600A8
:1047F00050610000737300002052000065730000D8
:10480000706F00006E73000065200000537400009C
:1048100061740000757300003A20000049640000D4
:104820006C65000000000000CF0278003220EF002D
:1048300023422200008041001040BA000160EF00D6
:1048400000000600506100006E2F00005469000057
:104850006C74000020530000746100007475000047
:10486000733A000020410000637400006976000084
:1048700065000000CF0278003220EF008344220060
:10488000008041001040BA000160EF000000060007
:10489000506100006E2F0000546900006C7400002D
:1048A000205300007461000074750000733A00002A
:1048B00020490000646C000065000000CF02780011
:1048C0003220EF00C3462200008041001040BA00B1
:1048D0000160EF00000006005A6F00006F6D0000DD
:1048E000205300007461000074750000733A0000EA
:1048F000204100006374000069760000650000003C
:10490000CF0278003220EF00E3482200008041000F
:104910001040BA000160EF00000006005A6F00006E
:104920006F6D00002053000074610000747500007A
:10493000733A000020490000646C0000650000002C
:10494000CF0278003220EF00E34A220000804100CD
:104950001040BA000160EF00000006005054000053
:104960005A200000536500006E64000020530000D0
:1049700074610000746500003A200000506500007A
:104980006E640000696E000067000000CF027800CE
:104990003220EF00434D2200008041001040BA0059
:1049A0000160EF0000000600505400005A20000093
:1049B000536500006E640000205300007461000025
:1049C000746500003A200000496400006C65000036
:1049D00000000000CF0278003220EF00834F220059
:1049E000008041001040BA000160EF0000000600A6
:1049F00050720000657300006574000020500000D4
:104A0000726F000067720000616D0000204D0000B1
:104A10006F640000653A0000204F00006E00000047
:104A2000CF0278003220EF00E351220000804100E5
:104A30001040BA000160EF00000006005072000054
:104A4000657300006574000020500000726F000064
:104A500067720000616D0000204D00006F6400006F
:104A6000653A0000204F000066660000000000006C
:104A7000CF0278003220EF00635422000080410012
:104A80001040BA000160EF0000000600484400003A
:104A90002031000030380000307000002035000068
:104AA000392E000039340000487A00002000000050
:104AB000CF0278003220EF006356220000804100D0
:104AC0001040BA000160EF000000060048440000FA
:104AD0002031000030380000307000002035000028
:104AE000304800007A200000202000002000000054
:104AF000CF0278003220EF0063582200008041008E
:104B00001040BA000160EF000000060048440000B9
:104B100020310000303800003069000020350000EE
:104B2000392E000039340000487A000020000000CF
:104B3000CF0278003220EF00635A2200008041004B
:104B40001040BA000160EF00000006004844000079
:104B500020310000303800003069000020350000AE
:104B6000304800007A2000002020000020000000D3
:104B7000CF0278003220EF00635C22000080410009
:104B80001040BA000160EF00000006004844000039
:104B90002020000037320000307000002035000077
:104BA000392E000039340000487A0000200000004F
:104BB000CF0278003220EF00635E220000804100C7
:104BC0001040BA000160EF000000060048440000F9
:104BD0002020000037320000307000002035000037
:104BE000304800007A200000202000002000000053
:104BF000CF0278003220EF00636022000080410085
:104C00001040BA000160EF000000060048560000A6
:104C100020200000363400003078000020340000EE
:104C20003830000020360000304800007A000000D4
:104C3000CF0278003220EF00636222000080410042
:104C40001040BA000160EF00000006004856000066
:104C500020200000383000003078000020360000AE
:104C60003030000020360000304800007A0000009C
:104C7000CF0278003220EF00636422000080410000
:104C80001040BA000160EF00000006004856000026
:104C9000203100003032000034780000203700005E
:104CA0003638000020360000304800007A0000004E
:104CB000CF0278003220EF006366220000804100BE
:104CC0001040BA000160EF000000060048560000E6
:104CD000203100003238000030780000203700001A
:104CE0003638000020360000304800007A0000000E
:104CF000CF0278003220EF0063682200008041007C
:104D00001040BA000160EF000000060048560000A5
:104D100020310000323800003078000031300000CF
:104D20003234000020360000304800007A000000D5
:104D3000CF0278003220EF00636A22000080410039
:104D40001040BA000160EF00000006004856000065
:104D50002031000033360000367800002037000094
:104D60003638000020360000304800007A0000008D
:104D7000CF0278003220EF00636C220000804100F7
:104D80001040BA000160EF00000006004856000025
:104D90002031000034300000307800003130000055
:104DA0003530000020360000304800007A00000056
:104DB000CF0278003220EF00636E220000804100B5
:104DC0001040BA000160EF000000060048560000E5
:104DD0002031000036300000307800003132000011
:104DE0003030000020360000304800007A0000001B
:104DF000CF0278003220EF00637022000080410073
:104E00001040BA000160EF00000006002020000002
:104E10004E6F0000742000004176000061690000C0
:104E20006C610000626C0000652000002000000042
:104E3000CF0278003220EF00637222000080410030
:104E40001040BA000160EF00000006004856000064
:104E5000203100003932000030780000313200008B
:104E60003030000020360000304800007A0000009A
:104E7000CF0278003220EF006374220000804100EE
:104E80001040BA000160EF0000000600534400002B
:104E90002034000038300000692000003239000062
:104EA0002E390000374800007A2000002000000062
:104EB000CF0278003220EF006376220000804100AC
:104EC0001040BA000160EF000000060053440000EB
:104ED000204E00005453000043200000532D0000DA
:104EE00056690000646500006F200000200000008B
:104EF000CF0278003220EF0063782200008041006A
:104F00001040BA000160EF000000060053440000AA
:104F100020350000373600006920000032350000DF
:104F2000487A00002020000020200000200000001F
:104F3000CF0278003220EF00637A22000080410027
:104F40001040BA000160EF0000000600534400006A
:104F500020500000414C0000205300002D5600005E
:104F600069640000656F0000202000002000000040
:104F7000CF0278003220EF00637C220000804100E5
:104F80001040BA000160EF0000000600534400002A
:104F90002034000038300000692000007950000003
:104FA000625000007220000020200000200000005D
:104FB000CF0278003220EF00637E220000804100A3
:104FC0001040BA000160EF000000060053440000EA
:104FD000204E00005453000043200000436F0000A7
:104FE0006D7000006F7300006974000065000000C0
:104FF000CF0278003220EF00638022000080410061
:105000001040BA000160EF000000060053440000A9
:10501000203500003736000069200000795000007C
:1050200062500000722000002020000020000000DC
:10503000CF0278003220EF0063822200008041001E
:105040001040BA000160EF00000006005344000069
:1050500020500000414C0000204300006F6D000014
:10506000706F00007369000074650000200000008C
:10507000CF0278003220EF006384220000804100DC
:105080001040BA000160EF00000006004E6F000003
:105090006E65000000000000CF0278003220EF00B3
:1050A000A3852200008041001040BA000160EF009B
:1050B000000006000A0D0000553500005F490000A1
:1050C0005352000020250000325800002025000027
:1050D0003258000020250000325800002025000032
:1050E0003258000020250000325800000000000067
:1050F000CF0278003220EF00638822000080410058
:105100001040BA000160EF000000060055350000B5
:105110005F4200003020000049530000522D000083
:105120004572000072200000253200005820000067
:1051300025320000582000002532000058200000D1
:1051400025320000582000005B2500003258000086
:105150005D0A00000D000000CF0278003220EF0051
:10516000A38B2200008041001040BA000160EF00D4
:1051700000000600553500005F42000031200000AD
:1051800049530000522D00004572000072200000BB
:105190002532000058200000253200005820000071
:1051A00025320000582000005B2500003258000026
:1051B0005D20000025320000580A00000D000000AC
:1051C000CF0278003220EF00E38E22000080410001
:1051D0001040BA000160EF000000060055350000E5
:1051E0005F4200003320000049530000522D0000B0
:1051F0004572000072200000253200005820000097
:105200005B250000325800005D20000025320000C0
:1052100058200000253200005820000025320000F0
:10522000582000000A0D000000000000CF027800A6
:105230003220EF00E301200083015000050031001F
:1052400043932200008041001040BA000160EF004B
:1052500000000600409322008381410080814100CC
:105260001380BA00000006000A0D4C0055315800AA
:10527000303120005F49250053524C002025580052
:105280004C582000202525004C584C002020580068
:1052900055310A0030300D005F49000053520000C4
:1052A00020250000CF0278003220EF000396220074
:1052B000008041001040BA000160EF0000000600CD
:1052C0000A0D0000202D00002D200000446F00007A
:1052D0006E650000202D00002D0A00000D0000006A
:1052E000CF0278003220EF00E397220000804100D7
:1052F0001040BA000160EF00000006000A0D000037
:1053000055310000303000005F55000031300000A2
:10531000315F00004953000052200000507200002D
:105320006573000065740000733A000020000000FF
:10533000CF0278003220EF00639A22000080410003
:105340001040BA000160EF00000006000A0D0000E6
:10535000416300007469000076650000507200002F
:1053600065730000657400003D250000750A0000AB
:105370000D000000CF0278003220EF00839C220055
:10538000008041001040BA000160EF0000000600FC
:105390000A0D0000466900007273000074200000CE
:1053A000537400006570000000000000CF02780018
:1053B0003220EF00439E2200008041001040BA00DE
:1053C0000160EF00000006000A0D00002846000002
:1053D00053290000536B000069700000207000002A
:1053E00072650000736500007420000025750000E0
:1053F000206100006374000069760000652E0000E3
:1054000000000000CF0278003220EF0003A122004C
:10541000008041001040BA000160EF00000006006B
:105420000A0D0000284600005329000050720000B9
:1054300065730000657400002025000075200000E1
:10544000736500006C650000637400006564000013
:105450002E000000CF0278003220EF0083A322004C
:10546000008041001040BA000160EF00000006001B
:105470000A0D00004C61000073740000205300000E
:105480007465000070000000CF0278003220EF0049
:1054900023A52200008041001040BA000160EF0007
:1054A000000006000A0D0000284C000053290000EF
:1054B000536B0000697000002070000072650000EE
:1054C0007365000074200000257500002061000055
:1054D0006374000069760000652E00000000000083
:1054E000CF0278003220EF00E3A7220000804100C5
:1054F0001040BA000160EF00000006000A0D000035
:10550000284C000053290000507200006573000011
:105510006574000020250000752000007365000000
:105520006C65000063740000656400002E000000DC
:10553000CF0278003220EF0063AA220000804100F1
:105540001040BA000160EF00000006000A0D0000E4
:10555000284C000053290000536B000069700000C4
:105560002050000072650000736500007473000035
:105570002025000075200000257500002073000024
:10558000656C00006563000074650000642E000017
:1055900000000000CF0278003220EF0083AD22002F
:1055A000008041001040BA000160EF0000000600DA
:1055B0000A0D00004D7500006C74000069200000A9
:1055C000537400006570000000000000CF027800F6
:1055D0003220EF0043AF2200008041001040BA00AB
:1055E0000160EF00000006000A0D0000284D0000D9
:1055F000532900006E70000020500000726500000A
:105600007365000074200000257500002073000001
:10561000656C00006563000074650000642E000086
:1056200000000000CF0278003220EF0003B2220019
:10563000008041001040BA000160EF000000060049
:105640000A0D0000536B000069700000284D000037
:1056500053290000706D00002050000072650000AA
:10566000736500007420000025750000202E0000E6
:1056700000000000CF0278003220EF0083B4220047
:10568000008041001040BA000160EF0000000600F9
:105690000A0D0000536B000069700000284D0000E7
:1056A000532900002050000072650000736500005F
:1056B00074200000257500002025000075200000E2
:1056C000282500007529000020530000616D0000AE
:1056D000652E000000000000CF0278003220EF00AD
:1056E000A3B72200008041001040BA000160EF0023
:1056F000000006000A0D0000536B000069700000F6
:10570000284D000053290000205000007265000061
:10571000736500007420000025750000202500003E
:105720007520000028250000752900002053000086
:10573000656C00006563000074650000642E000065
:1057400000000000CF0278003220EF0003BB2200EF
:10575000008041001040BA000160EF000000060028
:105760000A0D0000536B000069700000284D000016
:10577000532900002050000072650000736500008E
:1057800074200000257500002020000053650000F3
:105790006C65000063740000656400002E0000006A
:1057A000CF0278003220EF00E3BD220000804100EC
:1057B0001040BA000160EF00000006000A0D000072
:1057C000536B000069700000284D00005329000051
:1057D0006E610000205000007265000073650000DB
:1057E00074200000257500002025000075200000B1
:1057F000536500006C650000637400006564000080
:105800002E000000CF0278003220EF00C3012000FC
:10581000830150000500310003C2220000804100D6
:105820001040BA000160EF000000060000C2220034
:1058300083814100808141001380BA00000006008E
:105840000A0D2500284D75005329290020502000FD
:10585000726553007365650074206C005B256500FC
:10586000755D6300205B7400257565005D20640034
:1058700025752E0020280000CF0278003220EF008E
:10588000E30120008301500005003100A3C5220080
:10589000008041001040BA000160EF0000000600E7
:1058A000A0C5220083814100808141001380BA009D
:1058B000000006000A0D7500284D2900532920001C
:1058C000205053007265650073656C00742065009C
:1058D0005B256300755D74002025650075206400FC
:1058E000205B2E00257500005D20000028250000AB
:1058F000CF0278003220EF00E30120008301500046
:105900000500310063C92200008041001040BA0048
:105910000160EF000000060060C9220083814100A1
:10592000808141001380BA00000006000A0D750056
:10593000284D29005329200020505300726565002E
:1059400073656C007420650025756300205B74002E
:10595000257565005D206400205B2E002575000024
:105960005D20000028250000CF0278003220EF00E3
:1059700023022000830150000500310023CD2200C6
:10598000008041001040BA000160EF0000000600F6
:1059900020CD220083814100808141001380BA0024
:1059A000000006000A0D7300284D6500532974009D
:1059B000204D2000756C2500746975002D50200065
:1059C0007265250073657500742020006E6F2500D8
:1059D000742075004163200074692E007665000014
:1059E0002050000072650000CF0278003220EF00E6
:1059F00043022000830150000500310023D1220022
:105A0000008041001040BA000160EF000000060075
:105A100020D1220083814100808141001380BA009F
:105A2000000006000A0D2000284D250053297500AE
:105A3000204D2000756C5B00746925002D507500A9
:105A400072655D0073652000742020006E6F5B003E
:105A500074202500666F7500756E5D00642020005F
:105A600050722E006573000065740000CF0278004C
:105A70003220EF0023022000830150000500310096
:105A800043D52200008041001040BA000160EF00C1
:105A90000000060040D52200838141008081410042
:105AA0001380BA00000006000A0D5D00284D20009A
:105AB00053292500206E75006F742000204D2000B2
:105AC000756C2500746975002D50200072652800E2
:105AD00073652500742075005072290065732E00CF
:105AE00065740000205B000025750000CF0278007F
:105AF0003220EF0023022000830150000500310016
:105B000043D92200008041001040BA000160EF003C
:105B10000000060040D922008381410080814100BD
:105B20001380BA00000006000A0D5B00284D250016
:105B300053297500206E5D006F742000204D2000F9
:105B4000756C2500746975002D5020007265280061
:105B500073652500742075005072290065732E004E
:105B6000657400002025000075200000CF02780039
:105B70003220EF0023022000830150000500310095
:105B800043DD2200008041001040BA000160EF00B8
:105B90000000060040DD2200838141008081410039
:105BA0001380BA00000006000A0D2500284D75007C
:105BB00053292000206E20006F745B00204D2500CB
:105BC000756C750074695D002D50200072652800A9
:105BD00073652500742075005072290065732E00CE
:105BE000657400002025000075200000CF027800B9
:105BF0003220EF0003032000830150000500310034
:105C000043E12200008041001040BA000160EF0033
:105C10000000060040E122008381410080814100B4
:105C20001380BA00000006000A0D74004E6F650074
:105C300020532E007465530070207900696473004E
:105C4000656E74007469650066696D006564460080
:105C5000206E6C00416361007469670076653100F5
:105C60005374200065703D00203D25002532320030
:105C7000782C780043750A0072720D00656E000082
:105C80007453000074610000CF0278003220EF00EE
:105C900023E52200008041001040BA000160EF00BF
:105CA00000000600204E00006F7400002046000037
:105CB0006F7500006E6400000A0D00000000000017
:105CC000CF0278003220EF00E3E62200008041009E
:105CD0001040BA000160EF00000006002042000002
:105CE000746E000028250000327800002F25000087
:105CF000752900002D47000072700000312000005F
:105D00000A0D000000000000CF0278003220EF00F2
:105D100023E92200008041001040BA000160EF003A
:105D200000000600202000004D6100007374000098
:105D300065720000205000006F770000657200005F
:105D4000204F00006666000020000000CF027800AF
:105D50003220EF0043EB2200008041001040BA00E7
:105D60000160EF0000000600202000004D610000EF
:105D70007374000065720000205000006F7700000F
:105D800065720000204F00006E200000200000001F
:105D9000CF0278003220EF0063ED22000080410046
:105DA0001040BA000160EF00000006002043000030
:105DB00075740000204F00006E0A00000D00000006
:105DC000CF0278003220EF00E3EE22000080410095
:105DD0001040BA000160EF00000006002020000023
:105DE000202000002020000020200000437500003B
:105DF000742000002020000020200000202000004F
:105E000020000000CF0278003220EF0003F12200D2
:105E1000008041001040BA000160EF000000060061
:105E20002057000069700000652000004F6E0000E0
:105E30000A0D000000000000CF0278003220EF00C1
:105E4000A3F22200008041001040BA000160EF0080
:105E5000000006002020000020200000202000007C
:105E6000202000005769000070650000202000001D
:105E7000202000002020000020000000CF02780039
:105E80003220EF00C3F42200008041001040BA002D
:105E90000160EF0000000600204D0000697800005E
:105EA000204F00006E0A00000D000000CF027800B5
:105EB0003220EF0043F62200008041001040BA007B
:105EC0000160EF00000006002020000020200000FC
:105ED0002020000020200000204D000069780000F4
:105EE00020200000202000002020000020000000D2
:105EF000CF0278003220EF0063F8220000804100DA
:105F00001040BA000160EF0000000600204D0000C4
:105F1000756C000074690000205300007465000077
:105F2000702000004F6E00000A0D0000000000000D
:105F3000CF0278003220EF0063FA22000080410097
:105F40001040BA000160EF000000060020200000B1
:105F500020200000204D0000756C000074690000D6
:105F60002053000074650000702000002020000015
:105F700020000000CF0278003220EF0083FC2200D6
:105F8000008041001040BA000160EF0000000600F0
:105F9000204C000061730000742000005374000066
:105FA00065700000204F00006E0A00000D00000028
:105FB000CF0278003220EF0063FE22000080410013
:105FC0001040BA000160EF00000006002020000031
:105FD00020200000204C00006173000074200000AD
:105FE0005374000065700000202000002020000095
:105FF00020000000CF0278003220EF008300230051
:10600000008041001040BA000160EF00000006006F
:1060100020460000697200007374000020530000E5
:1060200074650000702000004F6E00000A0D000033
:1060300000000000CF0278003220EF00830223002E
:10604000008041001040BA000160EF00000006002F
:10605000202000002020000020460000697200007F
:10606000737400002053000074650000702000006D
:106070002020000020000000CF0278003220EF0036
:10608000A3042300008041001040BA000160EF002B
:10609000000006002020000020200000205000000A
:1060A000726F000067720000616D0000204F0000F9
:1060B000666600002020000020000000CF0278006B
:1060C0003220EF00C3062300008041001040BA00D8
:1060D0000160EF000000060020500000726F000019
:1060E00067720000616D0000204F000066660000CE
:1060F0000A0D000000000000CF0278003220EF00FF
:10610000A3082300008041001040BA000160EF00A6
:106110000000060020200000202000002050000089
:10612000726F000067720000616D0000204F000078
:106130006E2000002020000020000000CF02780028
:106140003220EF00C30A2300008041001040BA0053
:106150000160EF000000060020500000726F000098
:1061600067720000616D0000204F00006E0A0000A1
:106170000D000000CF0278003220EF00830C2300D6
:10618000008041001040BA000160EF0000000600EE
:106190002050000072650000736500007444000028
:1061A00069730000616200006C650000204F000010
:1061B0006666000020000000CF0278003220EF0069
:1061C000A30E2300008041001040BA000160EF00E0
:1061D000000006002050000072650000736500009A
:1061E0007444000069730000616200006C65000087
:1061F000204F0000666600000A0D0000000000004D
:10620000CF0278003220EF00E3102300008041002D
:106210001040BA000160EF000000060020500000AE
:10622000726500007365000074440000697300002B
:10623000616200006C650000204F00006E200000CD
:1062400020000000CF0278003220EF00031323006B
:10625000008041001040BA000160EF00000006001D
:106260002050000072650000736500007444000057
:1062700069730000616200006C650000204F00003F
:106280006E0A00000D000000CF0278003220EF00FF
:1062900023152300008041001040BA000160EF0088
:1062A0000000060020200000504700004D200000A4
:1062B0004D6F000064650000204100006374000021
:1062C000697600006520000020000000CF02780001
:1062D0003220EF0043172300008041001040BA0035
:1062E0000160EF000000060020420000746E000014
:1062F00028250000327800002F25000075290000B5
:106300002D4700007270000033000000CF027800BB
:106310003220EF0043192300008041001040BA00F2
:106320000160EF0000000600204900006E700000D0
:1063300075740000203600000A0D00000000000007
:10634000CF0278003220EF00E31A230000804100E2
:106350001040BA000160EF0000000600202000009D
:106360002020000020200000496E00007075000011
:1063700074200000362000002020000020200000B3
:1063800020000000CF0278003220EF00031D230020
:10639000008041001040BA000160EF0000000600DC
:1063A000204900006E700000757400002035000068
:1063B0000A0D000000000000CF0278003220EF003C
:1063C000A31E2300008041001040BA000160EF00CE
:1063D00000000600202000002020000020200000F7
:1063E000496E000070750000742000003520000028
:1063F000202000002020000020000000CF027800B4
:106400003220EF00C3202300008041001040BA007A
:106410000160EF0000000600204900006E700000DF
:1064200075740000203400000A0D00000000000018
:10643000CF0278003220EF00632223000080410069
:106440001040BA000160EF000000060020200000AC
:106450002020000020200000496E00007075000020
:1064600074200000342000002020000020200000C4
:1064700020000000CF0278003220EF0083242300A8
:10648000008041001040BA000160EF0000000600EB
:10649000204900006E700000757400002033000079
:1064A0000A0D000000000000CF0278003220EF004B
:1064B00023262300008041001040BA000160EF0055
:1064C0000000060020200000202000002020000006
:1064D000496E000070750000742000003320000039
:1064E000202000002020000020000000CF027800C3
:1064F0003220EF0043282300008041001040BA0002
:106500000160EF0000000600204900006E700000EE
:1065100075740000203200000A0D00000000000029
:10652000CF0278003220EF00E329230000804100F1
:106530001040BA000160EF000000060020200000BB
:106540002020000020200000496E0000707500002F
:1065500074200000322000002020000020200000D5
:1065600020000000CF0278003220EF00032C23002F
:10657000008041001040BA000160EF0000000600FA
:10658000204900006E70000075740000203100008A
:106590000A0D000000000000CF0278003220EF005A
:1065A000A32D2300008041001040BA000160EF00DD
:1065B0000000060020200000202000002020000015
:1065C000496E00007075000074200000312000004A
:1065D000202000002020000020000000CF027800D2
:1065E0003220EF00C32F2300008041001040BA008A
:1065F0000160EF000000060020500000495000003C
:10660000204F00006E0A00000D000000CF0278004D
:106610003220EF0043312300008041001040BA00D7
:106620000160EF0000000600202000002020000094
:106630002020000050490000502000004F6E000054
:10664000202000002020000020200000200000006A
:10665000CF0278003220EF00633323000080410036
:106660001040BA000160EF0000000600205000005A
:1066700049500000204F0000666600000A0D00002F
:1066800000000000CF0278003220EF000335230025
:10669000008041001040BA000160EF0000000600D9
:1066A0002020000020200000202000005049000091
:1066B000502000004F6600006620000020200000EF
:1066C0002020000020000000CF0278003220EF00E0
:1066D00023372300008041001040BA000160EF0022
:1066E0000000060020500000495000002043000038
:1066F000686100006E670000653A000020460000F7
:106700006F72000065670000726F0000756E000018
:10671000640A00000D000000CF0278003220EF0074
:10672000A3392300008041001040BA000160EF004F
:106730000000060050430000686100006E67000022
:1067400065200000466F000072650000677200005F
:106750006F7500006E64000000000000CF0278003A
:106760003220EF00C33B2300008041001040BA00FC
:106770000160EF00000006002050000049500000BA
:1067800020430000686100006E670000653A000069
:1067900020420000616300006B670000726F000020
:1067A000756E0000640A00000D000000CF02780042
:1067B0003220EF00433E2300008041001040BA0029
:1067C0000160EF0000000600504300006861000017
:1067D0006E6700006520000042610000636B0000EE
:1067E000677200006F7500006E640000000000001A
:1067F000CF0278003220EF00634023000080410088
:106800001040BA000160EF0000000600436F000076
:106810006E740000726F00006C5600004945000065
:10682000572000005848000044250000730A00006B
:106830000D000000CF0278003220EF0083422300D9
:10684000008041001040BA000160EF000000060027
:106850002020000020200000436F00006D70000029
:10686000696C0000656400003A2000002573000098
:106870002061000074200000257300000A0D000054
:1068800000000000CF0278003220EF000345230013
:10689000008041001040BA000160EF0000000600D7
:1068A000303600002D4A0000616E00002D310000DE
:1068B00030000000CF0278003220EF008346230032
:1068C000008041001040BA000160EF0000000600A7
:1068D000313500003A350000303A0000323900000E
:1068E00000000000CF0278003220EF0003482300B0
:1068F000008041001040BA000160EF000000060077
:1069000020460000696E0000646900006E670000A8
:1069100020430000616D000065720000617300009B
:1069200000000000CF0278003220EF00034A23006D
:10693000008041001040BA000160EF000000060036
:1069400020200000205200006573000065740000E4
:106950002056000069640000656F000020200000E0
:1069600000000000CF0278003220EF00034C23002B
:10697000008041001040BA000160EF0000000600F6
:10698000204300006C65000061720000696E000029
:1069900067200000507200006573000065740000FD
:1069A00073000000CF0278003220EF00034E230076
:1069B000008041001040BA000160EF0000000600B6
:1069C000204300006C65000061720000696E0000E9
:1069D00067200000416C00006C20000020200000B7
:1069E00000000000CF0278003220EF0003502300A7
:1069F000008041001040BA000160EF000000060076
:106A00002052000065730000746100007274000081
:106A10002053000079730000746500006D200000B1
:106A200000000000CF0278003220EF000352230064
:106A3000008041001040BA000160EF000000060035
:106A4000456E0000616200006C6500002048000097
:106A50006F7300007420000053650000726900002D
:106A6000616C000000000000CF0278003220EF00CF
:106A700023542300008041001040BA000160EF0061
:106A8000000006004469000073610000626C0000B1
:106A9000652000005365000072690000616C000011
:106AA000202000002020000000000000CF0278001D
:106AB0003220EF0043562300008041001040BA000E
:106AC0000160EF00000006000A0D0000436F0000A7
:106AD0006D6D0000616E000064200000436F0000D7
:106AE0006D7000006C650000746500000A0D000008
:106AF0003E000000CF0278003220EF0083582300D0
:106B0000008041001040BA000160EF000000060064
:106B1000202000002053000061760000696E000014
:106B200067200000436F00006E6600006967000088
:106B30002020000000000000CF0278003220EF008B
:106B4000A35A2300008041001040BA000160EF000A
:106B5000000006002020000053680000757400004B
:106B6000646F0000776E0000204100006374000035
:106B7000697600006520000000000000CF02780068
:106B80003220EF00C35C2300008041001040BA00B7
:106B90000160EF000000060020430000616D00006E
:106BA0006572000061200000506F000077650000F2
:106BB000726400006F7700006E200000000000008B
:106BC000CF0278003220EF00E35E23000080410016
:106BD0001040BA000160EF000000060020420000F3
:106BE000746E000028250000327800002F25000078
:106BF000752900002D47000072700000352000004C
:106C00000A0D000000000000CF0278003220EF00E3
:106C100023612300008041001040BA000160EF00B2
:106C200000000600507200006F63000065730000F2
:106C3000732000005072000065730000657400004E
:106C40002042000075740000746F00006E20000088
:106C5000257500000A0D000000000000CF0278003A
:106C60003220EF00C3632300008041001040BA00CF
:106C70000160EF0000000600566100006C69000032
:106C8000642000005072000065730000657400000D
:106C900020250000750A00000D000000CF027800DA
:106CA0003220EF00C3652300008041001040BA008D
:106CB0000160EF00000006005072000065730000E4
:106CC000657400002025000033750000205400008A
:106CD0006F200000486900006768000000000000A5
:106CE000CF0278003220EF00E367230000804100EC
:106CF0001040BA000160EF00000006005072000072
:106D000065730000657400002025000075200000F8
:106D1000746F00002068000069670000680A0000C6
:106D20000D000000CF0278003220EF00036A23003C
:106D3000008041001040BA000160EF000000060032
:106D4000507200006F670000726100006D2000004B
:106D50004D6F0000646500000A0D00000000000097
:106D6000CF0278003220EF00E36B23000080410067
:106D70001040BA000160EF00000006004D750000F1
:106D80006C7400006953000074650000700A000014
:106D90000D000000CF0278003220EF00836D230049
:106DA000008041001040BA000160EF0000000600C2
:106DB000466900007273000074530000746500009F
:106DC000700A00000D000000CF0278003220EF00B2
:106DD000236F2300008041001040BA000160EF00E3
:106DE000000006004C610000737400005374000042
:106DF000657000000A0D000000000000CF0278005E
:106E00003220EF00C3702300008041001040BA0020
:106E10000160EF0000000600534500004C31000007
:106E200032200000436100006D2800002532000080
:106E300078290000204900006E700000282500001D
:106E40003278000029200000504300004328000051
:106E500025320000782900000D0A00000000000023
:106E6000CF0278003220EF00E3732300008041005E
:106E70001040BA000160EF000000060053740000EB
:106E80006F72000065200000507200006573000002
:106E900065740000284F00006E6C0000792000002F
:106EA000506F00007274000029200000257500005A
:106EB000204300006F6D0000706C000065740000DE
:106EC000650A00000D000000CF0278003220EF00BC
:106ED00023772300008041001040BA000160EF00DA
:106EE000000006002A500000726500007365000073
:106EF000742000002533000075200000537400004A
:106F00006F7200006564000000000000CF0278008E
:106F10003220EF0043792300008041001040BA0086
:106F20000160EF00000006002052000065740000C0
:106F3000726900006576000065200000536500005E
:106F400074740000696E00006773000000000000A8
:106F5000CF0278003220EF00637B230000804100E5
:106F60001040BA000160EF00000006004765000015
:106F700074200000436100006D6500007261000034
:106F80002044000061740000610A00000D00000050
:106F9000CF0278003220EF00637D230000804100A3
:106FA0001040BA000160EF0000000600205300000E
:106FB000746F0000726500002050000072650000D0
:106FC0007365000074200000253300007520000068
:106FD00000000000CF0278003220EF00837F230002
:106FE000008041001040BA000160EF000000060080
:106FF00020500000726500007365000074200000DE
:107000002533000075200000537400006F720000EB
:107010006564000000000000CF0278003220EF001D
:10702000A3812300008041001040BA000160EF00FE
:1070300000000600537400006F720000652000001D
:107040005072000065730000657400002025000088
:1070500075200000436F00006D7000006C6500003B
:10706000746500000A0D000000000000CF027800E7
:107070003220EF0043842300008041001040BA001A
:107080000160EF0000000600205000007265000063
:107090007365000074200000253300007520000097
:1070A00046610000696C000065640000000000009B
:1070B000CF0278003220EF00638623000080410079
:1070C0001040BA000160EF00000006005374000099
:1070D0006F720000652000005072000065730000B0
:1070E0006574000020250000752000004661000046
:1070F000696C0000656400000A0D000000000000DB
:10710000CF0278003220EF00E388230000804100A6
:107110001040BA000160EF0000000600507200004D
:107120006573000065740000204D00006F6400006E
:10713000650A00000D000000CF0278003220EF0049
:10714000A38A2300008041001040BA000160EF00D4
:10715000000006002020000052650000616400006D
:10716000205000007265000073650000742000006C
:10717000253300007520000000000000CF027800D9
:107180003220EF00C38C2300008041001040BA0081
:107190000160EF00000006005072000065730000FF
:1071A000657400002025000075200000666F000057
:1071B000756E0000640A00000D000000CF02780028
:1071C0003220EF00C38E2300008041001040BA003F
:1071D0000160EF00000006005072000065730000BF
:1071E0006574000020250000752000004C6100003F
:1071F0007374000053740000657000000A0D0000F5
:1072000000000000CF0278003220EF00039123003D
:10721000008041001040BA000160EF00000006004D
:1072200050720000657300006574000020250000A6
:10723000752000004669000072730000745300005E
:1072400074650000700A00000D000000CF02780095
:107250003220EF0043932300008041001040BA0029
:107260000160EF000000060050720000657300002E
:107270006574000020250000752000004D75000099
:107280006C7400006953000074650000700A00000F
:107290000D000000CF0278003220EF00839523001C
:1072A000008041001040BA000160EF0000000600BD
:1072B0005072000065730000657400002025000016
:1072C0007520000028530000746500007050000015
:1072D0006F73000073690000626C00006529000094
:1072E000506F000073730000696200006C6500005D
:1072F0000A0D000000000000CF0278003220EF00ED
:10730000A3982300008041001040BA000160EF0004
:1073100000000600534500004C31000033200000FF
:10732000436100006D28000025320000782900002C
:10733000204900006E70000028250000327800000F
:10734000292000005043000043280000253200009F
:10735000782900000D0A000000000000CF0278002C
:107360003220EF00C39B2300008041001040BA0090
:107370000160EF000000060050720000657300001D
:1073800065740000202500007520000043610000A6
:107390006D65000072610000204600006F750000FE
:1073A0006E6400000A0D000000000000CF027800AB
:1073B0003220EF00439E2300008041001040BA00BD
:1073C0000160EF0000000600202000005570000062
:1073D00064610000746900006E67000020430000D3
:1073E000616D000065720000612000000000000077
:1073F000CF0278003220EF0063A02300008041001C
:107400001040BA000160EF00000006004361000078
:107410006D2000004E6F0000744100007661000096
:10742000696C000020500000726500007365000068
:107430007420000025750000200A00000D000000E7
:10744000CF0278003220EF00E3A223000080410049
:107450001040BA000160EF00000006004E6F00000F
:10746000436100006D200000507200006573000051
:107470006574000020250000752000000A0D000042
:1074800000000000CF0278003220EF0003A52300A7
:10749000008041001040BA000160EF0000000600CB
:1074A000534500004C3100003420000043610000CF
:1074B0006D280000253200007829000020490000D6
:1074C0006E7000002825000032780000292000009E
:1074D00050430000432800002532000078290000B6
:1074E0000D0A000000000000CF0278003220EF00FB
:1074F00023A82300008041001040BA000160EF0083
:107500000000060020200000204E00006F20000038
:1075100050720000657300006574000020250000B3
:10752000337500002020000000000000CF0278002A
:107530003220EF0043AA2300008041001040BA002F
:107540000160EF000000060050720000657300004B
:107550006574000020250000752000004E6F0000BB
:1075600074200000466F0000756E0000640A000081
:107570000D000000CF0278003220EF0083AC230022
:10758000008041001040BA000160EF0000000600DA
:10759000536B0000697000002D460000532000006E
:1075A0005072000065730000657400002025000023
:1075B000752000004E6F000074200000466F000030
:1075C000756E0000640A00000D000000CF02780014
:1075D0003220EF0043AF2300008041001040BA008A
:1075E0000160EF00000006005072000065730000AB
:1075F00065740000204400006973000061620000AF
:107600006C650000640A00000D000000CF027800E5
:107610003220EF0043B12300008041001040BA0047
:107620000160EF00000006002050000072650000BD
:10763000736500007473000020440000697300004B
:10764000616200006C650000642000002000000002
:10765000CF0278003220EF0063B3230000804100A6
:107660001040BA000160EF00000006000A0D0000A3
:10767000436800006B540000726100006E5400000B
:10768000696D0000654500006E6300006F640000D6
:107690006572000028250000303400004C7800009E
:1076A00029000000CF0278003220EF0003B623004B
:1076B000008041001040BA000160EF0000000600A9
:1076C00020540000726100006E540000696D0000DB
:1076D00065200000256300002E25000063300000B7
:1076E000207300006563000000000000CF027800F6
:1076F0003220EF0043B82300008041001040BA0060
:107700000160EF00000006000A0D00004368000061
:107710006B5A00006F6F00006D4500006E63000043
:107720006F640000657200002825000030340000FE
:107730004C78000029000000CF0278003220EF00D2
:10774000A3BA2300008041001040BA000160EF009E
:1077500000000600202000004D610000782000009D
:107760005A6F00006F6D00002025000075000000BA
:10777000CF0278003220EF0063BC2300008041007C
:107780001040BA000160EF00000006000A0D000082
:10779000436800006B500000616E0000456E000001
:1077A000636F00006465000072280000253000004F
:1077B000344C00007829000000000000CF0278005F
:1077C0003220EF00C3BE2300008041001040BA0009
:1077D0000160EF0000000600202000004D61000065
:1077E00078200000506100006E2000002575000028
:1077F00000000000CF0278003220EF0083C0230099
:10780000008041001040BA000160EF000000060057
:107810000A0D0000436800006B540000696C000012
:10782000744500006E6300006F6400006572000024
:1078300028250000303400004C78000029000000AA
:10784000CF0278003220EF00E3C223000080410025
:107850001040BA000160EF00000006002020000088
:107860004D61000078200000546900006C74000035
:107870002025000075000000CF0278003220EF00C4
:10788000A3C42300008041001040BA000160EF0053
:10789000000006000A0D0000436800006B4600006F
:1078A0006F63000075730000456E0000636F000099
:1078B000646500007228000025300000344C000090
:1078C0007829000000000000CF0278003220EF008D
:1078D00023C72300008041001040BA000160EF0080
:1078E000000006000A0D0000436800006B4900001C
:1078F00072690000735000006F730000456E000055
:10790000636F0000646500007228000025300000ED
:10791000344C00007829000000000000CF027800FD
:107920003220EF00C3C92300008041001040BA009C
:107930000160EF00000006000A0D0000436800002F
:107940006B52000065640000456E0000636F00002C
:10795000646500007228000025300000344C0000EF
:107960007829000000000000CF0278003220EF00EC
:1079700023CC2300008041001040BA000160EF00DA
:10798000000006000A0D0000436800006B42000082
:107990006C750000654500006E6300006F640000B8
:1079A0006572000028250000303400004C7800008B
:1079B00029000000CF0278003220EF0083CE2300A0
:1079C000008041001040BA000160EF000000060096
:1079D0000A0D0000436800006B440000657400005D
:1079E000616900006C4500006E6300006F64000078
:1079F0006572000028250000303400004C7800003B
:107A000029000000CF0278003220EF0003D12300CC
:107A1000008041001040BA000160EF000000060045
:107A20000A0D0000436800006B4700006169000018
:107A30006E5000006F730000456E0000636F000021
:107A4000646500007228000025300000344C0000FE
:107A50007829000000000000CF0278003220EF00FB
:107A6000A3D32300008041001040BA000160EF0062
:107A7000000006003E250000732000004E6F00004D
:107A800074200000466F0000756E0000640A00005C
:107A90000D3E000000000000CF0278003220EF0011
:107AA000A3D52300008041001040BA000160EF0020
:107AB00000000600436F00006D700000696C00005C
:107AC000656400003A20000025730000206100007A
:107AD00074200000257300000A0D00000000000063
:107AE000CF0278003220EF00E30120008301500034
:107AF00005003100E3D82300008041001040BA00A7
:107B00000160EF0000000600E0D8230083814100FF
:107B1000808141001380BA00000006000D0A500069
:107B20005379720073746500656D730020536500AE
:107B30006574740074693A006E672000733A25001A
:107B40000A0D64000A0D0A0044650D00666100001C
:107B5000756C000074200000CF0278003220EF0026
:107B6000A3DB2300008041001040BA000160EF0059
:107B700000000600416300007469000076650000A3
:107B800020430000616D000065720000613A000052
:107B900020250000730A00000D000000CF027800CD
:107BA0003220EF00C3DD2300008041001040BA0006
:107BB0000160EF0000000600436100006D650000F9
:107BC0007261000020530000656C000065630000D6
:107BD000743A000020250000750A00000D00000026
:107BE000CF0278003220EF00E3DF23000080410065
:107BF0001040BA000160EF000000060020490000BC
:107C00006E7000007574000020530000656C000069
:107C100065630000743A000020250000750A00002A
:107C20000D000000CF0278003220EF0003E22300B5
:107C3000008041001040BA000160EF000000060023
:107C40000D0A000057690000706500002044000024
:107C500065730000637200006970000074690000C1
:107C60006F6E00003A200000257300000A0D00002E
:107C700000000000CF0278003220EF0083E42300F0
:107C8000008041001040BA000160EF0000000600D3
:107C90000D0A00005049000050200000446500001B
:107CA000736300007269000070740000696F000067
:107CB0006E3A000020250000730A00000D0000004D
:107CC000CF0278003220EF00E3E62300008041007D
:107CD0001040BA000160EF00000006000D0A00002D
:107CE000504900005020000043680000616E000011
:107CF000676500003A200000257300000A0D0000AF
:107D000000000000CF0278003220EF0003E92300DA
:107D1000008041001040BA000160EF000000060042
:107D20004F7500007470000075740000204600005C
:107D30006F7200006D610000743A000020250000A1
:107D4000730A00000D000000CF0278003220EF001F
:107D500023EB2300008041001040BA000160EF00D7
:107D600000000600506F0000727400002025000023
:107D700075200000496E000070750000742000003E
:107D8000466F0000726D0000617400003A20000030
:107D9000257300000A0D000000000000CF027800EB
:107DA0003220EF0043032000830150000500310022
:107DB000C3EE2300008041001040BA000160EF00D4
:107DC00000000600C0EE2300838141008081410055
:107DD0001380BA00000006000A0D610050616E00B9
:107DE0006E532000706554006564690020206D00AA
:107DF00020206500546920006C74200053705000EE
:107E00006565610064206E00202065005A6F6C007B
:107E10006F6D200053704C00656569006420670039
:107E200020496800646C74006520730052650A0084
:107E300074750D00726E0000202000005472000066
:107E4000CF0278003220EF00E302200083015000CF
:107E500005003100E3F32300008041001040BA0028
:107E60000160EF0000000600E0F323008381410081
:107E7000808141001380BA0000000600202020000D
:107E80002025200064202000202020002020200029
:107E900020202500202075002020200025642000BF
:107EA0002020200020202000202020002020200052
:107EB00020202000256420002020200020202500F4
:107EC0002020640020200A0020200D0025640A00E4
:107ED00020200D0020200000CF0278003220EF008B
:107EE000A3F72300008041001040BA000160EF00BA
:107EF000000006000A0D00005072000065730000CB
:107F000065740000733A00000A0D00000A0D0000BD
:107F100000000000CF0278003220EF00E3022000D2
:107F2000830150000500310083FA230000804100E6
:107F30001040BA000160EF000000060080FA230044
:107F400083814100808141001380BA000000060057
:107F500050725A0065206F0053726F0063206D00ED
:107F60004D6F2000646520006C20540020207200BA
:107F70002020610020206E0020207300202020009F
:107F8000202020002020460020206C0020206100BE
:107F900020506700616E7300202020002020200008
:107FA00054690A006C740D0020200000CF02780094
:107FB0003220EF0043FE2300008041001040BA0051
:107FC0000160EF00000006004F6E00006C790000B9
:107FD00020540000726100006E730000697400009C
:107FE000696F00006E2000002020000020000000CB
:107FF000CF0278003220EF002302200083015000DE
:108000000500310063012400008041001040BA00E7
:108010000160EF0000000600600124008381410040
:10802000808141001380BA00000006002533320031
:1080300064205800202520006420200020252000F6
:10804000313820007320200020202500254C3200EC
:1080500058205800202520004C58200020200A00DD
:10806000254C0D0058200000202000002025000095
:10807000CF0278003220EF0063042400008041002A
:108080001040BA000160EF00000006000A0D000079
:108090005043000043200000507200006573000050
:1080A00065740000733A00000A0D00000A0D00001C
:1080B00000000000CF0278003220EF0063032000B0
:1080C0008301500005003100830724000080410037
:1080D0001040BA000160EF00000006008007240095
:1080E00083814100808141001380BA0000000600B6
:1080F000436172006D20690050727300652020009A
:108100004D6F2000646547006C20610020206900ED
:1081100020206E002020200020202000202052005F
:108120002020650020506400616E20002020200087
:108130002020200020544200696C6C0074207500DF
:10814000205A65006F6F20006D20440020466500B6
:108150006F63740075732E0020490000CF02780011
:108160003220EF00C30B2400008041001040BA0011
:108170000160EF0000000600205B00004972000073
:10818000697300002C4600006F63000075730000E7
:108190002C410000574200002C200000424C0000FF
:1081A000435D000020540000726100006E73000007
:1081B00020200000466C000061670000730A000088
:1081C0000D0A00000D000000CF0278003220EF0001
:1081D000C302200083015000050031002310240059
:1081E000008041001040BA000160EF00000006006E
:1081F0002010240083814100808141001380BA0057
:1082000000000600202558006420200020252000C2
:108210003264250020204C0025315800387320009E
:10822000255820002558250025584C0020205800AE
:10823000254C200058202000202525004C583200D5
:1082400020204C00254C58005820200020252000DC
:108250004C58200020202000254C0000CF02780040
:108260003220EF00C3132400008041001040BA0008
:108270000160EF00000006004F6E000020200000AB
:1082800020000000CF0278003220EF000315240008
:10829000008041001040BA000160EF0000000600BD
:1082A0004F6600006620000020000000CF0278002A
:1082B0003220EF0043162400008041001040BA0035
:1082C0000160EF00000006002020000020200000D8
:1082D000253200005820000020200000202000004F
:1082E0002532000058000000CF0278003220EF0055
:1082F00023182400008041001040BA000160EF0004
:10830000000006000A0D0000436100006D2000001F
:108310004D6F0000646500006C0A00000D00000055
:10832000CF0278003220EF00E319240000804100E2
:108330001040BA000160EF00000006002025000098
:1083400064200000204E00006F2000004361000008
:108350006D650000726100000A0D00000000000061
:10836000CF0278003220EF00E31B240000804100A0
:108370001040BA000160EF00000006004545000013
:10838000507200006F6D000020440000756D000009
:10839000703A00000A0D000000000000CF027800D3
:1083A0003220EF00C31D2400008041001040BA00BD
:1083B0000160EF000000060045450000507200001B
:1083C0006F6D0000204300006F6E000066690000C2
:1083D00067200000447500006D7000003A0A00003C
:1083E0000D000000CF0278003220EF0003202400AF
:1083F000008041001040BA000160EF00000006005C
:1084000045450000507200006F6D000020500000D4
:108410007265000073650000742000004475000060
:108420006D7000003A0A00000D000000CF027800D5
:108430003220EF0043222400008041001040BA00A7
:108440000160EF000000060045450000507200008A
:108450006F6D000020480000696700006820000080
:10846000447500006D7000003A0A00000D00000025
:10847000CF0278003220EF00632424000080410006
:108480001040BA000160EF00000006004545000002
:10849000507200006F6D0000205000004343000048
:1084A0002050000072650000736500007420000019
:1084B000447500006D7000003A0A00000D000000D5
:1084C000CF0278003220EF00E32624000080410034
:1084D0001040BA000160EF000000060020200000FC
:1084E000202000002020000000000000CF027800C3
:1084F0003220EF00E301200083015000050031002D
:1085000043292400008041001040BA000160EF00C0
:108510000000060040292400838141008081410041
:108520001380BA00000006000A0D65000A0D7300F2
:108530005265700061646F0020496E003243730021
:10854000204D650075783D002041250064643200AF
:108550007265580073730A003D250D003258000003
:1085600020520000CF0278003220EF00032C2400BC
:10857000008041001040BA000160EF0000000600DA
:108580004D750000782000005772000069740000EB
:108590006542000079740000653D0000257500000B
:1085A0000A0D000000000000CF0278003220EF002A
:1085B000C30120008301500005003100232F240057
:1085C000008041001040BA000160EF00000006008A
:1085D000202F240083814100808141001380BA0054
:1085E000000006000A0D58000A0D2C0057724400C6
:1085F00069746100652074004932610063203D00A8
:108600004D752500782032004164580064722000C6
:1086100065730A00733D0D0025320000CF0278001B
:108620003220EF00C3312400008041001040BA0026
:108630000160EF00000006000A0D00000A0D0000B6
:10864000204900006E760000616C00006964000043
:108650002052000065670000697300007465000027
:108660007220000028250000732900000A0D000078
:1086700000000000CF0278003220EF008334240095
:10868000008041001040BA000160EF0000000600C9
:108690000A0D00000A0D0000204900006E7600005F
:1086A000616C000069640000204900003263000032
:1086B00020410000646400007265000073730000D4
:1086C0002028000025730000290A00000D0000008A
:1086D000CF0278003220EF00633724000080410091
:1086E0001040BA000160EF00000006000A0D000013
:1086F0000A0D0000204900006E760000616C000049
:10870000696400002049000032630000205200002C
:108710006567000069730000746500007220000046
:1087200028250000732900000A0D00000000000049
:10873000CF0278003220EF00430220008301500076
:1087400005003100633B2400008041001040BA0066
:108750000160EF0000000600603B240083814100BF
:10876000808141001380BA00000006000A0D580005
:108770000A0D2000526552006164650020497300B3
:108780003243700020416F0064646E0072657300B4
:10879000737365003D253D0032582500205232009C
:1087A0006567580069730A0074650D00723D00002A
:1087B00025320000CF0278003220EF0003022000B3
:1087C0008301500005003100833F240000804100F8
:1087D0001040BA000160EF0000000600803F240056
:1087E00083814100808141001380BA0000000600AF
:1087F0000A0D32000A0D580057722C0069744400AB
:1088000065206100416474006472610065733D001D
:10881000733D250025323200582C58005265200047
:1088200067690A0073740D00657200003D25000041
:10883000CF0278003220EF00430220008301500075
:108840000500310063432400008041001040BA005D
:108850000160EF00000006006043240083814100B6
:10886000808141001380BA00000006000A0D52000A
:108870000A0D6500204967006E766900616C73001F
:108880006964740020496500326372002041200051
:10889000646428007265250073737300282529001D
:1088A00073290A0020610D006E6400002F6F000024
:1088B00072200000CF0278003220EF0083462400AF
:1088C000008041001040BA000160EF000000060087
:1088D0000A0D00000A0D0000204E00006F2000006D
:1088E00064610000746100000A0D000000000000D7
:1088F000CF0278003220EF0063482400008041005E
:108900001040BA000160EF00000006000A0D0000F0
:1089100053500000492D0000577200006974000098
:108920006520000025320000782500003278000024
:108930000A0D000000000000CF0278003220EF0096
:10894000A34A2400008041001040BA000160EF00FB
:10895000000006000A0D00003E2000005049000003
:10896000503D00004F660000660A00000D3E00000A
:1089700020000000CF0278003220EF00834C24005A
:10898000008041001040BA000160EF0000000600C6
:108990000A0D00003E20000050490000503D00003C
:1089A0004F6E00000A0D00003E2000000000000095
:1089B000CF0278003220EF00634E24000080410097
:1089C0001040BA000160EF00000006000A0D000030
:1089D0003E20000044690000616700003D4F000038
:1089E0006E0A00000D3E000020000000CF0278005B
:1089F0003220EF0043502400008041001040BA00B4
:108A00000160EF00000006000A0D00003E2000009B
:108A100044690000616700003D4F00006666000089
:108A20000A0D00003E20000000000000CF02780088
:108A30003220EF0043522400008041001040BA0071
:108A40000160EF00000006000A0D00003E2000005B
:108A500050490000502000004C6F0000636100008E
:108A6000746900006F6E00003D3000003A4E000057
:108A70006F6E0000650A00000D3E0000200000003F
:108A8000CF0278003220EF00E35424000080410040
:108A90001040BA000160EF00000006000A0D00005F
:108AA0003E20000050490000502000004C6F0000A4
:108AB00063610000746900006F6E00003D310000CA
:108AC0003A550000520A00000D3E00002000000050
:108AD000CF0278003220EF0063572400008041006D
:108AE0001040BA000160EF00000006000A0D00000F
:108AF0003E20000050490000502000004C6F000054
:108B000063610000746900006F6E00003D32000078
:108B10003A4C0000520A00000D3E00002000000008
:108B2000CF0278003220EF00E3592400008041009A
:108B30001040BA000160EF00000006000A0D0000BE
:108B40003E20000050490000502000004C6F000003
:108B500063610000746900006F6E00003D33000027
:108B60003A4C00004D0A00000D3E000020000000BD
:108B7000CF0278003220EF00635C240000804100C7
:108B80001040BA000160EF00000006000A0D00006E
:108B90003E20000050490000502000004C6F0000B3
:108BA00063610000746900006F6E00003D340000D6
:108BB0003A4C00004C0A00000D3E0000200000006E
:108BC000CF0278003220EF00E35E240000804100F5
:108BD0001040BA000160EF00000006000A0D00001E
:108BE0003E20000050490000502000004C6F000063
:108BF00063610000746900006F6E00003D35000085
:108C00003A5500004C0A00000D3E00002000000014
:108C1000CF0278003220EF00636124000080410021
:108C20001040BA000160EF00000006000A0D0000CD
:108C30003E200000506F000077650000723D00008C
:108C40004F6E00000A0D00003E20000000000000F2
:108C5000CF0278003220EF006363240000804100DF
:108C60001040BA000160EF00000006000A0D00008D
:108C70003E200000506F000077650000723D00004C
:108C80004F660000660A00000D3E00002000000054
:108C9000CF0278003220EF0063652400008041009D
:108CA0001040BA000160EF00000006000A0D00004D
:108CB0003E2000005344000069610000673D000051
:108CC0004F6E00000A0D00003E2000000000000072
:108CD000CF0278003220EF0063672400008041005B
:108CE0001040BA000160EF00000006000A0D00000D
:108CF0003E2000005344000069610000673D000011
:108D00004F660000660A00000D3E000020000000D3
:108D1000CF0278003220EF00636924000080410018
:108D20001040BA000160EF00000006000A0D0000CC
:108D30003E200000546100006C6C0000793D000092
:108D4000416300007469000076650000204C00005B
:108D50006F7700000A0D00003E20000000000000B8
:108D6000CF0278003220EF00E36B24000080410046
:108D70001040BA000160EF00000006000A0D00007C
:108D80003E200000546100006C6C0000793D000042
:108D9000416300007469000076650000204800000F
:108DA00069670000680A00000D3E00002000000016
:108DB000CF0278003220EF00636E24000080410073
:108DC0001040BA000160EF00000006000A0D00002C
:108DD0003E20000050490000502000005369000070
:108DE0007A6500003D5300006D6100006C6C00006E
:108DF0000A0D00003E20000000000000CF027800B5
:108E00003220EF00C3702400008041001040BA00FF
:108E10000160EF00000006000A0D00003E20000087
:108E20005049000050200000536900007A6500009E
:108E30003D4D000065640000697500006D0A00008A
:108E40000D3E000020000000CF0278003220EF002D
:108E500023732400008041001040BA000160EF003D
:108E6000000006000A0D00003E20000050490000EE
:108E700050200000536900007A6500003D4C00005E
:108E800061720000676500000A0D00003E200000CE
:108E900000000000CF0278003220EF00837524002C
:108EA000008041001040BA000160EF0000000600A1
:108EB0000A0D00003E200000436100006D650000C7
:108EC000726100002025000064200000496E00004F
:108ED000766100006C690000640A00000D3E00002D
:108EE00020000000CF0278003220EF000378240039
:108EF000008041001040BA000160EF000000060051
:108F0000203000003A570000697000006520000022
:108F1000523E00004C000000CF0278003220EF00EB
:108F2000A3792400008041001040BA000160EF00E6
:108F300000000600203100003A5700006970000070
:108F4000652000004C3E000052000000CF02780077
:108F50003220EF00437B2400008041001040BA0023
:108F60000160EF0000000600203200003A570000C8
:108F70006970000065200000546F0000703E000022
:108F8000426F000074000000CF0278003220EF0032
:108F9000237D2400008041001040BA000160EF00F2
:108FA00000000600203300003A57000069700000FE
:108FB00065200000426F0000743E0000546F000006
:108FC00070000000CF0278003220EF00037F240001
:108FD000008041001040BA000160EF000000060070
:108FE000203400003A4300006F7200006E650000FC
:108FF000722000004C5200003E5500004C00000062
:10900000CF0278003220EF00E3802400008041008E
:109010001040BA000160EF0000000600203500009B
:109020003A4300006F7200006E650000722000007D
:109030004C4C00003E55000052000000CF0278006A
:109040003220EF00C3822400008041001040BA00AB
:109050000160EF0000000600203600003A430000E7
:109060006F7200006E650000722000005552000013
:109070003E4C00004C000000CF0278003220EF0090
:10908000A3842400008041001040BA000160EF007A
:1090900000000600203700003A4300006F72000015
:1090A0006E65000072200000554C00003E4C000030
:1090B00052000000CF0278003220EF0083862400A7
:1090C000008041001040BA000160EF00000006007F
:1090D000203800003A570000697000006520000049
:1090E0004F750000743E0000436500006E74000080
:1090F0006572000000000000CF0278003220EF000F
:10910000A3882400008041001040BA000160EF00F5
:1091100000000600203900003A5700006970000086
:10912000652000004C3E0000436500006E740000A6
:10913000657200003C52000000000000CF02780081
:109140003220EF00C38A2400008041001040BA00A2
:109150000160EF000000060020310000303A0000FE
:109160005769000070650000205400003E43000075
:10917000656E000074650000723C00004200000053
:10918000CF0278003220EF00E38C24000080410001
:109190001040BA000160EF0000000600202000002F
:1091A0003A4E00006F6E000065200000536500001D
:1091B0006C6500006374000065640000000000003E
:1091C000CF0278003220EF00E38E240000804100BF
:1091D0001040BA000160EF00000006000A0D000018
:1091E0003E200000576900007065000053650000D4
:1091F0006C3D0000257300000A0D00003E200000B9
:1092000000000000CF0278003220EF00039124001C
:10921000008041001040BA000160EF00000006002D
:109220000A0D00003E200000496400006C6500004B
:10923000527400006E3D00002564000020530000C1
:10924000656300006F6E0000647300000A0D00008B
:109250003E20000000000000CF0278003220EF0026
:10926000A3932400008041001040BA000160EF0089
:10927000000006000A0D00003E20000050490000DA
:109280005020000043680000616E00006765000028
:109290003D420000616300006B670000726F0000D8
:1092A000756E0000640A00000D3E00002000000002
:1092B000CF0278003220EF00639624000080410046
:1092C0001040BA000160EF00000006000A0D000027
:1092D0003E2000005049000050200000436800007C
:1092E000616E0000676500003D4600006F7200007F
:1092F00065670000726F0000756E0000640A000070
:109300000D3E000020000000CF0278003220EF0068
:1093100023992400008041001040BA000160EF0052
:10932000000006000A0D00003E2000005061000011
:109330006E53000070650000656400003D2500006C
:10934000640A00000D3E000020000000CF027800FB
:109350003220EF00439B2400008041001040BA00FF
:109360000160EF00000006000A0D00003E20000032
:10937000546900006C7400005370000065650000C3
:10938000643D0000256400000A0D00003E2000003E
:1093900000000000CF0278003220EF00839D2400FF
:1093A000008041001040BA000160EF00000006009C
:1093B0000A0D00003E2000005A6F00006F6D000093
:1093C0005370000065650000643D000025640000E6
:1093D0000A0D00003E20000000000000CF027800CF
:1093E0003220EF00C39F2400008041001040BA00EB
:1093F0000160EF0000000600202000002020000097
:10940000496E000069740000204D0000757800006E
:109410002020000020000000CF0278003220EF0062
:10942000A3A12400008041001040BA000160EF00B9
:10943000000006002020000020200000496E0000EF
:10944000697400002056000069640000656F000028
:10945000202000002020000000000000CF02780043
:109460003220EF00C3A32400008041001040BA0066
:109470000160EF000000060020200000496E00009F
:1094800069740000205300007562000053790000E9
:1094900073740000656D00002020000000000000D3
:1094A000CF0278003220EF00E3A5240000804100C5
:1094B0001040BA000160EF00000006000A0D000035
:1094C0003E530000657400004465000066610000C2
:1094D000756C00007420000025640000200A000064
:1094E0000D3E000020000000CF0278003220EF0087
:1094F00023A82400008041001040BA000160EF0062
:10950000000006000A0D00003E2000005365000028
:1095100072690000616C000045630000686F000024
:109520003D4500006E610000626C00006564000053
:109530000A0D00003E20000000000000CF0278006D
:109540003220EF00C3AA2400008041001040BA007E
:109550000160EF00000006000A0D00003E20000040
:109560005365000072690000616C000045630000F3
:10957000686F00003D4400006973000061620000F4
:109580006C650000640A00000D3E00002000000031
:10959000CF0278003220EF0063AD2400008041004C
:1095A0001040BA000160EF00000006000A0D000044
:1095B0003E2000005365000072690000616C0000ED
:1095C000496E0000666F00003D4500006E610000BE
:1095D000626C0000656400000A0D00003E2000007F
:1095E00000000000CF0278003220EF0003B024001A
:1095F000008041001040BA000160EF00000006004A
:109600000A0D00003E200000536500007269000052
:10961000616C0000496E0000666F00003D44000070
:1096200069730000616200006C650000640A00005C
:109630000D3E000020000000CF0278003220EF0035
:10964000A3B22400008041001040BA000160EF0086
:1096500000000600536500006172000063680000AE
:10966000696E000067200000666F00007220000035
:1096700041740000746100006368000065640000CC
:1096800020430000616D00006572000061730000FE
:109690000D0A000000000000CF0278003220EF0029
:1096A000A3B52400008041001040BA000160EF0023
:1096B000000006000A0D0000506F000072740000E8
:1096C00020250000643A00000A0D000000000000A0
:1096D000CF0278003220EF0063B724000080410001
:1096E0001040BA000160EF00000006000A0D000003
:1096F000436100006D6500007261000020530000AE
:10970000656100007263000068200000436F000084
:109710006D7000006C650000746500000A0D0000AB
:109720000A000000CF0278003220EF0003BA2400C4
:10973000008041001040BA000160EF000000060008
:1097400020560000432D0000433500003069000022
:1097500020200000205000006F72000074200000E4
:109760003020000020000000CF0278003220EF00FF
:1097700023BC2400008041001040BA000160EF00CB
:1097800000000600436100006E6F00006E200000C4
:1097900044650000746500006374000065640000A7
:1097A0000D0A000000000000CF0278003220EF0018
:1097B00023BE2400008041001040BA000160EF0089
:1097C00000000600204E00006F20000043610000F2
:1097D0006D20000020200000205000006F7200006B
:1097E000742000003020000020000000CF0278002C
:1097F0003220EF0043C02400008041001040BA0036
:109800000160EF00000006000D0A0000506100003A
:109810006E610000736F00006E690000632000003D
:10982000415700002D480000453100003030000055
:109830000D0A000000000000CF0278003220EF0087
:10984000A3C22400008041001040BA000160EF0074
:109850000000060020410000572D00004845000090
:109860003130000030200000205000006F720000F6
:10987000742000003020000020000000CF0278009B
:109880003220EF00C3C42400008041001040BA0021
:109890000160EF0000000600204700006574000032
:1098A0003820000000000000CF0278003220EF00D6
:1098B00023C62400008041001040BA000160EF0080
:1098C0000000060020200000202D00002D200000B8
:1098D00025320000582000002D2D00000A0D000048
:1098E00000000000CF0278003220EF0003C82400FF
:1098F000008041001040BA000160EF000000060047
:109900000A0D0000202000002067000065740000A0
:109910003136000020000000CF0278003220EF0036
:10992000A3C92400008041001040BA000160EF008C
:109930000000060020200000202D00002D20000047
:10994000254C0000582000002D2D0000200A0000AA
:109950000D000000CF0278003220EF0083CB2400FE
:10996000008041001040BA000160EF0000000600D6
:109970000A0D000020200000206700006574000030
:109980003332000020000000CF0278003220EF00C8
:1099900023CD2400008041001040BA000160EF0098
:1099A0000000060020200000202D00002D200000D7
:1099B000254C0000582000002D2D00000A0D00004D
:1099C00000000000CF0278003220EF0003CF240017
:1099D000008041001040BA000160EF000000060066
:1099E0000A0D000020430000616D00006572000058
:1099F0006154000079700000652000000000000044
:109A0000CF0278003220EF00E3D024000080410034
:109A10001040BA000160EF00000006000D0A0000CF
:109A2000536F00006E790000204500005649000089
:109A30002D4400003330000028720000290D000082
:109A40000A000000CF0278003220EF0003D3240088
:109A5000008041001040BA000160EF0000000600E5
:109A600020450000564900002D440000333000001E
:109A700028720000295000006F720000742000005E
:109A80003020000020000000CF0278003220EF00DC
:109A900023D52400008041001040BA000160EF008F
:109AA00000000600496E0000766100006C6900004D
:109AB00064200000436100006D65000072610000D9
:109AC0000D0A000000000000CF0278003220EF00F5
:109AD00023D72400008041001040BA000160EF004D
:109AE00000000600204900006E760000616C000056
:109AF0006964000020430000616D00006572000091
:109B000061000000CF0278003220EF0003D924006A
:109B1000008041001040BA000160EF000000060024
:109B20000D0A0000536F00006E7900002045000010
:109B3000564900002D440000333000002F33000050
:109B4000312000000D0A000000000000CF02780064
:109B50003220EF0043DB2400008041001040BA00B7
:109B60000160EF000000060020450000564900009B
:109B70002D440000333000002F330000315000002E
:109B80006F720000742000003020000020000000F0
:109B9000CF0278003220EF0063DD24000080410016
:109BA0001040BA000160EF00000006000D0A00003E
:109BB000536F00006E7900002045000056490000F8
:109BC0002D440000333000000D0A000000000000AA
:109BD000CF0278003220EF0063DF240000804100D4
:109BE0001040BA000160EF000000060020450000B0
:109BF000564900002D4400003330000020200000B2
:109C0000205000006F72000074200000302000001F
:109C100020000000CF0278003220EF0083E1240012
:109C2000008041001040BA000160EF000000060013
:109C30000D0A00005661000064640000696F0000B6
:109C400020410000646400002D4100002D4300000D
:109C5000616D00000D0A000000000000CF027800D6
:109C60003220EF00C3E32400008041001040BA001E
:109C70000160EF0000000600204100006464000065
:109C80002D4100002D430000616D000020500000B8
:109C90006F720000742000003020000020000000DF
:109CA000CF0278003220EF00E3E52400008041007D
:109CB0001040BA000160EF00000006000D0A00002D
:109CC000536F00006E7900002045000056490000E7
:109CD0002D44000031300000300D00000A0000006B
:109CE000CF0278003220EF00E3E72400008041003B
:109CF0001040BA000160EF0000000600204500009F
:109D0000564900002D440000313000003020000092
:109D1000205000006F72000074200000302000000E
:109D200020000000CF0278003220EF0003EA240078
:109D3000008041001040BA000160EF000000060002
:109D40000D0A0000536F00006E79000020450000EE
:109D5000564900002D440000373000000D0A000075
:109D600000000000CF0278003220EF0003EC240056
:109D7000008041001040BA000160EF0000000600C2
:109D800020450000564900002D44000037300000F7
:109D900020200000205000006F720000742000009E
:109DA0003020000020000000CF0278003220EF00B9
:109DB00023EE2400008041001040BA000160EF0053
:109DC000000006000D0A0000536F00006E790000CD
:109DD0002042000052430000482D000037300000B0
:109DE000300D00000A000000CF0278003220EF00A2
:109DF00023F02400008041001040BA000160EF0011
:109E0000000006002042000052430000482D0000E0
:109E10003730000030200000205000006F7200003A
:109E2000742000003020000020000000CF027800E5
:109E30003220EF0043F22400008041001040BA00BD
:109E40000160EF00000006000D0A0000456C0000F4
:109E50006D6F000020430000616D0000657200001E
:109E6000610D00000A000000CF0278003220EF00F0
:109E700023F42400008041001040BA000160EF008C
:109E800000000600204500006C6D00006F200000FF
:109E90002020000020200000205000006F720000F1
:109EA000742000003020000020000000CF02780065
:109EB0003220EF0043F62400008041001040BA0039
:109EC0000160EF00000006000D0A0000536F000063
:109ED0006E79000020420000524300002D33000044
:109EE000303000000D0A000000000000CF027800B2
:109EF0003220EF0043F82400008041001040BA00F7
:109F00000160EF0000000600204200005243000004
:109F10002D330000303000002020000020500000D1
:109F20006F7200007420000030200000200000004C
:109F3000CF0278003220EF0063FA24000080410055
:109F40001040BA000160EF00000006000D0A00009A
:109F5000536F00006E790000204200005243000061
:109F60002D5A000037300000300D00000A000000BC
:109F7000CF0278003220EF0063FC24000080410013
:109F80001040BA000160EF0000000600204200000F
:109F9000524300002D5A00003730000030200000EE
:109FA000205000006F72000074200000302000007C
:109FB00020000000CF0278003220EF0083FE240052
:109FC000008041001040BA000160EF000000060070
:109FD0000D0A0000536F00006E790000204200005F
:109FE000524300002D5A000033330000300D0000B2
:109FF0000A000000CF0278003220EF008300250025
:10A00000008041001040BA000160EF00000006002F
:10A0100020420000524300002D5A0000333300005C
:10A0200030200000205000006F72000074200000FB
:10A030003020000020000000CF0278003220EF0026
:10A04000A3022500008041001040BA000160EF002B
:10A05000000006000D0A0000566100006464000064
:10A06000696F000020480000442D000031380000D6
:10A070000D0A000000000000CF0278003220EF003F
:10A08000A3042500008041001040BA000160EF00E9
:10A090000000060020200000484400002D31000090
:10A0A0003820000020200000205000006F720000C7
:10A0B000742000003020000020000000CF02780053
:10A0C0003220EF00C3062500008041001040BA0096
:10A0D0000160EF00000006000D0A0000536F000051
:10A0E0006E79000020450000564900002D48000010
:10A0F000443100000D0A000000000000CF0278008B
:10A100003220EF00C3082500008041001040BA0053
:10A110000160EF00000006002045000056490000E5
:10A120002D48000044310000202000002050000095
:10A130006F7200007420000030200000200000003A
:10A14000CF0278003220EF00E30A250000804100B2
:10A150001040BA000160EF00000006000D0A000088
:10A160005661000064640000696F00002043000035
:10A17000656900006C6900006E67000056490000C8
:10A18000455700000D0A000000000000CF027800D3
:10A190003220EF00430D2500008041001040BA003E
:10A1A0000160EF000000060020430000562F000071
:10A1B000435600004D5000002020000020500000B9
:10A1C0006F720000742000003020000020000000AA
:10A1D000CF0278003220EF00630F2500008041009D
:10A1E0001040BA000160EF0000000600556E00004C
:10A1F0006B6E00006F7700006E200000436100006E
:10A200006D650000726100000D0A00000000000092
:10A21000CF0278003220EF0063112500008041005A
:10A220001040BA000160EF00000006002055000059
:10A230006E6B00006E6F0000776E00002020000043
:10A24000205000006F7200007420000030200000D9
:10A2500020000000CF0278003220EF008313250099
:10A26000008041001040BA000160EF0000000600CD
:10A270000A0D000020410000542F00004D44000052
:10A280005F4D00006F640000654900006E710000C2
:10A2900020000000CF0278003220EF008315250057
:10A2A000008041001040BA000160EF00000006008D
:10A2B0000D0A00002057000061690000745300007F
:10A2C0006F6E000079410000636B00000000000029
:10A2D000CF0278003220EF00631725000080410094
:10A2E0001040BA000160EF00000006000D0A0000F7
:10A2F0002057000061690000745300006F6E000079
:10A3000079000000CF0278003220EF000319250009
:10A31000008041001040BA000160EF00000006001C
:10A320002A57000061690000745300006F6E00003E
:10A3300079000000CF0278003220EF00831A250058
:10A34000008041001040BA000160EF0000000600EC
:10A350000A0D00005761000069740000526500009A
:10A3600073700000536F00006E7900003A20000007
:10A3700000000000CF0278003220EF00831C25008F
:10A38000008041001040BA000160EF0000000600AC
:10A39000202D000020540000696D0000656F000052
:10A3A000757400002025000075200000286D000055
:10A3B000732900000D0A000000000000CF027800A1
:10A3C0003220EF00C31E2500008041001040BA007B
:10A3D0000160EF0000000600436100006E630000B2
:10A3E000656C0000205300003120000000000000D8
:10A3F000CF0278003220EF0063202500008041006A
:10A400001040BA000160EF00000006004361000048
:10A410006E630000656C00002053000032200000D5
:10A4200000000000CF0278003220EF000322250058
:10A43000008041001040BA000160EF0000000600FB
:10A440000A0D000020200000204700006574000075
:10A450004252000043500000616E00005469000049
:10A460006C740000506F00007320000000000000BA
:10A47000CF0278003220EF006324250000804100E5
:10A480001040BA000160EF0000000600202000002C
:10A49000202D00002D200000503A0000254C000027
:10A4A000582C0000543A0000254C000058200000B1
:10A4B0002D2D00000A0D000000000000CF027800E2
:10A4C0003220EF00C3262500008041001040BA0072
:10A4D0000160EF0000000600205D00000A0D000092
:10A4E00000000000CF0278003220EF000328250092
:10A4F000008041001040BA000160EF00000006003B
:10A500000D0A00002057000061690000744300003C
:10A51000616E00006F6E000000000000CF02780046
:10A520003220EF00C3292500008041001040BA000E
:10A530000160EF0000000600202D00002054000004
:10A54000696D0000656F0000757400002025000033
:10A550006C750000202800006D730000290D0000BC
:10A560000A000000CF0278003220EF00032C250003
:10A57000008041001040BA000160EF0000000600BA
:10A580000D0A0000205700006169000074500000AF
:10A59000616E0000617300006F6E0000696300006F
:10A5A00000000000CF0278003220EF00032E2500CB
:10A5B000008041001040BA000160EF00000006007A
:10A5C0002020000020530000595300005445000093
:10A5D0004D2000004D4500004E5500002020000099
:10A5E0002020000000000000CF0278003220EF00A1
:10A5F00023302500008041001040BA000160EF00C8
:10A6000000000600202000002053000065720000BA
:10A61000696100006C200000496E00007075000048
:10A62000742000002020000000000000CF0278000D
:10A630003220EF0043322500008041001040BA0074
:10A640000160EF0000000600202000002053000001
:10A6500065720000696100006C2000004563000025
:10A66000686F000020200000202000000000000093
:10A67000CF0278003220EF006334250000804100D3
:10A680001040BA000160EF0000000600202000002A
:10A690002053000065720000696100006C2000001A
:10A6A000496E0000666F000020200000202000009E
:10A6B00000000000CF0278003220EF008336250032
:10A6C000008041001040BA000160EF000000060069
:10A6D0002020000020500000616E0000656C00002A
:10A6E000204C0000696700006874000073200000BF
:10A6F0002020000000000000CF0278003220EF0090
:10A70000A3382500008041001040BA000160EF002E
:10A710000000060020200000204300006C650000BF
:10A7200061720000204D0000656D00006F72000036
:10A73000792000002020000000000000CF027800F7
:10A740003220EF00C33A2500008041001040BA00DB
:10A750000160EF0000000600202000002043000000
:10A760006C650000617200002050000072650000FE
:10A7700073650000747300002020000000000000DA
:10A78000CF0278003220EF00E33C2500008041003A
:10A790001040BA000160EF00000006002020000019
:10A7A00054720000616E000073690000746900005B
:10A7B0006F6E000020540000696D000065200000ED
:10A7C00000000000CF0278003220EF00033F250098
:10A7D000008041001040BA000160EF000000060058
:10A7E0002020000054720000616E000073690000B8
:10A7F000746900006F6E0000204D00006F6400005F
:10A800006520000000000000CF0278003220EF0039
:10A8100023412500008041001040BA000160EF0094
:10A82000000006002020000057690000706500004D
:10A8300020530000656C000065630000746900002F
:10A840006F6E00002020000000000000CF027800A2
:10A850003220EF0043432500008041001040BA0041
:10A860000160EF00000006002020000020530000DF
:10A8700065740000746C00006520000054690000DD
:10A880006D65000020200000202000000000000076
:10A89000CF0278003220EF006345250000804100A0
:10A8A0001040BA000160EF00000006002020000008
:10A8B0002020000020200000546100006C6C00008B
:10A8C000792000002020000020200000202000002F
:10A8D00000000000CF0278003220EF0083472500FF
:10A8E000008041001040BA000160EF000000060047
:10A8F00020200000496E0000697400002054000010
:10A900007269000067670000657200007320000034
:10A910002020000000000000CF0278003220EF006D
:10A92000A3492500008041001040BA000160EF00FB
:10A93000000006002020000020500000726500008A
:10A940007365000074200000363700002D370000CA
:10A95000322000002020000000000000CF0278001C
:10A960003220EF00C34B2500008041001040BA00A8
:10A970000160EF000000060020560000494400007E
:10A98000454F0000204900004E5000005554000083
:10A99000204D0000454E0000552000000000000042
:10A9A000CF0278003220EF00E34D25000080410007
:10A9B0001040BA000160EF000000060020200000F7
:10A9C000434100004D20000053450000415200006B
:10A9D00043480000204D0000454E00005520000077
:10A9E00000000000CF0278003220EF000350250065
:10A9F000008041001040BA000160EF000000060036
:10AA00002020000020200000204100006C6C00008D
:10AA1000205000006F7200007473000020200000BE
:10AA20002020000000000000CF0278003220EF005C
:10AA300023522500008041001040BA000160EF0061
:10AA40000000060020200000202000002020000040
:10AA5000506F0000727400002030000031200000B0
:10AA6000202000002020000000000000CF0278001D
:10AA70003220EF0043542500008041001040BA000E
:10AA80000160EF00000006002020000020200000F0
:10AA900020200000506F0000727400002030000081
:10AAA00032200000202000002020000000000000D4
:10AAB000CF0278003220EF0063562500008041006D
:10AAC0001040BA000160EF000000060020200000E6
:10AAD0002020000020200000506F00007274000051
:10AAE0002030000033200000202000002020000043
:10AAF00000000000CF0278003220EF0083582500CC
:10AB0000008041001040BA000160EF000000060024
:10AB1000202000002020000020200000506F0000B6
:10AB2000727400002030000034200000202000005B
:10AB30002020000000000000CF0278003220EF004B
:10AB4000A35A2500008041001040BA000160EF00C8
:10AB5000000006002020000020200000202000002F
:10AB6000506F00007274000020300000352000009B
:10AB7000202000002020000000000000CF0278000C
:10AB80003220EF00C35C2500008041001040BA0075
:10AB90000160EF00000006002020000020200000DF
:10ABA00020200000506F0000727400002030000070
:10ABB00036200000202000002020000000000000BF
:10ABC000CF0278003220EF00E35E250000804100D4
:10ABD0001040BA000160EF000000060020200000D5
:10ABE00020200000204D0000414900004E200000C0
:10ABF0004D4500004E5500002020000020200000A0
:10AC000000000000CF0278003220EF000361250031
:10AC1000008041001040BA000160EF000000060013
:10AC2000202000005265000073630000616E000088
:10AC300020430000616D0000657200006173000038
:10AC40002020000000000000CF0278003220EF003A
:10AC500023632500008041001040BA000160EF002E
:10AC60000000060020200000205200006573000054
:10AC7000636100006E2000005669000064650000FA
:10AC80006F2000002020000000000000CF027800AC
:10AC90003220EF0043652500008041001040BA00DB
:10ACA0000160EF0000000600202000002056000098
:10ACB00069640000656F0000204F0000757400009B
:10ACC00070750000742000002020000000000000CB
:10ACD000CF0278003220EF0063672500008041003A
:10ACE0001040BA000160EF0000000600205600008E
:10ACF00069640000656F0000204900006E7000006C
:10AD000075740000204D0000656E00007520000085
:10AD100000000000CF0278003220EF008369250098
:10AD2000008041001040BA000160EF000000060002
:10AD30002044000065660000617500006C7400002E
:10AD40002050000072650000736500007420000050
:10AD50004E6F000000000000CF0278003220EF00AC
:10AD6000A36B2500008041001040BA000160EF0095
:10AD7000000006002020000020440000656600005E
:10AD8000617500006C74000020540000696D0000C3
:10AD9000657200002020000000000000CF02780053
:10ADA0003220EF00C36D2500008041001040BA0042
:10ADB0000160EF00000006002050000072650000F6
:10ADC0007365000074200000506100006E200000D8
:10ADD0005370000065650000642000000000000062
:10ADE000CF0278003220EF00E36F250000804100A1
:10ADF0001040BA000160EF00000006002050000083
:10AE00007265000073650000742000005469000042
:10AE10006C74000020530000706500006564000041
:10AE200000000000CF0278003220EF0003722500FE
:10AE3000008041001040BA000160EF0000000600F1
:10AE4000205000007265000073650000742000004F
:10AE50005A6F00006F6D0000205300007065000005
:10AE60006564000000000000CF0278003220EF008F
:10AE700023742500008041001040BA000160EF00FB
:10AE80000000060020200000436100006D2000004B
:10AE9000536500006172000063680000204D0000EF
:10AEA000656E00007520000000000000CF027800F1
:10AEB0003220EF0043762500008041001040BA00A8
:10AEC0000160EF00000006002020000020200000AC
:10AED0005379000073740000656D0000204D000080
:10AEE000656E0000752000002020000000000000BA
:10AEF000CF0278003220EF00637825000080410007
:10AF00001040BA000160EF000000060020200000A1
:10AF10002020000020200000537400006172000017
:10AF200074200000202000002020000020200000CD
:10AF300000000000CF0278003220EF00837A250065
:10AF4000008041001040BA000160EF0000000600E0
:10AF5000204800004420000031300000383000005C
:10AF600070200000353900002E3900003448000000
:10AF70007A20000000000000CF0278003220EF00AD
:10AF8000A37C2500008041001040BA000160EF0062
:10AF9000000006002048000044200000313000007E
:10AFA000383000007020000035300000487A000082
:10AFB000202000002020000000000000CF027800C8
:10AFC0003220EF00C37E2500008041001040BA000F
:10AFD0000160EF000000060020480000442000004F
:10AFE00031300000383000006920000035390000A1
:10AFF0002E390000344800007A20000000000000D4
:10B00000CF0278003220EF00E3802500008041006D
:10B010001040BA000160EF00000006002048000068
:10B02000442000003130000038300000692000006A
:10B0300035300000487A0000202000002020000069
:10B0400000000000CF0278003220EF0003832500CB
:10B05000008041001040BA000160EF0000000600CF
:10B06000204800004420000020370000323000005B
:10B0700070200000353900002E39000034480000EF
:10B080007A20000000000000CF0278003220EF009C
:10B0900023852500008041001040BA000160EF00C8
:10B0A0000000060020480000442000002037000077
:10B0B000323000007020000035300000487A000077
:10B0C000202000002020000000000000CF027800B7
:10B0D0003220EF0043872500008041001040BA0075
:10B0E0000160EF000000060020480000562000002C
:10B0F0002036000034300000782000003438000092
:10B100003020000036300000487A000000000000C7
:10B11000CF0278003220EF006389250000804100D3
:10B120001040BA000160EF00000006002048000057
:10B130005620000020380000303000007820000049
:10B14000363000003020000036300000487A000021
:10B1500000000000CF0278003220EF00838B250032
:10B16000008041001040BA000160EF0000000600BE
:10B17000204800005620000031300000323400002A
:10B1800078200000373600003820000036300000FC
:10B19000487A000000000000CF0278003220EF0063
:10B1A000A38D2500008041001040BA000160EF002F
:10B1B0000000060020480000562000003132000048
:10B1C00038300000782000003736000038200000BA
:10B1D00036300000487A000000000000CF027800FE
:10B1E0003220EF00C38F2500008041001040BA00DC
:10B1F0000160EF000000060020480000562000001B
:10B200003132000038300000783100003032000068
:10B210003420000036300000487A000000000000B2
:10B22000CF0278003220EF00E3912500008041003A
:10B230001040BA000160EF00000006002048000046
:10B240005620000031390000323000007831000013
:10B25000323000003020000036300000487A000014
:10B2600000000000CF0278003220EF000394250098
:10B27000008041001040BA000160EF0000000600AD
:10B2800020530000442000004E54000053430000AF
:10B2900020320000392E000039370000487A0000C3
:10B2A0002020000000000000CF0278003220EF00D4
:10B2B00023962500008041001040BA000160EF0095
:10B2C0000000060020530000442000005041000010
:10B2D0004C2000002020000032350000487A000099
:10B2E000202000002020000000000000CF02780095
:10B2F0003220EF0043982500008041001040BA0042
:10B300000160EF0000000600205300004420000010
:10B31000343800003069000020200000795000001F
:10B320006250000072200000202000000000000099
:10B33000CF0278003220EF00639A250000804100A0
:10B340001040BA000160EF0000000600205300002A
:10B35000442000003537000036690000202000003E
:10B360007950000062500000722000002020000090
:10B3700000000000CF0278003220EF00839C2500FF
:10B38000008041001040BA000160EF00000006009C
:10B3900020200000202000002020000020200000AD
:10B3A0004F4E000020200000202000002020000040
:10B3B0002020000000000000CF0278003220EF00C3
:10B3C000A39E2500008041001040BA000160EF00FC
:10B3D00000000600202000002020000020200000A7
:10B3E000204F0000464600002020000020200000E2
:10B3F000202000002020000000000000CF02780084
:10B400003220EF00C3A02500008041001040BA00A8
:10B410000160EF0000000600202000002020000056
:10B4200020200000204700006C6F000062610000D7
:10B430006C20000020200000202000000000000000
:10B44000CF0278003220EF00E3A225000080410007
:10B450001040BA000160EF0000000600202000004C
:10B460002020000020200000427900002050000031
:10B470007265000073650000742000002020000049
:10B4800000000000CF0278003220EF0003A5250065
:10B49000008041001040BA000160EF00000006008B
:10B4A000202000002052000069670000687400003E
:10B4B000207400006F2000004C65000066740000DE
:10B4C0002020000000000000CF0278003220EF00B2
:10B4D00023A72500008041001040BA000160EF0062
:10B4E0000000060020200000204C000065660000DF
:10B4F00074200000746F0000205200006967000093
:10B50000687400002020000000000000CF027800D6
:10B510003220EF0043A92500008041001040BA000E
:10B520000160EF0000000600202000002054000011
:10B530006F700000207400006F200000426F000058
:10B54000747400006F6D00002020000000000000F7
:10B55000CF0278003220EF0063AB2500008041006D
:10B560001040BA000160EF0000000600202000003B
:10B57000204200006F740000746F00006D20000016
:10B58000746F0000205400006F7000002020000045
:10B5900000000000CF0278003220EF0083AD2500CC
:10B5A000008041001040BA000160EF00000006007A
:10B5B000204400006E5200006967000068740000BB
:10B5C000207400006F200000557000004C650000E2
:10B5D0006674000000000000CF0278003220EF0007
:10B5E000A3AF2500008041001040BA000160EF00C9
:10B5F00000000600204400006E4C0000656600005C
:10B6000074200000746F000020550000705200008C
:10B61000696700006874000000000000CF02780035
:10B620003220EF00C3B12500008041001040BA0075
:10B630000160EF000000060020550000705200007D
:10B640006967000068740000207400006F2000002B
:10B65000446E00004C6500006674000000000000AD
:10B66000CF0278003220EF00E3B3250000804100D4
:10B670001040BA000160EF000000060020550000F5
:10B68000704C00006566000074200000746F0000BC
:10B69000204400006E5200006967000068740000DA
:10B6A00000000000CF0278003220EF0003B6250032
:10B6B000008041001040BA000160EF000000060069
:10B6C000204100006C6C00005369000064650000BC
:10B6D00073200000746F000020430000656E0000BE
:10B6E0007420000000000000CF0278003220EF003C
:10B6F00023B82500008041001040BA000160EF002F
:10B7000000000600204C000065660000743E00004A
:10B71000436500006E740000657200003C5200003A
:10B72000696700006874000000000000CF02780024
:10B730003220EF0043BA2500008041001040BA00DB
:10B740000160EF0000000600205400006F70000050
:10B750003E430000656E000074650000723C00000E
:10B76000426F0000747400006F6D00000000000064
:10B77000CF0278003220EF0063BC2500008041003A
:10B780001040BA000160EF00000006002020000019
:10B79000202000004163000074690000766500000D
:10B7A000204C00006F7700002020000020200000C7
:10B7B00000000000CF0278003220EF0083BE250099
:10B7C000008041001040BA000160EF000000060058
:10B7D0002020000020200000416300007469000068
:10B7E00076650000204800006967000068200000BE
:10B7F0002020000000000000CF0278003220EF007F
:10B80000A3C02500008041001040BA000160EF0095
:10B810000000060020430000616D00002050000081
:10B82000726500007365000074730000204F000013
:10B830004E2000002020000000000000CF02780011
:10B840003220EF00C3C22500008041001040BA0042
:10B850000160EF000000060020430000616D000061
:10B8600020500000726500007365000074730000D2
:10B87000204F00004646000020200000000000008D
:10B88000CF0278003220EF00E3C4250000804100A1
:10B890001040BA000160EF00000006002020000008
:10B8A000204E00006F7400002053000075700000EF
:10B8B000706F0000727400006564000020200000BA
:10B8C00000000000CF0278003220EF0003C72500FF
:10B8D000008041001040BA000160EF000000060047
:10B8E00020530000442000004E5400005343000049
:10B8F0002D280000532D00005669000064650000EB
:10B900006F29000000000000CF0278003220EF0015
:10B9100023C92500008041001040BA000160EF00FB
:10B9200000000600205300004420000020500000CA
:10B93000414C00002D280000532D000056690000E6
:10B94000646500006F29000000000000CF0278004D
:10B950003220EF0043CB2500008041001040BA00A8
:10B960000160EF00000006002053000044200000AA
:10B970004E54000053430000204300006F6D000050
:10B98000706F000073690000746500000000000023
:10B99000CF0278003220EF0063CD25000080410007
:10B9A0001040BA000160EF000000060020530000C4
:10B9B0004420000020500000414C000020430000C3
:10B9C0006F6D0000706F0000736900007465000007
:10B9D00000000000CF0278003220EF0083CF250066
:10B9E000008041001040BA000160EF000000060036
:10B9F00020410000757400006F20000053650000B6
:10BA00006172000063680000204D00006F64000058
:10BA10006520000000000000CF0278003220EF0017
:10BA2000A3D12500008041001040BA000160EF0062
:10BA3000000006002020000020200000205300000D
:10BA40006F6E0000792000004F6E00006C790000DE
:10BA5000202000002020000000000000CF0278001D
:10BA60003220EF00C3D32500008041001040BA000F
:10BA70000160EF00000006002020000020200000F0
:10BA8000436100006E6F00006E2000004F6E0000EA
:10BA90006C79000020200000202000000000000041
:10BAA000CF0278003220EF00E3D52500008041006E
:10BAB0001040BA000160EF000000060020200000E6
:10BAC000506100006E610000736F00006E6900003D
:10BAD000632000004F6E00006C7900002020000001
:10BAE00000000000CF0278003220EF0003D82500CC
:10BAF000008041001040BA000160EF000000060025
:10BB0000202000004E6F000020430000616D000007
:10BB10006572000061200000496E00007075000031
:10BB20007420000000000000CF0278003220EF00F7
:10BB300023DA2500008041001040BA000160EF00C8
:10BB400000000600205300007973000074650000B7
:10BB50006D200000496E0000205300007461000059
:10BB60006E6400006279000000000000CF027800DF
:10BB70003220EF0043DC2500008041001040BA0075
:10BB80000160EF00000006002020000020200000DF
:10BB900020200000203000002563000020730000FA
:10BBA000656300002020000020200000000000004D
:10BBB000CF0278003220EF0063DE250000804100D4
:10BBC0001040BA000160EF000000060020200000D5
:10BBD00020200000202E00003025000063300000EF
:10BBE000207300006563000020200000202000007A
:10BBF00000000000CF0278003220EF0083E0250033
:10BC0000008041001040BA000160EF000000060013
:10BC10002020000020200000203000002E25000001
:10BC200063300000207300006563000020200000E6
:10BC30002020000000000000CF0278003220EF003A
:10BC4000A3E22500008041001040BA000160EF002F
:10BC5000000006002020000020200000202000001E
:10BC6000202000002025000063200000202000008C
:10BC7000202000002020000000000000CF027800FB
:10BC80003220EF00C3E42500008041001040BA00DC
:10BC90000160EF00000006002020000020200000CE
:10BCA0002020000020250000632500006320000004
:10BCB00073650000632000002020000020000000C9
:10BCC000CF0278003220EF00E3E62500008041003B
:10BCD0001040BA000160EF000000060020200000C4
:10BCE00020200000202E00002563000025630000B6
:10BCF0003020000073650000632000002020000059
:10BD000020000000CF0278003220EF0003E9250078
:10BD1000008041001040BA000160EF000000060002
:10BD2000202000002020000020250000632E0000BD
:10BD300025630000302000007365000063200000D0
:10BD40002020000020000000CF0278003220EF0009
:10BD500023EB2500008041001040BA000160EF0095
:10BD6000000006002020000020200000202000000D
:10BD70002025000063250000632000002020000033
:10BD8000202000002020000000000000CF027800EA
:10BD90003220EF0043ED2500008041001040BA0042
:10BDA0000160EF00000006002020000020200000BD
:10BDB00020200000256300002563000025630000AB
:10BDC00020730000656300002020000000000000D8
:10BDD000CF0278003220EF0063EF250000804100A1
:10BDE0001040BA000160EF000000060020200000B3
:10BDF00020200000202E00002563000025630000A5
:10BE0000256300002073000065630000202000000F
:10BE100000000000CF0278003220EF0083F12500FF
:10BE2000008041001040BA000160EF0000000600F1
:10BE30002020000020200000256300002563000072
:10BE40002E250000633000002073000065630000B1
:10BE50002020000000000000CF0278003220EF0018
:10BE6000A3F32500008041001040BA000160EF00FC
:10BE700000000600202000002020000020200000FC
:10BE800020250000632500006325000063200000DA
:10BE9000202000002020000000000000CF027800D9
:10BEA0003220EF00C3F52500008041001040BA00A9
:10BEB0000160EF00000006004F5300004346000001
:10BEC000414900004C5F000045520000524F000005
:10BED000520A00000D000000CF0278003220EF006F
:10BEE000A3F72500008041001040BA000160EF0078
:10BEF000000006004144000044520000455200008A
:10BF0000525F000045520000524F0000520A0000EC
:10BF10000D000000CF0278003220EF0083F92500E9
:10BF2000008041001040BA000160EF0000000600F0
:10BF300053540000414300004B45000052520000A2
:10BF40005F450000525200004F5200000A0D0000F1
:10BF500000000000CF0278003220EF0083FB2500B4
:10BF6000008041001040BA000160EF0000000600B0
:10BF70004D4100005448000045520000525F00004F
:10BF800045520000524F0000520A00000D00000010
:10BF9000CF0278003220EF0063FD250000804100D1
:10BFA0001040BA000160EF0000000600444D0000A0
:10BFB00041450000525200005F450000525200000F
:10BFC0004F5200000A0D000000000000CF02780070
:10BFD0003220EF0043FF2500008041001040BA00EE
:10BFE0000160EF0000000600202000002042000059
:10BFF00065670000696E0000204E00006F7700004A
:10C000002020000020200000202000000000000070
:10C01000CF0278003220EF0063012600008041004B
:10C020001040BA000160EF00000006002020000070
:10C03000202000002025000073000000CF027800BF
:10C040003220EF00C3022600008041001040BA00F9
:10C050000160EF0000000600204900006E6900004A
:10C0600074690000616C00007A65000020450000E2
:10C0700045500000726F00006D20000000000000BD
:10C08000CF0278003220EF00E30426000080410058
:10C090001040BA000160EF000000060020450000DB
:10C0A00045500000726F00006D200000496E0000D6
:10C0B00069740000696100006C7A0000656400002A
:10C0C00020000000CF0278003220EF000307260096
:10C0D000008041001040BA000160EF00000006003F
:10C0E000204C00006F610000646900006E67000072
:10C0F0002044000065660000617500006C7400005B
:10C100007320000000000000CF0278003220EF0012
:10C1100023092600008041001040BA000160EF00B2
:10C120000000060020200000202000002052000017
:10C130006573000065740000204D000075780000F4
:10C14000202500007520000000000000CF027800CC
:10C150004200F8003600F800801F78002000200020
:10C160000C000900B01F78000100200001007800D9
:10C17000505F0200000000008100E800811F78008D
:10C180002322AF00FEFF370020118800CF00780087
:10C19000E00020000008E600F4FF37008020A9003E
:10C1A0008020A900A00120000C0009004F10780099
:10C1B0004F0078003600F9004200F9000040060008
:10C1C0004200F8003600F800801F780020002000B0
:10C1D0000C000900B01F7800010020000100780069
:10C1E0006E5F0200000000008100E800811F7800FF
:10C1F0002322AF00FEFF370020118800CF00780017
:10C20000E00020000008E600F4FF37008060A9008D
:10C210008060A900A00120000C0009004F107800E8
:10C220004F0078003600F9004200F9000040060097
:10C230004200F8003600F800801F7800200020003F
:10C240000C000900B01F78000100200001007800F8
:10C250008C5F0200000000008100E800811F780070
:10C260002322AF00FEFF370020118800CF007800A6
:10C27000F00020000008E600F4FF37008040A9002D
:10C280008040A900A00120000C0009004F10780098
:10C290004F0078003600F9004200F9000040060027
:10C2A0004200F8003600F800801F780020002000CF
:10C2B0000C000900B01F7800010020000100780088
:10C2C000AC5F0200000000008100E800811F7800E0
:10C2D0002322AF00FEFF370020118800CF00780036
:10C2E000E00020000008E600F4FF37008080A9008D
:10C2F0008080A900A00120000C0009004F107800E8
:10C300004F0078003600F9004200F90000400600B6
:10C310004200F8003600F800801F7800200020005E
:10C320000C000900B01F7800010020000100780017
:10C33000CA5F0200000000008100E800811F780051
:10C340002322AF00FEFF370020118800CF007800C5
:10C35000D00020000008E600F4FF370080A0A9000C
:10C3600080A0A900A00120000C0009004F10780057
:10C370004F0078003600F9004200F9000040060046
:10C380004200F8003600F800801F780020002000EE
:10C390000C000900B01F780025CFBF000160EF003E
:10C3A0004100DD0004ED200084024000A40880006C
:10C3B000840298001421EF00247980004822DE00D6
:10C3C00083022000041CE100040036000000370056
:10C3D000256FEC00F061040000000000256FEF0005
:10C3E0008680A900A00120000C0009004F107800F1
:10C3F0004F0078003600F9004200F90000400600C6
:10C400004200F8003600F800801F7800200020006D
:10C410000C000900B01F780004002000042B8900E4
:10C4200004002000142B890004002000242B890024
:10C43000302B810000C0B300302B8900302B8100ED
:10C440000160EF00302B8900402B810000C0B30059
:10C45000402B8900402B81000160EF00402B8900B8
:10C46000502B810000C0B300502B8900502B81005D
:10C470000160EF00502B8900602B810000C0B300E9
:10C48000602B89009500A90000082800E422B7006D
:10C49000E602F8006025F900002B81000002780018
:10C4A0000008280004006000102B8900102B810078
:10C4B0008C8DB600202B8900202B81000000E0002D
:10C4C0003E00320000003700202B81006825F80074
:10C4D000F0FF9F006825F9006425F8004F00780000
:10C4E0004800DE006A25F800E0FF9F006A25F90099
:10C4F000402B81004800DE00542B8100044068007E
:10C500006625F800F0FF9F006625F9008CCDBF007E
:10C510006A25F800F0FF9F006A25F9008DCDBF0065
:10C520006C25F800E0FF9F006C25F900502B81007E
:10C53000542B81004822DE00044068006825F80082
:10C54000E0FF9F006825F900102B81006825F800A6
:10C55000F0FF9F006825F900402B81004800DE00B5
:10C56000642B8100044068006625F800E0FF9F000E
:10C570006625F900342B810004F0A7000100370084
:10C5800008003700342B81000470A600010037003A
:10C5900003003700902DED00D2620400000000007F
:10C5A000902DEC006225F8008C0DF9008B2DA80071
:10C5B0008E2DEF00E0620400000000008E2DEC00E4
:10C5C0000628EC0034408000037D20000418E100C0
:10C5D00019003E00000037000628EF0010A8AF0049
:10C5E00001003700040037000868EF008500A9004B
:10C5F0009500A800120037001028AF000100370096
:10C60000090037000868EC00C0CABF004440800041
:10C610000024E10004003900000037001008A800E1
:10C620001028A9000868EF008BEDAF00010037006B
:10C63000010037000968EC008500A9009500A800FA
:10C640008500A900A00120000C0009004F1078000F
:10C650004F0078003600F9004200F9000040060063
:10C660004200F8003600F800801F7800200020000B
:10C670000C000900B01F7800002B810000C0B3003F
:10C68000002B89002202AE00FEFF3700301180002F
:10C690006025F800E0FF9F006025F900C44180009C
:10C6A0004822DE00C3B4200083024200002B810038
:10C6B00080429800C44180004822DE00C3B42000BC
:10C6C00003004200104278006D24E10004003A00AB
:10C6D000000037004B6BEC0010C0B30011E8B7004E
:10C6E000C44180004822DE006142420004407800DC
:10C6F00000E0B700040820000024E10004003E0030
:10C70000000037003968EF008A6304000000000071
:10C710003968EC0010C8A8001A0AAE000100370002
:10C7200045003700BC4AAF00010037004200370027
:10C73000002B8100140220000024E10001003A00D7
:10C740000A003700002B8100240220000024E100B1
:10C7500001003A0005003700002B8100040320008F
:10C760000024E1000E003A0000003700645E800003
:10C7700013082000041CE10009003E0000003700FF
:10C78000645E800093082000041CE100040039006E
:10C7900000003700002B810000C0B300002B89008F
:10C7A000002B81006804E10001003A000500370019
:10C7B000002B8100F40720000024E10010003A0063
:10C7C0000000370080C0B3002322AF00FEFF370017
:10C7D00024E2B7002562EF0000C2B3002322AF00BD
:10C7E000FEFF370024E2B7002562EF0080C0B300EF
:10C7F0002322AF00FEFF370024E2B7002562EF00DE
:10C80000002B81007F04E1000B00360000003700A0
:10C81000002B8100F40720000024E1000600360010
:10C8200000003700002B81002322AF00FEFF3700FD
:10C8300024E2B7002562EF00002B8100CCEBB700AB
:10C840009560A8008560A900A00120000C000900E7
:10C850004F1078004F0078003600F9004200F900D0
:10C86000004006004200F8003600F800801F780003
:10C87000200020000C000900B01F7800002B810070
:10C8800000C0B300002B89003202AE00FEFF37006B
:10C89000B01180006025F800E0FF9F006025F900DE
:10C8A000645E80004822DE00E3BC20008302420078
:10C8B000002B810080429800645E80004822DE00E8
:10C8C000E3BC200003004200104278006D24E10028
:10C8D00004003A00000037004F6CEC0020C0B300A9
:10C8E00011E8B700645E80004822DE006142420029
:10C8F0000440780000E0B700040820000024E100B4
:10C9000004003E0000003700CD6BEF008C64040093
:10C9100000000000CD6BEC0010E8A8001A0AAE0081
:10C920000100370040003700BC4AAF00010037006B
:10C930003D003700002B8100140220000024E1009C
:10C9400001003A000A003700002B81002402200079
:10C950000024E10001003A0005003700002B8100AF
:10C96000040320000024E1000E003A00000037001C
:10C970008462800013082000041CE10009003E00CE
:10C98000000037008462800093082000041CE1004E
:10C990000400390000003700002B810000C0B30004
:10C9A000002B8900002B81006804E10010003A0090
:10C9B00000003700002B81003322AF00FEFF37005C
:10C9C00034E2B7003562EF0000C2B3003322AF009B
:10C9D000FEFF370034E2B7003562EF00002B810024
:10C9E0003322AF00FEFF370034E2B7003562EF00BC
:10C9F000002B81007F04E1000B00360000003700AF
:10CA0000002B8100F40720000024E100060036001E
:10CA100000003700002B81003322AF00FEFF3700FB
:10CA200034E2B7003562EF00002B810050ECB70014
:10CA300097C0A80087C0A900A00120000C00090031
:10CA40004F1078004F0078003600F9004200F900DE
:10CA5000004006000000E0004220AF000400370064
:10CA6000793E0900000000000000E900F9FF3700EE
:10CA700000000600249A80006124E10004003A00CE
:10CA8000D262A900D662A9004C6504000000000033
:10CA9000D262A900D662A800D222A900D622A8009C
:10CAA000D642A900D242A9001E00090000000000E1
:10CAB000D822EF0045D3BF00DCE2B700DD62EF0013
:10CAC0001E00090000000000D642A800D242A900C2
:10CAD0001E000900000000000000060000CBB300AB
:10CAE0003DF3B7003E13A800E49980006924E100FB
:10CAF0000300360080C0B3003CF3B7003E13A9002A
:10CB00003DD3BF003C53B4003DF3B70010C0B300A9
:10CB100044F3B7003DD3BF0045F3B7003A650200C8
:10CB2000000000000040EB003E13AF000000E800F2
:10CB300000000600851F78003D73EF003E73EF0094
:10CB40003F13A800E499800033082000041CE10092
:10CB50000300310030C8B3003CF3B7003F13A90015
:10CB60003CD3BF003DF3B7003CD3BF000160EF00F2
:10CB70004400DE00704070003EF3B70010C0B30008
:10CB800044F3B7003ED3BF0045F3B7003A65020057
:10CB900000000000A00020002A6502000000000044
:10CBA0003CD3BF00EF42600010C0B30044F3B700B5
:10CBB0000540780045F3B7003A6502000000000028
:10CBC000A00020002A650200000000000040EB00E9
:10CBD0003F13AF000000E800CF027800000006001D
:10CBE0002D72EF002E72EF00649180006824E10046
:10CBF0000400360080C0B3002DF2B70006660400C2
:10CC0000000000002CD2BF002DF2B7002CD2BF00D4
:10CC10003CF3B7006E650200000000003C73EF00BB
:10CC20009A650200000000002E72EF0074918000EF
:10CC300043082000041CE100070036004473EF00A5
:10CC40004573EF003A650200000000002E72EC0010
:10CC5000166604000000000010C0B30000E0B7003A
:10CC600000000600FE71EF00FE71EF00F48F8000FF
:10CC70006924E10007003100FED1BF002CF2B700AB
:10CC8000F065020000000000FE71EC003666040052
:10CC9000000000000000060010C0B30044F3B7001D
:10CCA000E0CAB30045F3B7003A6502000000000097
:10CCB000D282A900D682A9003E010900000000002E
:10CCC000D282A900D682A800803E20002A650200F8
:10CCD0000000000010C0B30044F3B70080C2B300EE
:10CCE00045F3B7003A6502000000000010C0B30031
:10CCF00044F3B70020CEB30045F3B7003A65020015
:10CD00000000000010C0B30044F3B70000C1B3003E
:10CD100045F3B7003A6502000000000010C0B30000
:10CD200044F3B7004573EF003A65020000000000CD
:10CD300010C0B30044F3B70000CBB30045F3B70015
:10CD40003A6502000000000010C0B30044F3B700D1
:10CD500000C4B30045F3B7003A65020000000000CC
:10CD600010C0B30044F3B70010CAB30045F3B700D6
:10CD70003A6502000000000010C0B30044F3B700A1
:10CD800000CCB30045F3B7003A6502000000000094
:10CD900010C0B30044F3B700F0CAB30045F3B700C6
:10CDA0003A65020000000000400620002A650200EB
:10CDB0000000000010C0B30044F3B70070CEB30011
:10CDC00045F3B7003A650200000000003266020039
:10CDD00000000000200320002A650200000000007F
:10CDE00000000600851F78003F73EF004073EF00DE
:10CDF000F499800003022000041CE10020003E00A2
:10CE0000F4998000F3032000041CE1001C003900A9
:10CE1000F49980000442B100044078003FF3B70069
:10CE20004073EF00049A80006524E1001200310095
:10CE3000F49980004822DE006520B8008002780066
:10CE4000049A80000960EF0004804200A48320005F
:10CE500004004000904278004473EF0005407800E1
:10CE600045F3B7003A650200000000004073EC0093
:10CE70001267040000000000FE67040000000000CC
:10CE8000F499800003042000041CE10020003E000F
:10CE9000F4998000F3052000041CE1001C00390017
:10CEA000F49980000444B100044078003FF3B700D7
:10CEB0004073EF00049A80006524E1001200310005
:10CEC000F49980004822DE006520B80080027800D6
:10CED000049A80000960EF0004804200A48D2000C5
:10CEE00004004000904278004473EF000540780051
:10CEF00045F3B7003A650200000000004073EC0003
:10CF00005A67040000000000FE67040000000000F3
:10CF1000F499800003062000041CE10020003E007C
:10CF2000F4998000F3072000041CE1001C00390084
:10CF3000F49980000446B100044078003FF3B70044
:10CF40004073EF00049A80006524E1001200310074
:10CF5000F49980004822DE006520B8008002780045
:10CF6000049A80000960EF0004804200A49720002A
:10CF700004004000904278004473EF0005407800C0
:10CF800045F3B7003A650200000000004073EC0072
:10CF9000A267040000000000FE670400000000001B
:10CFA0003F73EF004073EF00049A80006524E100B6
:10CFB00012003100F49980004822DE006520B8009C
:10CFC00080027800049A80000960EF00048042002B
:10CFD000A483200004004000904278004473EF00D6
:10CFE0000540780045F3B7003A65020000000000F4
:10CFF0004073EC00D46704000000000010C0B300D0
:10D0000000E0B700CF02780000000600851F78001E
:10D010003573EF0030D3BF003CF3B7006E650200FC
:10D020000000000031D3BF003CF3B7009A65020056
:10D03000000000003573EF0035D3BF00A4998000D5
:10D040000024E10015003400A49980004822DE008D
:10D05000040078003213B400904278003E13F800C8
:10D06000E5FF9F003E13F900F26602000000000099
:10D070004473EF004573EF003A65020000000000C2
:10D080004473EF004573EF003A65020000000000B2
:10D090003573EC001C68040000000000CF0278002B
:10D0A00000000600F0FF2F000862AE000500370008
:10D0B00009C2AF00FEFF37001110880009C2AF009F
:10D0C000FEFF37000000200009E2AF000000E8008A
:10D0D000000006000862AE00040037000622A80027
:10D0E0000622AF00FEFF3700030037000602A8004B
:10D0F0000602AF00FEFF3700510F810052680200A8
:10D1000000000000EA21F800CF007800C808DE0027
:10D110005268020000000000610F810052680200A6
:10D1200000000000F00120000602B600FDFF3A00FA
:10D130000642A8000642AF00FEFF3700BE0009000D
:10D140000000000000000600F0FF2F000862AE00A3
:10D1500011003700321080007F016100FDFF3A00AE
:10D160000662A8000100A70006A2A9000100A6000F
:10D1700006A2A800321080007F016100FDFF3A0086
:10D180000682A8000822AE00FEFF370000108000D3
:10D1900008C2AF0008C2A90000000600851F780081
:10D1A0000862AE00040037000622A8000622AF0085
:10D1B000FEFF3700030037000602A8000602AF009A
:10D1C000FEFF370031988000526802000000000026
:10D1D00007D3BF0080007800526802000000000002
:10D1E0000862AE00040037000622A8000622AF0045
:10D1F000FEFF3700030037000602A8000602AF005A
:10D20000FEFF370006D3BF00E14270008540780082
:10D2100052680200000000004598800001002000D4
:10D22000811F7800CF007800A46802000000000091
:10D23000804A7800F00120000602B600FDFF3A00A7
:10D240000642A8000642AF00FEFF3700BE000900FC
:10D2500000000000459880000540900000E0B70005
:10D26000CF02780000000600F0FF2F001862AE0029
:10D270000500370019C2AF00FEFF3700911088008B
:10D2800019C2AF00FEFF37000000200019E2AF0016
:10D290000000E800000006001862AE00040037003D
:10D2A0001622A8001622AF00FEFF37000300370049
:10D2B0001602A8001602AF00FEFF3700319880006A
:10D2C000346902000000000007D3BF00800078002E
:10D2D00034690200000000004198800034690200B7
:10D2E00000000000F00120001602B600FDFF3A0029
:10D2F0001642A8001642AF00FEFF3700BE0009002C
:10D300000000000000000600FE71EF00500F8100D9
:10D3100000CBB300500F8900500F81000080FD004A
:10D3200080C1B3000080FD00500F8900600F8100B4
:10D33000F0CFB300600F89006A68020000000000AF
:10D34000500F810000CBB300500F8900500F8100B7
:10D350000080FD0090C1B3000080FD00500F8900E7
:10D36000600F8100F0CFB300600F89006A6802008F
:10D3700000000000500F810000CBB300500F890067
:10D38000500F81000080FD00A0C1B3000080FD00AF
:10D39000500F8900600F8100F0CFB300600F89004B
:10D3A0006A68020000000000500F810000CBB3004B
:10D3B000500F8900500F81000080FD00B0C1B30004
:10D3C0000080FD00500F8900600F8100F0CFB30096
:10D3D000600F89006A68020000000000500F8100A1
:10D3E00000CBB300500F8900500F81000080FD007A
:10D3F000C0C1B3000080FD00500F8900600F8100A4
:10D40000F0CFB300600F89006A68020000000000DE
:10D41000500F810000CBB300500F8900500F8100E6
:10D420000080FD0000C2B3000080FD00500F8900A5
:10D43000600F810000C0B300600F89006A680200BD
:10D4400000000000500F810000CBB300500F890096
:10D45000500F81000080FD0010C2B3000080FD006D
:10D46000500F8900600F810000C0B300600F890079
:10D470006A68020000000000500F810000CBB3007A
:10D48000500F8900500F81000080FD0020C2B300C2
:10D490000080FD00500F8900600F810000C0B300C4
:10D4A000600F89006A68020000000000500F8100D0
:10D4B00000CBB300500F8900500F81000080FD00A9
:10D4C00030C2B3000080FD00500F8900600F810062
:10D4D00000C0B300600F89006A680200000000000D
:10D4E000500F810000CBB300500F8900500F810016
:10D4F0000080FD0040C2B3000080FD00500F890095
:10D50000600F810000C0B300600F89006A680200EC
:10D510000000000000CBB30006F3B7000773EF0074
:10D52000E41F210044988800CE680200000000003B
:10D53000FEF1B70000CBB30006F3B70010C0B30094
:10D5400007F3B700E41F210044988800CE6802006A
:10D5500000000000FEF1B70000CBB30006F3B700F7
:10D5600020C0B30007F3B700E41F210044988800EF
:10D57000CE68020000000000FEF1B70000CBB3004F
:10D5800006F3B70030C0B30007F3B700E41F210073
:10D5900044988800CE68020000000000FEF1B70049
:10D5A00000CBB30006F3B70040C0B30007F3B700E9
:10D5B000E41F210044988800CE68020000000000AB
:10D5C000FEF1B700500F810080CBB300500F8900EF
:10D5D000500F81000080FD0080C1B3000080FD007D
:10D5E000500F8900600F810010C0B300600F8900E8
:10D5F0006A68020000000000500F810080CBB30079
:10D60000500F8900500F81000080FD0090C1B300D1
:10D610000080FD00500F8900600F8100F0CFB30043
:10D62000600F89006A68020000000000500F81004E
:10D6300080CBB300500F8900500F81000080FD00A7
:10D64000A0C1B3000080FD00500F8900600F810071
:10D65000F0CFB300600F89006A680200000000008C
:10D66000500F810080CBB300500F8900500F810014
:10D670000080FD00B0C1B3000080FD00500F8900A4
:10D68000600F8100F0CFB300600F89006A6802006C
:10D6900000000000500F810080CBB300500F8900C4
:10D6A000500F81000080FD00C0C1B3000080FD006C
:10D6B000500F8900600F8100F0CFB300600F890028
:10D6C0006A68020000000000500F810080CBB300A8
:10D6D000500F8900500F81000080FD0000C2B30090
:10D6E0000080FD00500F8900600F8100E0CFB30083
:10D6F000600F89006A68020000000000500F81007E
:10D7000080CBB300500F8900500F81000080FD00D6
:10D7100010C2B3000080FD00500F8900600F81002F
:10D7200000C0B300600F89006A68020000000000BA
:10D73000500F810080CBB300500F8900500F810043
:10D740000080FD0020C2B3000080FD00500F890062
:10D75000600F810000C0B300600F89006A6802009A
:10D7600000000000500F810080CBB300500F8900F3
:10D77000500F81000080FD0030C2B3000080FD002A
:10D78000500F8900600F810000C0B300600F890056
:10D790006A68020000000000500F810080CBB300D7
:10D7A000500F8900500F81000080FD0040C2B3007F
:10D7B0000080FD00500F8900600F810000C0B300A1
:10D7C000600F89006A6802000000000080CBB3008F
:10D7D00006F3B7000773EF00E41F210044988800A8
:10D7E000CE68020000000000FEF1B70080CBB3005D
:10D7F00006F3B70010C0B30007F3B700E41F210021
:10D8000044988800CE68020000000000FEF1B700D6
:10D8100080CBB30006F3B70020C0B30007F3B70016
:10D82000E41F210044988800CE6802000000000038
:10D83000FEF1B70080CBB30006F3B70030C0B300F1
:10D8400007F3B700E41F210044988800CE68020067
:10D8500000000000FEF1B70080CBB30006F3B70074
:10D8600040C0B30007F3B700E41F210044988800CC
:10D87000CE68020000000000FEF1B700500F8100EA
:10D8800000C5B300500F8900500F81000080FD00DB
:10D8900080C1B3000080FD00500F8900600F81003F
:10D8A000F0CFB300600F89006A680200000000003A
:10D8B000500F810000C5B300500F8900500F810048
:10D8C0000080FD0090C1B3000080FD00500F890072
:10D8D000600F8100F0C1B300600F89006A68020028
:10D8E00000000000500F810000C5B300500F8900F8
:10D8F000500F81000080FD00A0C1B3000080FD003A
:10D90000500F8900600F810000C0B300600F8900D4
:10D910006A68020000000000500F810000C5B300DB
:10D92000500F8900500F81000080FD00B0C1B3008E
:10D930000080FD00500F8900600F8100E0C7B30038
:10D94000600F89006A68020000000000500F81002B
:10D9500000C5B300500F8900500F81000080FD000A
:10D96000C0C1B3000080FD00500F8900600F81002E
:10D9700000C0B300600F89006A6802000000000068
:10D98000500F810000C5B300500F8900500F810077
:10D990000080FD0000C2B3000080FD00500F890030
:10D9A000600F810000C0B300600F89006A68020048
:10D9B00000000000500F810000C5B300500F890027
:10D9C000500F81000080FD0010C2B3000080FD00F8
:10D9D000500F8900600F810000CEB300600F8900F6
:10D9E0006A68020000000000500F810000C5B3000B
:10D9F000500F8900500F81000080FD0020C2B3004D
:10DA00000080FD00500F8900600F810000C0B3004E
:10DA1000600F89006A68020000000000500F81005A
:10DA200000C5B300500F8900500F81000080FD0039
:10DA300030C2B3000080FD00500F8900600F8100EC
:10DA400010C8B300600F89006A680200000000007F
:10DA5000500F810000C5B300500F8900500F8100A6
:10DA60000080FD0040C2B3000080FD00500F89001F
:10DA7000600F8100F0CFB300600F89006A68020078
:10DA80000000000000C5B30006F3B7000773EF0005
:10DA9000E41F210044988800CE68020000000000C6
:10DAA000FEF1B70000C5B30006F3B70010C0B30025
:10DAB00007F3B700E41F210044988800CE680200F5
:10DAC00000000000FEF1B70000C5B30006F3B70088
:10DAD00030C0B30007F3B700E41F2100449888006A
:10DAE000CE68020000000000FEF1B700C0CBB3001A
:10DAF00006F3B70080C1B30007F3B7000873EF0067
:10DB00004C69020000000000C0CBB30006F3B70070
:10DB100090C1B30007F3B7000873EF004C6902002F
:10DB200000000000C0CBB30006F3B700A0C1B300F3
:10DB300007F3B7000873EF004C6902000000000013
:10DB4000C0CBB30006F3B700B0C1B30007F3B70012
:10DB50000873EF004C69020000000000C0CBB30066
:10DB600006F3B700C0C1B30007F3B7000873EF00B6
:10DB70004C69020000000000C0CBB30006F3B70000
:10DB800000C2B30007F3B70008F3EF004C690200CE
:10DB900000000000C0CBB30006F3B70010C2B30012
:10DBA00007F3B70008F3EF004C6902000000000023
:10DBB000C0CBB30006F3B70020C2B30007F3B70031
:10DBC00008F3EF004C69020000000000C0CBB30076
:10DBD00006F3B70030C2B30007F3B70008F3EF0055
:10DBE0004C69020000000000C0CBB30006F3B70090
:10DBF00040C2B30007F3B70008F3EF004C6902001E
:10DC000000000000F40F200094628800C0CBB30035
:10DC100006F3B70080C0B30007F3B70052CCBF00D3
:10DC200008F3B7004C69020000000000F40F200068
:10DC3000A4628800C0CBB30006F3B70090C0B30065
:10DC400007F3B70054CCBF0008F3B7004C690200DB
:10DC500000000000C0CBB30006F3B700A0C0B300C3
:10DC600007F3B7000873EF004C69020000000000E2
:10DC7000F40F2000B4628800C0CBB30006F3B700F5
:10DC8000B0C0B30007F3B70056CCBF0008F3B7002D
:10DC90004C69020000000000C0CBB30006F3B700DF
:10DCA000C0C0B30007F3B7000873EF004C6902006F
:10DCB0000000000020C4B30006F3B70040C0B3006A
:10DCC00007F3B7000873EF004C6902000000000082
:10DCD00020C4B30006F3B70050C0B30007F3B70089
:10DCE0000873EF004C6902000000000020C4B3007C
:10DCF00006F3B70060C0B30007F3B7000873EF0086
:10DD00004C6902000000000020C4B30006F3B70015
:10DD100070C0B30007F3B7000873EF004C6902004E
:10DD20000000000020C4B30006F3B70020C0B30019
:10DD300007F3B70008F3EF004C6902000000000091
:10DD400020C4B30006F3B70030C0B30007F3B70038
:10DD500008F3EF004C69020000000000000006001C
:10DD6000811F7800618E8000805878008048EB0029
:10DD7000CF007800CC31EC000000060060C5B30095
:10DD80000EEBB7000F6BEF00106BEF0090C1B3000C
:10DD900011EBB700126BEF0000C4B30013EBB70038
:10DDA00010C0B30014EBB70000C4B30015EBB7000C
:10DDB000E0C1B30016EBB700176BEF00186BEF0074
:10DDC000196BEF0020C0B3001AEBB70020C0B300FE
:10DDD0001BEBB70020C0B3001CEBB70020C0B300A2
:10DDE0001DEBB70020C0B3001EEBB70020C0B3008E
:10DDF0001FEBB70020C0B30020EBB70020C0B3007A
:10DE000021EBB70020C1B30022EBB700C0C0B300C4
:10DE100023EBB70050C0B30024EBB70080C1B300C0
:10DE200025EBB70080C1B30026EBB70080C1B3007B
:10DE300027EBB70080C1B30028EBB70080C1B30067
:10DE400029EBB70080C1B3002AEBB70080C1B30053
:10DE50002BEBB70040C1B3002CEBB70040C1B300BF
:10DE60002DEBB70040C1B3002EEBB70040C1B300AB
:10DE70002FEBB70040C1B30030EBB70040C1B30097
:10DE800031EBB70040C1B30032EBB70070C0B30054
:10DE900033EBB70070C0B30034EBB70070C0B30011
:10DEA00035EBB70070C0B30036EBB70070C0B300FD
:10DEB00037EBB70070C0B30038EBB70070C0B300E9
:10DEC00039EBB70010C0B3003AEBB70010C0B30095
:10DED0003BEBB70010C0B3003CEBB70010C0B30081
:10DEE0003DEBB70010C0B3003EEBB70010C0B3006D
:10DEF0003FEBB70010C0B30040EBB700F0CFB3006A
:10DF000041EBB70042EBEF00F0CFB30043EBB700BB
:10DF100044EBEF00456BEF0046EBEF00F0CFB300B2
:10DF200047EBB70048EBEF00F0CFB30049EBB70089
:10DF30004AEBEF00000006000862AE000400370064
:10DF40000622A8000622AF00FEFF370003003700BC
:10DF50000602A8000602AF00FEFF370001CEB300A4
:10DF60005268020000000000510F81005268020058
:10DF700000000000F00120000602B600FDFF3A009C
:10DF80000642A8000642AF00FEFF3700BE000900AF
:10DF90000000000000000600851F78001C33EF0021
:10DFA00014002000E4988800E49880006720E100D5
:10DFB00018003100E4988000670242008402780073
:10DFC000EA21F800E5FF9F00EA21F9009C6F0200BA
:10DFD00000000000500F8100A0C9B300500F89005D
:10DFE000500F81000080FD00E0C1B3000080FD0003
:10DFF000500F8900600F810060CBB300600F890073
:10E000006A680200000000001C33EC00D46F0400BA
:10E0100000000000CC42A900D042A800140020005B
:10E02000E4988800E49880006720E1001E00310039
:10E03000E49880006702420084027800EA21F80038
:10E04000E5FF9F00EA21F9009C6F0200000000003C
:10E05000500020002A65020000000000500F8100DF
:10E0600020C4B300500F8900500F81000080FD00D4
:10E07000F0C0B3000080FD00500F8900600F8100E8
:10E0800040C4B300600F89006A680200000000000D
:10E09000500020002A650200000000001C33EC0044
:10E0A0001270040000000000CF027800000006009B
:10E0B000851F78004233EF004053E20002003A002F
:10E0C00010C0B30040F3B7000862AE000400370090
:10E0D0000622A8000622AF00FEFF3700030037002B
:10E0E0000602A8000602AF00FEFF370001CAB30017
:10E0F00052680200000000003DD3BF00800278009B
:10E10000854078005268020000000000E599800018
:10E110008540780052680200000000000862AE00EE
:10E12000040037000622A8000622AF00FEFF3700D9
:10E13000030037000602A8000602AF00FEFF37000A
:10E1400011CAB30052680200000000004233EF0021
:10E15000049A800061405200149A80000020E1007F
:10E160000C003100109A80003E13B4008002780049
:10E1700011002000811F7800CF007800A468020001
:10E1800000000000804A78004233EC00A8700400D0
:10E1900000000000049A8000614052000080FB00F3
:10E1A000F49980008402400001002000811F780063
:10E1B000CF007800A468020000000000804A7800C8
:10E1C000F00120000602B600FDFF3A000642A8005A
:10E1D0000642AF00FEFF3700DE000900000000002D
:10E1E000000020003E13B40080027800054090003B
:10E1F00000E0B700CF02780000000600851F78001D
:10E200001852E20021003200A09080009042780075
:10E21000B09080000002780014407800002CE100EB
:10E220000E003200A090800090427800B0908000F4
:10E230000002780014407800002CE1000300310057
:10E2400000C0EB00287104000000000010C0B30003
:10E250000F0037003871040000000000A09080001B
:10E260001004E00002003A000060EF0008003700F0
:10E27000A09080001432EC00B09080001632EC00C8
:10E280001872ED0000710400000000000060EF0053
:10E29000CF02780000000600851F7800FE71EF00B5
:10E2A00004022200049088000402220014908800D6
:10E2B0000402220024908800040222003490880086
:10E2C0000402220044908800040222005490880036
:10E2D00004022200649088000402220074908800E6
:10E2E00004022200849088001272EF0020C1B30063
:10E2F00040F3B700E4FC2100E499880004202100E9
:10E30000F49988005870020000000000FEF1B70088
:10E3100020C1B30018F2B70004202100A4908800A7
:10E3200064822000B4908800FE70020000000000AB
:10E330000004E00004003A000060EF000400370031
:10E34000A87104000000000000E0EF0000003700AA
:10E35000CF02780000000600851F78003013F80017
:10E360003613F9003453E2000C003200909980001B
:10E370001004E00009003200B09980003633EC0050
:10E3800080027800909980003233EC00904A780047
:10E390003473ED00B2710400000000003453E20059
:10E3A00007003200B09980003633EC00800278001C
:10E3B000804AEB003473ED00CE71040000000000D1
:10E3C0003013F8000000F900CF02780000000600CA
:10E3D000C131210002002000120009008058EB002A
:10E3E00020C1B30034F3B700C43121008499880000
:10E3F0001A13F8003213F900AC710200000000009B
:10E4000070C0B30030F3B7003173EF0020C1B30028
:10E4100034F3B700C43121009499880006680200E3
:10E420000000000000000600851F78003633EF0072
:10E430000862AE00040037000622A8000622AF00E2
:10E44000FEFF3700030037000602A8000602AF00F7
:10E45000FEFF370001CAB30052680200000000004E
:10E4600031D3BF00800278008540780052680200F6
:10E470000000000085998000854078005268020005
:10E48000000000003633EF00B0998000A4998000AE
:10E490000960EF000020E10009003600B09980001B
:10E4A0003213B40090427800854078005268020030
:10E4B000000000003633EC0044720400000000004D
:10E4C000F00120000602B600FDFF3A000642A80057
:10E4D0000642AF00FEFF3700BE000900000000004A
:10E4E000CF02780000000600851F78000862AE00A9
:10E4F000040037000622A8000622AF00FEFF370006
:10E50000030037000602A8000602AF00FEFF370036
:10E5100001CAB300526802000000000031D3BF00FE
:10E5200080027800854078005268020000000000F8
:10E530008599800085407800526802000000000044
:10E54000919980005268020000000000F001200054
:10E550000602B600FDFF3A000642A8000642AF00E0
:10E56000FEFF3700BE00090000000000CF02780067
:10E5700000000600844080004822DE006124E100A3
:10E5800007003A00500F81002322AF00FEFF370042
:10E5900024E2B7002562EF00DA72040000000000F8
:10E5A000500F81003322AF00FEFF370034E2B70086
:10E5B0003562EF0000000600851F78002C33EF0065
:10E5C0002B73EF003033EF002AD3BF0034F3B700D2
:10E5D000E4B020009499880014720200000000004A
:10E5E0002C33EF0060998000549980000960EF009F
:10E5F0000020E10009003600E4B0200063998000AB
:10E600000480410000027800144078002B73B400AD
:10E610002C33EC00F27204000000000054998000DA
:10E620004822DE00F4CFB200044078002BF3B7009C
:10E63000549980004822DE00614242000440780084
:10E640002BF3B7002AD3BF0030F3B7003173EF00CC
:10E650002BD3BF0032F3B700747202000000000039
:10E66000BD0AAE000F003700010020000100780055
:10E6700070190200000000008100E800811F78008E
:10E68000EA21F800E0FF9F00EA21F900BA720200D7
:10E6900000000000CF007800D00020000008E60055
:10E6A000F2FF3700CF027800000006002A32EF00A8
:10E6B0002C72EF002D72EF00E120210002002000FB
:10E6C0001B0009008058EB000405200054918800CD
:10E6D0002C72EF0064918000A3082000041CE1006C
:10E6E0000E00360000C1B30034F3B7002A12F80060
:10E6F0003013F900E420210094998800147202007C
:10E700000000000054918000700242005491880083
:10E710002C72EC006A7304000000000004902000DA
:10E72000549188002D72EF00649180004822DE0031
:10E730006624E100150031002C72EF006491800026
:10E740006E24E1000E003100C0C1B30034F3B70005
:10E750002A12F8003013F900E4202100949988006F
:10E760001472020000000000549180007C024200FC
:10E77000549188002C72EC009E730400000000008D
:10E780002D72EC00947304000000000000000600ED
:10E79000851F7800FE31EF000032EF000272EF00BB
:10E7A0000372EF000463230024908800D4A22400A5
:10E7B0003490880014E6260044908800D412230088
:10E7C000549088000403200064908800BE6E02000C
:10E7D00000000000D0C3B3002AF3B700DC720200CF
:10E7E00000000000567302000000000020C1B300CA
:10E7F00034F3B700E4FC210084998800648220008F
:10E8000094998800147202000000000004FE2100A8
:10E81000F48F88000032EF000272EF001490800045
:10E820007324E10028003100149080000960EF009B
:10E83000238120000300420090427800040320005E
:10E840000524E10004003E00940320000524E100BB
:10E8500001003900030037000040EB00347404006D
:10E860000000000010C0B3006104E10013003A0092
:10E87000049080006520E10010003E0014908000AC
:10E880000960EF002381200003004200104078005F
:10E8900003F2B70003D2BF0032F3B700FE11F80055
:10E8A0003013F90074720200000000000032EC0026
:10E8B000F48F800061024200F48F88000272EC0045
:10E8C0000E7404000000000090C0B30034F3B700E1
:10E8D00064FE2100849988004420210094998800D6
:10E8E0001472020000000000CF0278000000060051
:10E8F000851F7800C500200003000900B51F7800BF
:10E90000800378008404780004F0A1000400E00093
:10E9100006003A0009F0A7000200370005002000B9
:10E9200011003700050020000F003700E6425200BA
:10E930000C0039000003200009F0A60000022000AE
:10E94000EA21F800E0FF9F00EA21F900BA72020014
:10E95000000000008502E900F9FF3B00550020009F
:10E9600001003700840278006400200005E0A00068
:10E9700009F0A70005F0A0000871220011000900AD
:10E980008883D800FA740200000000008103780038
:10E99000883E2000110009008883D800FA74020024
:10E9A00000000000810378004806200011000900E3
:10E9B0008883D800FA740200000000008103780008
:10E9C000A8002000110009008883D800FA74020012
:10E9D000000000000003200000C04000EA21F80011
:10E9E000E0FF9F00EA21F900BA7202000000000077
:10E9F0001B003700060320000000E0000E003A0074
:10EA000005E0A6000D0037000402E9000524E1003E
:10EA1000020032004200AF00000006000000E000EB
:10EA200005003A0005E0A6000400370005F0A60046
:10EA3000060220000100370005E0A100004043006D
:10EA4000811F7800EA21F800E0FF9F00EA21F90029
:10EA5000BA72020000000000CF007800000006003B
:10EA60002501200003000900CF127800CF027800B2
:10EA700000000600851F78000862AE000400370021
:10EA80000622A8000622AF00FEFF37000300370071
:10EA90000602A8000602AF00FEFF370001CAB3005D
:10EAA000526802000000000035D3BF0080027800E9
:10EAB000854078005268020000000000A59980009F
:10EAC0008540780052680200000000000862AE0035
:10EAD000040037000622A8000622AF00FEFF370020
:10EAE000030037000602A8000602AF00FEFF370051
:10EAF00011CAB3005268020000000000B5998000FE
:10EB000001002000811F7800CF007800A468020077
:10EB100000000000804A7800F00120000602B600E4
:10EB2000FDFF3A000642A8000642AF00FEFF370094
:10EB3000DE00090000000000B5998000054090004B
:10EB400000E0B700CF02780000000600851F7800C3
:10EB5000861F78000001EB000103780064C11000FB
:10EB60004211DD000200DD00800278000C60EC0044
:10EB70000C60ED000F00320005007800C42ADD00B3
:10EB80004C00DE00F000B2000003B000A203200041
:10EB90000200E100010039000D40B400EA21F80054
:10EBA000E0FF9F00EA21F900BA72020000000000B5
:10EBB000EFFF37004F037800CF0278000000060017
:10EBC000851F78002C33EF002E33EF002B73EF00FE
:10EBD0003073EF003173EF002E33EF007499800033
:10EBE0006220E100BE0031002AD3BF0040F3B7002D
:10EBF0002C13F8003C13F900E4B02000F4998800CD
:10EC000058700200000000000EEBB700BD0AAE0015
:10EC1000230037000100200001007800BC1802002A
:10EC2000000000008100E800811F7800EA21F80060
:10EC3000E0FF9F00EA21F900BA7202000000000024
:10EC4000CF007800D00020000008E600F2FF370077
:10EC50002AD3BF000160EF00040020007874020096
:10EC600000000000500F810090C2B300500F8900D7
:10EC7000BA72020000000000500F8100A0C3B30070
:10EC8000500F8900BA72020000000000500F81008E
:10EC900000C2B300500F8900BA72020000000000E9
:10ECA0002C33EF0060998000549980000960EF00D8
:10ECB0000020E1000F003600E4B0200063998000DE
:10ECC0000480410000027800144078002B73B400E7
:10ECD0002C13F8003413F90014332100B499880080
:10ECE0003A750200000000002C33EC00527604005C
:10ECF00000000000549980004822DE00F4CFB200EA
:10ED0000044078002BF3B700549980004822DE00BD
:10ED100061424200044078002BF3B7002AD3BF00C1
:10ED20002CF3B7002D73EF002C13F8003413F90007
:10ED300004332100B49988003A75020000000000F5
:10ED400030F3B70030D3BF002B53E30028003A0064
:10ED5000BD0AAE002300370001002000010078004A
:10ED6000DE180200000000008100E800811F78002A
:10ED7000EA21F800E0FF9F00EA21F900BA720200E0
:10ED800000000000CF007800900020000008E6009E
:10ED9000F2FF370030D3BF000160EF002170220086
:10EDA000A675020000000000D100200001007800DC
:10EDB000DE180200000000008100E800811F7800DA
:10EDC000EA21F800E0FF9F00EA21F900BA72020090
:10EDD00000000000CF007800300120000008E600AD
:10EDE000F2FF370010C0B30000E0B7007100370039
:10EDF000BD0AAE0037003700010020000100780096
:10EE000002190200000000008100E800811F780064
:10EE1000EA21F800E0FF9F00EA21F900BA7202003F
:10EE200000000000CF007800900020000008E600FD
:10EE3000F2FF370030D3BF000160EF0021702200E5
:10EE4000A675020000000000D1002000010078003B
:10EE500002190200000000008100E800811F780014
:10EE6000EA21F800E0FF9F00EA21F900BA720200EF
:10EE700000000000CF007800900120000008E600AC
:10EE8000F2FF37002BD3BF000160EF00217022009A
:10EE9000A675020000000000D101200001007800EA
:10EEA00002190200000000008100E800811F7800C4
:10EEB000EA21F800E0FF9F00EA21F900BA7202009F
:10EEC00000000000CF007800B00220000008E6003B
:10EED000F2FF37002E33EC00EE7504000000000056
:10EEE000BD0AAE00320037000100200001007800AA
:10EEF0003E190200000000008100E800811F780038
:10EF0000EA21F800E0FF9F00EA21F900BA7202004E
:10EF100000000000CF007800D00020000008E600CC
:10EF2000F2FF370030D3BF000160EF0021702200F4
:10EF3000A675020000000000110120000100780009
:10EF40003E190200000000008100E800811F7800E7
:10EF5000EA21F800E0FF9F00EA21F900BA720200FE
:10EF600000000000CF007800D00120000008E6007B
:10EF7000F2FF37002BD3BF000160EF0021702200A9
:10EF8000A675020000000000500F8100A0C0B30071
:10EF9000500F8900BA72020000000000500F81007B
:10EFA000D0C0B300500F8900BA7202000000000008
:10EFB0000060EF00CF02780000000600851F780097
:10EFC000D0C3B3002AF3B700E075020000000000D0
:10EFD0006104E10013003200BD0AAE000F003700EB
:10EFE00001002000010078008E19020000000000DE
:10EFF0008100E800811F7800EA21F800E0FF9F000F
:10F00000EA21F900BA72020000000000CF00780087
:10F01000400220000008E600F2FF3700BE6E02004A
:10F02000000000000ECBBF00BCEAB7000FCBBF0052
:10F03000BDEAB70011CBBF00C6EAB70013CBBF00D3
:10F04000BEEAB70014CBBF00BFEAB70015CBBF00C4
:10F0500021EAB70016CBBF0022EAB70017CBBF00EA
:10F06000C1EAB70018CBBF00C2EAB70019CBBF0096
:10F07000C0EAB7001ACBBF00DFEAB7001BCBBF0066
:10F08000E0EAB7001CCBBF00E1EAB7001DCBBF0030
:10F09000E2EAB7001ECBBF00E3EAB7001FCBBF0018
:10F0A000E4EAB70020CBBF00E5EAB70021CBBF0000
:10F0B000E7EAB70022CBBF00C4EAB70023CBBF000A
:10F0C000C3EAB70024CBBF00C5EAB70025CBBF0019
:10F0D000C7EAB70026CBBF00C8EAB70027CBBF00FE
:10F0E000C9EAB70028CBBF00CAEAB70029CBBF00E6
:10F0F000CBEAB7002ACBBF00CCEAB7002BCBBF00CE
:10F10000CDEAB7002CCBBF00CFEAB7002DCBBF00B4
:10F11000D0EAB7002ECBBF00D1EAB7002FCBBF009B
:10F12000D2EAB70030CBBF00D3EAB70031CBBF0083
:10F13000D4EAB70032CBBF00D5EAB70033CBBF006B
:10F14000D7EAB70034CBBF00D8EAB70035CBBF0051
:10F15000D9EAB70036CBBF00DAEAB70037CBBF0039
:10F16000DBEAB70038CBBF00DCEAB70039CBBF0021
:10F17000DDEAB7003ACBBF00E9EAB7003BCBBF00FE
:10F18000EAEAB7003CCBBF00EBEAB7003DCBBF00DB
:10F19000ECEAB7003ECBBF00EDEAB7003FCBBF00C3
:10F1A000EEEAB70040CBBF00EFEAB70041CBBF00AB
:10F1B00062ECB70042CBBF0061ECB70043CBBF00AD
:10F1C00060ECB70044CBBF005FECB70045CBBF009D
:10F1D0005EECB70046CBBF005CECB70047CBBF008E
:10F1E0005BECB70048CBBF005AECB70049CBBF007F
:10F1F00059ECB7004ACBBF0058ECB7001A2AEF0011
:10F20000CF02780000000600851F78000233EF006F
:10F210000053E20002003A0010C0B30000F3B70050
:10F220000862AE00040037000622A8000622AF00E4
:10F23000FEFF3700030037000602A8000602AF00F9
:10F24000FEFF3700E19780005268020000000000D6
:10F25000E5978000C82ADE000548B30085407800A5
:10F2600052680200000000000862AE00040037008F
:10F270000622A8000622AF00FEFF37000300370079
:10F280000602A8000602AF00FEFF3700FCD2BF0056
:10F29000E1427000854078005268020000000000E2
:10F2A0000233EF00049880006140520014988000FF
:10F2B0000020E1000C00310010988000FE12B40024
:10F2C0008002780011002000811F7800CF007800B4
:10F2D000A468020000000000804A78000233EC00BD
:10F2E0005279040000000000049880006140520040
:10F2F0000080FB00F49780008402400001002000A1
:10F30000811F7800CF007800A46802000000000090
:10F31000804A7800F00120000602B600FDFF3A00A6
:10F320000642A8000642AF00FEFF3700BE000900FB
:10F330000000000000002000FE12B40080027800EF
:10F340000540900000E0B700CF0278000000060002
:10F35000851F7800BCCABF000EEBB700BDCABF0056
:10F360000FEBB700106BEF00C6CABF0011EBB70080
:10F37000126BEF00BECABF0013EBB700BFCABF00DD
:10F3800014EBB70021CABF0015EBB70022CABF00BB
:10F3900016EBB700C1CABF0017EBB700C2CABF0067
:10F3A00018EBB700C0CABF0019EBB700DFCABF0037
:10F3B0001AEBB700E0CABF001BEBB700E1CABF0001
:10F3C0001CEBB700E2CABF001DEBB700E3CABF00E9
:10F3D0001EEBB700E4CABF001FEBB700E5CABF00D1
:10F3E00020EBB700E7CABF0021EBB700C4CABF00DB
:10F3F00022EBB700C3CABF0023EBB700C5CABF00EA
:10F4000024EBB700C7CABF0025EBB700C8CABF00CE
:10F4100026EBB700C9CABF0027EBB700CACABF00B6
:10F4200028EBB700CBCABF0029EBB700CCCABF009E
:10F430002AEBB700CDCABF002BEBB700CFCABF0085
:10F440002CEBB700D0CABF002DEBB700D1CABF006C
:10F450002EEBB700D2CABF002FEBB700D3CABF0054
:10F4600030EBB700D4CABF0031EBB700D5CABF003C
:10F4700032EBB700D7CABF0033EBB700D8CABF0022
:10F4800034EBB700D9CABF0035EBB700DACABF000A
:10F4900036EBB700DBCABF0037EBB700DCCABF00F2
:10F4A00038EBB700DDCABF0039EBB700E9CABF00CF
:10F4B0003AEBB700EACABF003BEBB700EBCABF00AC
:10F4C0003CEBB700ECCABF003DEBB700EDCABF0094
:10F4D0003EEBB700EECABF003FEBB700EFCABF007C
:10F4E00040EBB70062CCBF0041EBB70061CCBF007E
:10F4F00042EBB70060CCBF0043EBB7005FCCBF006E
:10F5000044EBB7005ECCBF0045EBB7005CCCBF005E
:10F5100046EBB7005BCCBF0047EBB7005ACCBF004F
:10F5200048EBB70059CCBF0049EBB70058CCBF003F
:10F530004AEBB700D0C3B3002AF3B700DC72020075
:10F5400000000000D0C3B3002AF3B700E07502004A
:10F55000000000006104E10011003200BD0AAE00AD
:10F560000F0037000100200001007800C2190200DE
:10F57000000000008100E800811F7800EA21F80007
:10F58000E0FF9F00EA21F900BA72020000000000CB
:10F59000CF007800800220000008E600F2FF37006C
:10F5A000CF02780000000600851F7800BD8AAE00FB
:10F5B00003003700D49780006124E10017003A006F
:10F5C000BD8AA80080CBB300FCF2B700FD72EF004B
:10F5D00050C0B30000F3B700E4C52000F4978800E2
:10F5E00004790200000000005EECB70000CBB3001D
:10F5F000FCF2B700FD72EF0050C0B30000F3B7009B
:10F6000084C52000F49788000479020000000000FF
:10F6100058ECB700A8790200000000005FCCBF00E2
:10F620006AECB70060CCBF006BECB70061CCBF00E8
:10F630006CECB70062CCBF006DECB70058CCBF00DB
:10F6400064ECB70059CCBF0065ECB7005ACCBF00E2
:10F6500066ECB7005BCCBF0067ECB7005CCCBF00CA
:10F6600068ECB700696CEF00CF027800000006007C
:10F670007A2DEF007A0DF8007C0DF900C1C720004B
:10F6800002002000FD0009008058EB008B0DA9004E
:10F6900000000600851F7800C50020000300090057
:10F6A000B51F7800800378008404780004F0A1007E
:10F6B0000400E00006003A0009F0A700020037004D
:10F6C0000500200010003700050020000E00370064
:10F6D000E64252000B0039000003200009F0A600AA
:10F6E00000022000801F78004F007800B06E0200FA
:10F6F000000000008502E900FAFF3B0055002000F1
:10F7000001003700840278006400200005E0A000BA
:10F7100009F0A70005F0A0000871220011000900FF
:10F720008883D800C87B02000000000081037800B5
:10F73000883E2000110009008883D800C87B0200A1
:10F740000000000081037800480620001100090035
:10F750008883D800C87B0200000000008103780085
:10F76000A8002000110009008883D800C87B02008F
:10F77000000000000003200000C04000801F78004F
:10F780004F007800B06E0200000000001A00370041
:10F79000060320000000E0000E003A0005E0A6008D
:10F7A0000D0037000402E9000524E10002003200E8
:10F7B0004200AF00000006000000E00005003A0033
:10F7C00005E0A6000400370005F0A60006022000B0
:10F7D0000100370005E0A10000404300811F7800D0
:10F7E000801F78004F007800B06E0200000000001B
:10F7F000CF0078000000060025012000030009006A
:10F80000CF127800CF02780000000600851F780034
:10F810001E33EF002073EF002173EF0014902800D7
:10F8200014998800240028002499880034002E00B0
:10F8300034998800440028004499880054502500D9
:10F8400054998800640020006499880074D02500D1
:10F8500074998800840020008499880094502500C1
:10F8600094998800A4002000A4998800B400240082
:10F87000B4998800C4002000C4998800D4002400F2
:10F88000D4998800E4002000E4998800F400240062
:10F89000F499880004012000049A880014012200D1
:10F8A000149A880024812100249A880034012200BF
:10F8B000349A880044812100449A880054A1200091
:10F8C000549A880064212000649A880074212000E2
:10F8D000749A880084A12200849A880094D122001E
:10F8E000949A8800A4412100A49A8800B4B123000E
:10F8F000B49A8800C4F12F00C49A8800D4812700EC
:10F90000D49A8800E4412A00E49A8800F46129002E
:10F91000F49A880004F22000049B8800140222005C
:10F92000149B880024222300249B88003462210039
:10F93000349B880044822000449B880054F22C00B1
:10F94000549B880064022100649B88007402260096
:10F95000749B880084F22B00849B880094222000F2
:10F96000949B8800A4022800A49B8800B402200075
:10F97000B49B8800C4022000C49B8800D4822E005F
:10F98000D49B8800E4022E00E49B880014502A00D7
:10F99000F49B880024002000049C880034002E0082
:10F9A000149C880044002800249C880054502500A2
:10F9B000349C880064002000449C880074D025009A
:10F9C000549C880084002000649C8800945025008A
:10F9D000749C8800A4002000849C8800B40024004B
:10F9E000949C8800C4002000A49C8800D4002400BB
:10F9F000B49C8800E4002000C49C8800F40024002B
:10FA0000D49C880004012000E49C8800140122009A
:10FA1000F49C880024812100049D88003401220088
:10FA2000149D880044812100249D880054A1200059
:10FA3000349D880064212000449D880074212000AA
:10FA4000549D880084A12200649D880094D12200E6
:10FA5000749D8800A4412100849D8800B4B12300D6
:10FA6000949D8800C4F12F00A49D8800D4812700B4
:10FA7000B49D8800E4412A00C49D8800F4612900F7
:10FA8000D49D880004F22000E49D88001402220026
:10FA9000F49D880024222300049E88003462210003
:10FAA000149E880044822000249E880054F22C007A
:10FAB000349E880064022100449E8800740226005F
:10FAC000549E880084F22B00649E880094222000BB
:10FAD000749E8800A4022800849E8800B40220003E
:10FAE000949E8800C4022000A49E8800D4822E0028
:10FAF000B49E8800E4022E00C49E88001490280062
:10FB0000D49E880024002800E49E880034002A0047
:10FB1000F49E880054502500049F88006400200053
:10FB2000149F880074D02500249F88008400200042
:10FB3000349F880094502500449F8800A400200032
:10FB4000549F8800B4002400649F8800C4002000F3
:10FB5000749F8800D4002400849F8800E400200063
:10FB6000949F8800F4002400A49F880004012000D2
:10FB7000B49F880014012200C49F880024812100C2
:10FB8000D49F880034012200E49F88004481210032
:10FB9000F49F880054A1200004A088006421200064
:10FBA00014A088007421200024A0880084A12200D1
:10FBB00034A0880094D1220044A08800A4412100F0
:10FBC00054A08800B4B1230064A08800C4F12F00C1
:10FBD00074A08800D481270084A08800E4412A0012
:10FBE00094A08800F4612900A4A0880004F22000F9
:10FBF000B4A0880014022200C4A08800242223009C
:10FC0000D4A0880034622100E4A08800448220004F
:10FC1000F4A0880054F22C0004A1880064022100A2
:10FC200014A188007402260024A1880084F22B000D
:10FC300034A188009422200044A18800A402280056
:10FC400054A18800B402200064A18800C4022000EE
:10FC500074A18800D4822E0084A18800E4022E00C2
:10FC600094A188003434EF0014402A00B4A1880025
:10FC700024002F00C4A1880034002A00D4A18800E9
:10FC800054502500E4A1880064002000F4A18800FD
:10FC900074D0250004A288008400200014A28800EB
:10FCA0009450250024A28800A400200034A28800DB
:10FCB000B400240044A28800C400200054A288009C
:10FCC000D400240064A28800E400200074A288000C
:10FCD000F400240084A288000401200094A288007B
:10FCE00014012200A4A2880024812100B4A288006B
:10FCF00034012200C4A2880044812100D4A28800DB
:10FD000054A12000E4A2880064212000F4A288000D
:10FD10007421200004A3880084A1220014A3880079
:10FD200094D1220024A38800A441210034A3880098
:10FD3000B4B1230044A38800C4F12F0054A3880069
:10FD4000D481270064A38800E4412A0074A38800BA
:10FD5000F461290084A3880004F2200094A38800A1
:10FD600014022200A4A3880024222300B4A3880044
:10FD700034622100C4A3880044822000D4A38800F8
:10FD800054F22C00E4A3880064022100F4A388004C
:10FD90007402260004A4880084F22B0014A48800B6
:10FDA0009422200024A48800A402280034A48800FF
:10FDB000B402200044A48800C402200054A4880097
:10FDC000D4822E0064A48800E4022E0074A488006B
:10FDD0009034EF001470260094A4880024002200C0
:10FDE000A4A4880034802A00B4A488004400280019
:10FDF000C4A4880054502500D4A4880064002000C6
:10FE0000E4A4880074D02500F4A4880084002000B5
:10FE100004A588009450250014A58800A4002000A3
:10FE200024A58800B400240034A58800C400200064
:10FE300044A58800D400240054A58800E4002000D4
:10FE400064A58800F400240074A588000401200043
:10FE500084A588001401220094A588002481210033
:10FE6000A4A5880044812100B4A5880054A12000E5
:10FE7000C4A5880064212000D4A588007421200036
:10FE8000E4A5880084A12200F4A5880094D1220072
:10FE900004A68800A441210014A68800B4B1230060
:10FEA00024A68800C4F12F0034A68800D48127003E
:10FEB00044A68800E4412A0054A68800F461290081
:10FEC00064A6880004F2200074A6880014022200B0
:10FED00084A688002422230094A6880034422100AE
:10FEE000A4A6880044822000B4A6880054F22C0006
:10FEF000C4A6880064022100D4A6880074022600EB
:10FF0000E4A6880084F22B00F4A688009422200046
:10FF100004A78800A402280014A78800B4022000C7
:10FF200024A78800C402200034A78800D4822E00B1
:10FF300044A78800E4022E0054A78800EC34EF00A8
:10FF400014B0270074A7880024002C0084A7880020
:10FF500034802A0094A7880044002800A4A78800C1
:10FF600054502500B4A7880064002000C4A788006E
:10FF700074D02500D4A7880084002000E4A788005E
:10FF800094502500F4A78800A400200004A888004D
:10FF9000B400240014A88800C400200024A888000D
:10FFA000D400240034A88800E400200044A888007D
:10FFB000F400240054A888000401200064A88800EC
:10FFC0001401220074A888002481210084A88800DC
:10FFD0004481210094A8880054A12000A4A888008E
:10FFE00064212000B4A8880074212000C4A88800DF
:10FFF00084A12200D4A8880094D12200E4A888001B
:020000040001F9
:10000000A4412100F4A88800B4B1230004A9880009
:10001000C4F12F0014A98800D481270024A98800E6
:10002000E4412A0034A98800F461290044A9880029
:1000300004F2200054A988001402220064A9880058
:100040002422230074A988003442210084A9880056
:100050004482200094A9880054F22C00A4A98800AE
:1000600064022100B4A9880074022600C4A9880093
:1000700084F22B00D4A9880094222000E4A98800EF
:10008000A4022800F4A98800B402200004AA880071
:10009000C402200014AA8800D4822E0024AA88005A
:1000A000E4022E0034AA88004835EF001420230013
:1000B00054AA88002400200064AA8800340022008A
:1000C00074AA880044002C0084AA880054002400EC
:1000D00094AA880064002000A4AA88007400240068
:1000E000B4AA880084002000C4AA880094002400D8
:1000F000D4AA8800A4002000E4AA8800B40020004C
:10010000F4AA8800C400280004AB8800D4002000B2
:1001100014AB8800E400280024AB8800F400200021
:1001200034AB88000401280044AB8800442120003F
:1001300054AB880054A1200064AB880064212000E7
:1001400074AB88007421200084AB880084012200F5
:1001500094AB880094812000A4AB8800A4412100C6
:10016000B4AB8800B4312700C4AB8800C4F12F00C1
:10017000D4AB8800D4812700E4AB8800E441280098
:10018000F4AB8800F461290004AC880004F220007C
:1001900014AC88001402220024AC8800242223001E
:1001A00034AC88003462210044AC8800444225000D
:1001B00054AC88005492200064AC88006402220091
:1001C00074AC880074022D0084AC880084F22B008B
:1001D00094AC880094222000A4AC8800A4022800DB
:1001E000B4AC8800B4022000C4AC8800C402200073
:1001F000D4AC8800D4822E00E4AC8800E4022E0047
:10020000F4AC8800A035EF001420240014AD880061
:100210002400200024AD88003400260034AD88007E
:1002200044002C0044AD88005400240054AD8800E4
:100230006400200064AD88007400240074AD880060
:100240008400200084AD88009400240094AD8800D0
:10025000A4002000A4AD8800B4002000B4AD880044
:10026000C4002800C4AD8800D4002000D4AD8800AC
:10027000E4002800E4AD8800F4002000F4AD88001C
:100280000401280004AE88004421200014AE880038
:1002900054A1200024AE88006421200034AE8800E0
:1002A0007421200044AE88008401220054AE8800EE
:1002B00094D1200064AE8800A441210074AE88006F
:1002C000B431270084AE8800C4F12F0094AE8800BA
:1002D000D4812700A4AE8800E4412800B4AE880091
:1002E000F4612900C4AE880004F22000D4AE880076
:1002F00014022200E4AE880024222300F4AE880019
:1003000034A2210004AF88004442250014AF8800C5
:100310005492200024AF88006402220034AF880089
:1003200074022D0044AF880084F22B0054AF880083
:100330009422200064AF8800A402280074AF8800D3
:10034000B402200084AF8800C402200094AF88006B
:10035000D4822E00A4AF8800E4022E00B4AF88003F
:10036000F835EF0014402500D4AF880024002000A9
:10037000E4AF880034802A00F4AF880044002C00E9
:1003800004B088005400240014B0880064002000E9
:1003900024B088007400240034B088008400200059
:1003A00044B088009400240054B08800A4002000C9
:1003B00064B08800B400200074B08800C400280035
:1003C00084B08800D400200094B08800E4002800A5
:1003D000A4B08800F4002000B4B088000401280014
:1003E000C4B0880014012200D4B088002481290000
:1003F000E4B0880034012200F4B0880044C1290030
:1004000004B1880054A1200014B1880064212000A8
:1004100024B188007421200034B1880084012200B6
:1004200044B188009441200054B18800A4412100C7
:1004300064B18800B431270074B18800C4F12F0082
:1004400084B18800D481270094B18800E4612B0036
:10045000A4B18800F4412900B4B1880004F220005E
:10046000C4B1880014022200D4B1880024222300E1
:10047000E4B1880034622100F4B1880044422500D0
:1004800004B288005492200014B288006402220052
:1004900024B2880074022D0034B2880084F22B004C
:1004A00044B288009422200054B28800A40228009C
:1004B00064B28800B402200074B28800C402200034
:1004C00084B28800D4822E0094B28800E4022E0008
:1004D000A4B288005636EF0014902600C4B28800FB
:1004E00024002800D4B2880034802A00E4B28800B6
:1004F00054002400F4B288006400200004B3880093
:100500007400240014B388008400200024B3880001
:100510009400240034B38800A400200044B3880071
:10052000B400200054B38800C400280064B38800DD
:10053000D400200074B38800E400280084B388004D
:10054000F400200094B3880004012800A4B38800BC
:1005500014012200B4B3880024812900C4B38800A8
:1005600044C12900D4B3880054A12000E4B388001A
:1005700064212000F4B388007421200004B48800B2
:100580008401220014B488009441200024B488001F
:10059000A441210034B48800B431270044B4880059
:1005A000C4F12F0054B48800D481270064B48800BB
:1005B000E4612B0074B48800F441290084B48800FD
:1005C00004F2200094B4880014022200A4B488002D
:1005D00024222300B4B4880034622100C4B488000B
:1005E00044422500D4B4880054922000E4B488002A
:1005F00064022200F4B4880074022D0004B588005F
:1006000084F22B0014B588009422200024B58800C1
:10061000A402280034B58800B402200044B5880044
:10062000C402200054B58800D4822E0064B588002E
:10063000E4022E0074B588001490260084B588006A
:100640002400280094B5880034002B00A4B588004D
:1006500044002C00B4B5880054002400C4B58800C0
:1006600064002000D4B5880074002400E4B588003C
:1006700084002000F4B588009400240004B68800AB
:10068000A400200014B68800B400200024B688001E
:10069000C400280034B68800D400200044B6880086
:1006A000E400280054B68800F400200064B68800F6
:1006B0000401280074B688001401220084B6880062
:1006C0002481290094B6880034012200A4B6880051
:1006D00044C12900B4B6880054A12000C4B68800E3
:1006E00064212000D4B6880074212000E4B688007C
:1006F00084012200F4B688009441200004B78800E9
:10070000A441210014B78800B431270024B7880021
:10071000C4F12F0034B78800D481270044B7880083
:10072000E4612B0054B78800F441290064B78800C5
:1007300004F2200074B788001402220084B78800F5
:100740002422230094B7880034622100A4B78800D3
:1007500044422500B4B7880054922000C4B78800F2
:1007600064022200D4B7880074022D00E4B7880028
:1007700084F22B00F4B788009422200004B888008B
:10078000A402280014B88800B402200024B888000D
:10079000C402200034B88800D4822E0044B88800F7
:1007A000E4022E0054B888000C37EF0014F0280043
:1007B00074B8880024D0200084B8880034002B004E
:1007C00094B8880044002C00A4B888005400240089
:1007D000B4B8880064002000C4B888007400240005
:1007E000D4B8880084002000E4B888009400240075
:1007F000F4B88800A400200004B98800B4002000E8
:1008000014B98800C400280024B98800D40020004E
:1008100034B98800E400280044B98800F4002000BE
:1008200054B988000401280064B98800140122002A
:1008300074B988002481290084B988003401220019
:1008400094B9880044C12900A4B9880054A12000AB
:10085000B4B9880064212000C4B988007421200044
:10086000D4B9880084012200E4B9880094412000B2
:10087000F4B98800A441210004BA8800B4312700EB
:1008800014BA8800C4F12F0024BA8800D48127004C
:1008900034BA8800E4612B0044BA8800F44129008E
:1008A00054BA880004F2200064BA880014022200BE
:1008B00074BA88002422230084BA8800346221009C
:1008C00094BA880044422500A4BA880054922000BB
:1008D000B4BA880064022200C4BA880074022D00F1
:1008E000D4BA880084F22B00E4BA88009422200055
:1008F000F4BA8800A402280004BB8800B4022000D7
:1009000014BB8800C402200024BB8800D4822E00BF
:1009100034BB8800E4022E0044BB8800140027008A
:1009200054BB88002480200064BB880034002B0066
:1009300074BB880044002C0084BB88005400240051
:1009400094BB880064002000A4BB880074002400CD
:10095000B4BB880084002000C4BB8800940024003D
:10096000D4BB8800A4002000E4BB8800B4002000B1
:10097000F4BB8800C400280004BC8800D400200018
:1009800014BC8800E400280024BC8800F400200087
:1009900034BC88000401280044BC880014012200F3
:1009A00054BC88002481290064BC880034012200E2
:1009B00074BC880044C1290084BC880054A1200074
:1009C00094BC880064212000A4BC8800742120000D
:1009D000B4BC880084012200C4BC8800944120007B
:1009E000D4BC8800A4412100E4BC8800B4312700B5
:1009F000F4BC8800C4F12F0004BD8800D481270016
:100A000014BD8800E4612B0024BD8800F441290056
:100A100034BD880004F2200044BD88001402220086
:100A200054BD88002422230064BD88003462210064
:100A300074BD88004442250084BD88005492200083
:100A400094BD880064022200A4BD880074022D00B9
:100A5000B4BD880084F22B00C4BD8800942220001D
:100A6000D4BD8800A4022800E4BD8800B4022000A0
:100A7000F4BD8800C402200004BE8800D4822E0089
:100A800014BE8800E4022E0024BE8800C637EF00A2
:100A90001470280044BE88002400200054BE880042
:100AA00034002F0064BE88004480270074BE880094
:100AB0005400240084BE88006400200094BE880096
:100AC00074002400A4BE880084002000B4BE880006
:100AD00094002400C4BE8800A4002000D4BE880076
:100AE000B4002000E4BE8800C4002800F4BE8800E2
:100AF000D400200004BF8800E400280014BF880050
:100B0000F400200024BF88000401280034BF8800BE
:100B10004421200044BF880054A1200054BF880015
:100B20006421200064BF88007421200074BF880005
:100B30008401220084BF88009481200094BF880033
:100B4000A4412100A4BF8800B4312700B4BF8800AD
:100B5000C4F12F00C4BF8800D4812700D4BF88000F
:100B6000E4612B00E4BF8800F4412900F4BF880051
:100B700004F2200004C088001402220014C088007F
:100B80002422230024C0880034A2210034C088001D
:100B90004442250044C088005492200054C088007C
:100BA0006402220064C0880074022D0074C08800B2
:100BB00084F22B0084C088009422200094C0880016
:100BC000A4022800A4C08800B4022000B4C0880099
:100BD000C4022000C4C08800D4822E00D4C0880083
:100BE000E4022E00E4C088001E38EF0004602000FC
:100BF00004C188003480200014C18800F408250056
:100C000024C188007492220034C18800142321007A
:100C100044C188002413280054C1880034432800AC
:100C200064C188004403200074C18800540320007C
:100C300084C1880064D3270094C1880074132A00FB
:100C4000A4C18800541E2400B4C18800644E28004A
:100C5000C4C18800746E2000D4C18800449F210064
:100C6000E4C18800F4002200F4C188000460200080
:100C700004C288003480200014C28800F4082500D3
:100C800024C288007492220034C2880014A3210078
:100C900044C288002413240054C28800344328002E
:100CA00064C288004403200074C2880054232000DA
:100CB00084C288006403200094C28800741320005A
:100CC000A4C28800545E2200B4C28800644E200092
:100CD000C4C28800743E2600D4C28800449F21000C
:100CE000E4C28800F4002200F4C28800042020003E
:100CF00004C388003480200014C38800F408250051
:100D000024C388007492220034C388001423210075
:100D100044C388002413280054C3880034432800A7
:100D200064C388004403200074C388005403200077
:100D300084C3880064D3270094C3880074132A00F6
:100D4000A4C38800541E2400B4C38800644E280045
:100D5000C4C38800746E2000D4C38800449F21005F
:100D6000E4C38800F4002200F4C3880004202000BB
:100D700004C488003480200014C48800F4082500CE
:100D800024C488007492220034C4880014A3210073
:100D900044C488002413240054C488003443280029
:100DA00064C488004403200074C4880054232000D5
:100DB00084C488006403200094C488007413200055
:100DC000A4C48800545E2200B4C48800644E20008D
:100DD000C4C48800743E2600D4C48800449F210007
:100DE000E4C48800F4002200F4C48800E498800081
:100DF000670242000400780021F3B70021D3BF004E
:100E0000EA21F800E0FF9F00EA21F9009C6F020050
:100E100000000000200320002A65020000000000FE
:100E2000BD0AAE002200370001002000010078005A
:100E300026020200000000008100E800811F780007
:100E4000EA21F800E0FF9F00EA21F900BA720200EF
:100E500000000000CF007800700020000008E600CD
:100E6000F2FF3700E0988000040020007874020050
:100E700000000000500F8100A0C3B300500F890094
:100E8000BA72020000000000500F810000C2B300DF
:100E9000500F8900BA72020000000000500F81005C
:100EA00000C2B300500F8900BA72020000000000B7
:100EB000E49880000960EF00530C2000048041009A
:100EC000A4A1200084024000154078000160EF00DA
:100ED0000080B200250032001080B20067003200AE
:100EE0003080B200A90032001080B200EB00320066
:100EF0007080B2002D0132001080B2006F0132000C
:100F00003080B200B10132001080B200F301320033
:100F1000F080B200350232001080B2007702320059
:100F20003080B200B90232001080B200FB02320001
:100F30007080B2003D0332001080B2007F033200A7
:100F40002080B200C1033200F081B20002043200FE
:100F50001080B200430432003080B20084043200BA
:100F6000C081B200C5043200D5043700500F8100A3
:100F700020C4B300500F8900500F81000080FD0095
:100F8000F0C0B3000080FD00500F8900600F8100A9
:100F900040C2B300600F89006A68020000000000D0
:100FA0001E33EF00F4988000E30220000418E100F3
:100FB0001F003600F5988000C12ADD002432210090
:100FC0000480420004998000004290000499880047
:100FD000F5988000C12ADD00E1824200050078001A
:100FE00024322100040040001040780021F3B700B3
:100FF000500F8100A0C9B300500F890020D3BF005B
:10100000EA21F800F0FF9F00EA21F90021D3BF0098
:10101000EC21F800E0FF9F00EC21F9006A68020073
:10102000000000001E33EC00D28704000000000026
:10103000BD0AAE000F00370001002000010078005B
:1010400042020200000000008100E800811F7800D9
:10105000EA21F800E0FF9F00EA21F900BA720200DD
:1010600000000000CF007800200220000008E60009
:10107000F2FF3700BA91040000000000500F810019
:1010800020C4B300500F8900500F81000080FD0084
:10109000F0C0B3000080FD00500F8900600F810098
:1010A00040C2B300600F89006A68020000000000BF
:1010B0001E33EF00F4988000E30220000418E100E2
:1010C0001F003600F5988000C12ADD00E4372100BA
:1010D0000480420004998000004290000499880036
:1010E000F5988000C12ADD00E18242000500780009
:1010F000E4372100040040001040780021F3B700DD
:10110000500F8100A0C9B300500F890020D3BF0049
:10111000EA21F800F0FF9F00EA21F90021D3BF0087
:10112000EC21F800E0FF9F00EC21F9006A68020062
:10113000000000001E33EC005A880400000000008C
:10114000BD0AAE000F00370001002000010078004A
:1011500074020200000000008100E800811F780096
:10116000EA21F800E0FF9F00EA21F900BA720200CC
:1011700000000000CF007800F00120000008E60029
:10118000F2FF3700BA91040000000000500F810008
:1011900020C4B300500F8900500F81000080FD0073
:1011A000F0C0B3000080FD00500F8900600F810087
:1011B00040C2B300600F89006A68020000000000AE
:1011C0001E33EF00F4988000D30220000418E100E1
:1011D0001F003600F5988000C12ADD00A43D2100E3
:1011E0000480420004998000004290000499880025
:1011F000F5988000C12ADD00E182420005007800F8
:10120000A43D2100040040001040780021F3B70005
:10121000500F8100A0C9B300500F890020D3BF0038
:10122000EA21F800F0FF9F00EA21F90021D3BF0076
:10123000EC21F800E0FF9F00EC21F9006A68020051
:10124000000000001E33EC00E288040000000000F3
:10125000BD0AAE000F003700010020000100780039
:10126000A4020200000000008100E800811F780055
:10127000EA21F800E0FF9F00EA21F900BA720200BB
:1012800000000000CF007800200220000008E600E7
:10129000F2FF3700BA91040000000000500F8100F7
:1012A00020C4B300500F8900500F81000080FD0062
:1012B000F0C0B3000080FD00500F8900600F810076
:1012C00040C2B300600F89006A680200000000009D
:1012D0001E33EF00F4988000D30220000418E100D0
:1012E0001F003600F5988000C12ADD00644321000C
:1012F0000480420004998000004290000499880014
:10130000F5988000C12ADD00E182420005007800E6
:1013100064432100040040001040780021F3B7002E
:10132000500F8100A0C9B300500F890020D3BF0027
:10133000EA21F800F0FF9F00EA21F90021D3BF0065
:10134000EC21F800E0FF9F00EC21F9006A68020040
:10135000000000001E33EC006A8904000000000059
:10136000BD0AAE000F003700010020000100780028
:10137000D6020200000000008100E800811F780012
:10138000EA21F800E0FF9F00EA21F900BA720200AA
:1013900000000000CF007800F00120000008E60007
:1013A000F2FF3700BA91040000000000500F8100E6
:1013B00020C4B300500F8900500F81000080FD0051
:1013C000F0C0B3000080FD00500F8900600F810065
:1013D00040C2B300600F89006A680200000000008C
:1013E0001E33EF00F4988000D30220000418E100BF
:1013F0001F003600F5988000C12ADD002449210035
:101400000480420004998000004290000499880002
:10141000F5988000C12ADD00E182420005007800D5
:1014200024492100040040001040780021F3B70057
:10143000500F8100A0C9B300500F890020D3BF0016
:10144000EA21F800F0FF9F00EA21F90021D3BF0054
:10145000EC21F800E0FF9F00EC21F9006A6802002F
:10146000000000001E33EC00F289040000000000C0
:10147000BD0AAE000F003700010020000100780017
:1014800006030200000000008100E800811F7800D0
:10149000EA21F800E0FF9F00EA21F900BA72020099
:1014A00000000000CF007800000220000008E600E5
:1014B000F2FF3700BA91040000000000500F8100D5
:1014C00020C4B300500F8900500F81000080FD0040
:1014D000F0C0B3000080FD00500F8900600F810054
:1014E00040C2B300600F89006A680200000000007B
:1014F0001E33EF00F4988000D30220000418E100AE
:101500001F003600F5988000C12ADD00E44E21005E
:1015100004804200049980000042900004998800F1
:10152000F5988000C12ADD00E182420005007800C4
:10153000E44E2100040040001040780021F3B70081
:10154000500F8100A0C9B300500F890020D3BF0005
:10155000EA21F800F0FF9F00EA21F90021D3BF0043
:10156000EC21F800E0FF9F00EC21F9006A6802001E
:10157000000000001E33EC007A8A04000000000026
:10158000BD0AAE000F003700010020000100780006
:1015900036030200000000008100E800811F78008F
:1015A000EA21F800E0FF9F00EA21F900BA72020088
:1015B00000000000CF007800D00120000008E60005
:1015C000F2FF3700BA91040000000000500F8100C4
:1015D00020C4B300500F8900500F81000080FD002F
:1015E000F0C0B3000080FD00500F8900600F810043
:1015F00040C2B300600F89006A680200000000006A
:101600001E33EF00F4988000B30220000418E100BC
:101610001F003600F5988000C12ADD00A454210087
:1016200004804200049980000042900004998800E0
:10163000F5988000C12ADD00E182420005007800B3
:10164000A4542100040040001040780021F3B700AA
:10165000500F8100A0C9B300500F890020D3BF00F4
:10166000EA21F800F0FF9F00EA21F90021D3BF0032
:10167000EC21F800E0FF9F00EC21F9006A6802000D
:10168000000000001E33EC00028B0400000000008C
:10169000BD0AAE000F0037000100200001007800F5
:1016A00064030200000000008100E800811F780050
:1016B000EA21F800E0FF9F00EA21F900BA72020077
:1016C00000000000CF007800200220000008E600A3
:1016D000F2FF3700BA91040000000000500F8100B3
:1016E00020C4B300500F8900500F81000080FD001E
:1016F000F0C0B3000080FD00500F8900600F810032
:1017000040C2B300600F89006A6802000000000058
:101710001E33EF00F4988000B30220000418E100AB
:101720001F003600F5988000C12ADD00245A2100F0
:1017300004804200049980000042900004998800CF
:10174000F5988000C12ADD00E182420005007800A2
:10175000245A2100040040001040780021F3B70013
:10176000500F8100A0C9B300500F890020D3BF00E3
:10177000EA21F800F0FF9F00EA21F90021D3BF0021
:10178000EC21F800E0FF9F00EC21F9006A680200FC
:10179000000000001E33EC008A8B040000000000F3
:1017A000BD0AAE000F0037000100200001007800E4
:1017B00096030200000000008100E800811F78000D
:1017C000EA21F800E0FF9F00EA21F900BA72020066
:1017D00000000000CF007800200220000008E60092
:1017E000F2FF3700BA91040000000000500F8100A2
:1017F00020C4B300500F8900500F81000080FD000D
:10180000F0C0B3000080FD00500F8900600F810020
:1018100040C2B300600F89006A6802000000000047
:101820001E33EF00F4988000E30220000418E1006A
:101830001F003600F5988000C12ADD00A45F21005A
:1018400004804200049980000042900004998800BE
:10185000F5988000C12ADD00E18242000500780091
:10186000A45F2100040040001040780021F3B7007D
:10187000500F8100A0C9B300500F890020D3BF00D2
:10188000EA21F800F0FF9F00EA21F90021D3BF0010
:10189000EC21F800E0FF9F00EC21F9006A680200EB
:1018A000000000001E33EC00128C04000000000059
:1018B000BD0AAE000F0037000100200001007800D3
:1018C000C8030200000000008100E800811F7800CA
:1018D000EA21F800E0FF9F00EA21F900BA72020055
:1018E00000000000CF007800300220000008E60071
:1018F000F2FF3700BA91040000000000500F810091
:1019000020C4B300500F8900500F81000080FD00FB
:10191000F0C0B3000080FD00500F8900600F81000F
:1019200040C2B300600F89006A6802000000000036
:101930001E33EF00F4988000E30220000418E10059
:101940001F003600F5988000C12ADD008465210063
:1019500004804200049980000042900004998800AD
:10196000F5988000C12ADD00E18242000500780080
:1019700084652100040040001040780021F3B70086
:10198000500F8100A0C9B300500F890020D3BF00C1
:10199000EA21F800F0FF9F00EA21F90021D3BF00FF
:1019A000EC21F800E0FF9F00EC21F9006A680200DA
:1019B000000000001E33EC009A8C040000000000C0
:1019C000BD0AAE000F0037000100200001007800C2
:1019D000040C0200000000008100E800811F780074
:1019E000EA21F800E0FF9F00EA21F900BA72020044
:1019F00000000000CF007800400220000008E60050
:101A0000F2FF3700BA91040000000000500F81007F
:101A100020C4B300500F8900500F81000080FD00EA
:101A2000F0C0B3000080FD00500F8900600F8100FE
:101A300040C2B300600F89006A6802000000000025
:101A40001E33EF00F4988000C30220000418E10068
:101A50001F003600F5988000C12ADD00046B2100CC
:101A6000048042000499800000429000049988009C
:101A7000F5988000C12ADD00E1824200050078006F
:101A8000046B2100040040001040780021F3B700EF
:101A9000500F8100A0C9B300500F890020D3BF00B0
:101AA000EA21F800F0FF9F00EA21F90021D3BF00EE
:101AB000EC21F800E0FF9F00EC21F9006A680200C9
:101AC000000000001E33EC00228D04000000000026
:101AD000BD0AAE000F0037000100200001007800B1
:101AE000380C0200000000008100E800811F78002F
:101AF000EA21F800E0FF9F00EA21F900BA72020033
:101B000000000000CF007800300220000008E6004E
:101B1000F2FF3700BA91040000000000500F81006E
:101B200020C4B300500F8900500F81000080FD00D9
:101B3000F0C0B3000080FD00500F8900600F8100ED
:101B400040C2B300600F89006A6802000000000014
:101B50001E33EF00F4988000E30220000418E10037
:101B60001F003600F5988000C12ADD00E4702100D6
:101B7000048042000499800000429000049988008B
:101B8000F5988000C12ADD00E1824200050078005E
:101B9000E4702100040040001040780021F3B700F9
:101BA000500F8100A0C9B300500F890020D3BF009F
:101BB000EA21F800F0FF9F00EA21F90021D3BF00DD
:101BC000EC21F800E0FF9F00EC21F9006A680200B8
:101BD000000000001E33EC00AA8D0400000000008D
:101BE000BD0AAE000F0037000100200001007800A0
:101BF0006C0C0200000000008100E800811F7800EA
:101C0000EA21F800E0FF9F00EA21F900BA72020021
:101C100000000000CF007800300220000008E6003D
:101C2000F2FF3700BA91040000000000500F81005D
:101C300020C4B300500F8900500F81000080FD00C8
:101C4000F0C0B3000080FD00500F8900600F8100DC
:101C500040C2B300600F89006A6802000000000003
:101C60001E33EF00F4988000E30220000418E10026
:101C70001F003600F5988000C12ADD00A4762100FF
:101C8000048042000499800000429000049988007A
:101C9000F5988000C12ADD00E1824200050078004D
:101CA000A4762100040040001040780021F3B70022
:101CB000500F8100A0C9B300500F890020D3BF008E
:101CC000EA21F800F0FF9F00EA21F90021D3BF00CC
:101CD000EC21F800E0FF9F00EC21F9006A680200A7
:101CE000000000001E33EC00328E040000000000F3
:101CF000BD0AAE000F00370001002000010078008F
:101D0000A00C0200000000008100E800811F7800A4
:101D1000EA21F800E0FF9F00EA21F900BA72020010
:101D200000000000CF007800400220000008E6001C
:101D3000F2FF3700BA91040000000000500F81004C
:101D400020C4B300500F8900500F81000080FD00B7
:101D5000F0C0B3000080FD00500F8900600F8100CB
:101D600040C2B300600F89006A68020000000000F2
:101D70001E33EF00F4988000B30220000418E10045
:101D80001F003600F5988000C12ADD00847C210008
:101D90000480420004998000004290000499880069
:101DA000F5988000C12ADD00E1824200050078003C
:101DB000847C2100040040001040780021F3B7002B
:101DC000500F8100A0C9B300500F890020D3BF007D
:101DD000EA21F800F0FF9F00EA21F90021D3BF00BB
:101DE000EC21F800E0FF9F00EC21F9006A68020096
:101DF000000000001E33EC00BA8E0400000000005A
:101E0000BD0AAE000F00370001002000010078007D
:101E1000D40C0200000000008100E800811F78005F
:101E2000EA21F800E0FF9F00EA21F900BA720200FF
:101E300000000000CF007800400220000008E6000B
:101E4000F2FF3700BA91040000000000500F81003B
:101E5000A0C9B300500F8900500F81000080FD0021
:101E6000E0C1B3000080FD00500F8900600F8100C9
:101E7000A0C0B300600F89006A6802000000000083
:101E80001E33EF00F49880007020E1001F00310045
:101E9000F5988000C12ADD00048221000480420000
:101EA000049980000042900004998800F598800011
:101EB000C12ADD00E1824200050078000482210091
:101EC000040040001040780021F3B700500F81005B
:101ED00020C4B300500F890020D3BF00EA21F800CE
:101EE000F0FF9F00EA21F90021D3BF00EC21F800A8
:101EF000E0FF9F00EC21F9006A680200000000008A
:101F00001E33EC00428F040000000000BD0AAE004A
:101F10000F0037000100200001007800080D0200CA
:101F2000000000008100E800811F7800EA21F8002D
:101F3000E0FF9F00EA21F900BA72020000000000F1
:101F4000CF007800700220000008E600F2FF3700A2
:101F5000BA91040000000000500F8100A0C9B30036
:101F6000500F8900500F81000080FD00E0C1B300D8
:101F70000080FD00500F8900600F8100A0C0B300F9
:101F8000600F89006A680200000000001E33EF0045
:101F9000F49880007020E1001F003100F598800067
:101FA000C12ADD00048421000480420004998000DD
:101FB0000042900004998800F5988000C12ADD0055
:101FC000E182420005007800048421000400400002
:101FD0001040780021F3B700500F810020C4B300F7
:101FE000500F890020D3BF00EA21F800F0FF9F00C6
:101FF000EA21F90021D3BF00EC21F800E0FF9F00A7
:10200000EC21F9006A680200000000001E33EC00B9
:10201000C88F040000000000BD0AAE000F003700AA
:102020000100200001007800400D020000000000C7
:102030008100E800811F7800EA21F800E0FF9F009E
:10204000EA21F900BA72020000000000CF00780017
:10205000600220000008E600F2FF3700BA91040099
:1020600000000000500F8100A0C9B300500F89008C
:10207000500F81000080FD00E0C1B3000080FD0032
:10208000500F8900600F8100A0C0B300600F89006D
:102090006A680200000000001E33EF00F498800020
:1020A0007020E1001F003100F5988000C12ADD009A
:1020B00004862100048042000499800000429000C0
:1020C00004998800F5988000C12ADD00E182420071
:1020D00005007800048621000400400010407800CC
:1020E00021F3B700500F810020C4B300500F8900C6
:1020F00020D3BF00EA21F800F0FF9F00EA21F90099
:1021000021D3BF00EC21F800E0FF9F00EC21F90093
:102110006A680200000000001E33EC004E900400CC
:1021200000000000BD0AAE000F00370001002000D3
:1021300001007800760D0200000000008100E80038
:10214000811F7800EA21F800E0FF9F00EA21F900F2
:10215000BA72020000000000CF007800A002200048
:102160000008E600F2FF3700BA910400000000000A
:10217000500F8100A0C9B300500F8900500F81009B
:102180000080FD00E0C1B3000080FD00500F890019
:10219000600F8100A0C0B300600F89006A68020070
:1021A000000000001E33EF00F49880007020E10072
:1021B0001F003100F5988000C12ADD00048821004D
:1021C0000480420004998000004290000499880035
:1021D000F5988000C12ADD00E18242000500780008
:1021E00004882100040040001040780021F3B7006B
:1021F000500F810020C4B300500F890020D3BF00CE
:10220000EA21F800F0FF9F00EA21F90021D3BF0086
:10221000EC21F800E0FF9F00EC21F9006A68020061
:10222000000000001E33EC00D49004000000000009
:10223000BD0AAE000F003700010020000100780049
:10224000B20D0200000000008100E800811F78004C
:10225000EA21F800E0FF9F00EA21F900BA720200CB
:1022600000000000CF007800800220000008E60097
:10227000F2FF3700BA91040000000000BD0AAE0072
:102280000F0037000100200001007800EC0D020073
:10229000000000008100E800811F7800EA21F800BA
:1022A000E0FF9F00EA21F900BA720200000000007E
:1022B000CF007800200220000008E600F2FF37007F
:1022C000500F8100A0C9B300500F8900500F81004A
:1022D0000080FD00E0C1B3000080FD00500F8900C8
:1022E000600F8100A0C0B300600F89006A6802001F
:1022F00000000000500F810020C4B300500F89007F
:10230000500F81000080FD00F0C0B3000080FD0090
:10231000500F8900600F810040C2B300600F890038
:102320006A68020000000000BD0AAE000F0037001E
:1023300001002000010078001E0E020000000000D5
:102340008100E800811F7800EA21F800E0FF9F008B
:10235000EA21F900BA72020000000000CF00780004
:10236000800020000008E600F2FF3700BA91040068
:1023700000000000CF02780000000600851F7800F2
:102380001A33EF00CC6F02000000000014002000A0
:10239000D4988800D49880006720E10007003100BD
:1023A0001A13F8001C13F900067C0200000000005C
:1023B0001A33EC00CA91040000000000BD0AAE0010
:1023C0000F00370001002000010078000002020029
:1023D000000000008100E800811F7800EA21F80079
:1023E000E0FF9F00EA21F900BA720200000000003D
:1023F000CF007800600120000008E600F2FF3700FF
:10240000CF02780000000600851F78001A33EF0025
:102410001C33EF001E73EF001F73EF002073EF00FB
:102420003410290014998800440020002499880061
:1024300054002000349988006400200044998800EA
:10244000740020005499880084002000649988005A
:102450009400200074998800A400200084998800CA
:10246000B400200094998800C4002000A49988003A
:10247000D4002000B4998800E4002000C4998800AA
:10248000F4002000D499880004012000E499880019
:1024900014012000F499880024012000049A880087
:1024A00034012000149A880044012000249A8800F6
:1024B00054012000349A880064012000449A880066
:1024C00074012000549A880084012000649A8800D6
:1024D00094312000749A8800A4012000849A880016
:1024E000B4012000949A8800C4012700A49A8800AF
:1024F000D4F12F00B49A8800E4912400C49A880093
:10250000F4612B00D49A880004F22F00E49A88002A
:1025100014F22F00F49A880024F22F00049B880004
:1025200034322100149B880044522100249B8800EF
:1025300054C22200349B880064822500449B88009A
:1025400074C22200549B880084422800649B880047
:1025500094022000749B8800A4022C00849B8800B5
:10256000B4022000949B8800C4022000A49B880031
:10257000D4022000B49B8800E4022000C49B8800A1
:10258000F4822500D49B880004032000E49B88008B
:1025900014032000F49B880024832500049C8800F9
:1025A00034032000149C880044832000249C88006D
:1025B00054832900349C880064032800449C8800CC
:1025C00074132000549C880084032800649C8800B5
:1025D00094432400749C8800A4532600849C8800A3
:1025E000B4532600949C8800C4032800A49C88004F
:1025F000D4032000B49C8800E4032000C49C88001D
:10260000F4032000D49C880004042000E49C88008B
:1026100014042400F49C880024042400049D8800F1
:1026200034042400149D880044342500249D88002F
:1026300054F42300349D880064F42300449D8800F2
:1026400074042400549D880084042400649D880040
:1026500094042400749D8800A4842000849D880034
:10266000B4042000949D8800C4042000A49D880028
:10267000D4042000B49D8800E4042000C49D880098
:10268000F4042000D49D880004052000E49D880007
:1026900014052000F49D880024052000049E880075
:1026A00034052000149E880044052000249E8800E4
:1026B00054052000349E880064052000449E880054
:1026C00074052000549E880084052000649E8800C4
:1026D00094052000749E8800A4052000849E880034
:1026E000B4052000949E8800C4052000A49E8800A4
:1026F000D4052000B49E8800E4052000C49E880014
:10270000F4052000D49E880004062000E49E880082
:1027100014062000F49E880024062000049F8800F0
:1027200034062000149F880044062000249F88005F
:1027300054062000349F880064062000449F8800CF
:1027400074062000549F880084062000649F88003F
:1027500094062000749F8800A4062000849F8800AF
:10276000B4062000949F8800C4062000A49F88001F
:10277000D4062000B49F8800E4062000C49F88008F
:10278000F4062000D49F880004872100E49F88007D
:1027900014872400F49F88002497290004A088004F
:1027A0003477210014A088004447200024A088002A
:1027B0005457260034A088006407200044A08800F5
:1027C0007427200054A088008427230064A0880078
:1027D0009407200074A08800A497200084A088009B
:1027E000B407200094A08800C4172000A4A088008B
:1027F00024B82100B4A0880034082000C4A08800B8
:1028000044082000D4A0880054082000E4A08800D8
:1028100034102900F4A088004400200004A188009E
:102820005400200014A188006400200024A1880026
:102830007400200034A188008400200044A1880096
:102840009400200054A18800A400200064A1880006
:10285000B400200074A18800C400200084A1880076
:10286000D400200094A18800E4002000A4A18800E6
:10287000F4002000B4A1880004012000C4A1880055
:1028800014012000D4A1880024012000E4A18800C4
:1028900034012000F4A188004401200004A2880033
:1028A0005401200014A288006401200024A28800A2
:1028B0007401200034A288008401200044A2880012
:1028C0009431200054A28800A401200064A2880052
:1028D000B401200074A28800C401270084A28800EB
:1028E000D4F12F0094A28800E4912400A4A28800CF
:1028F000F4612B00B4A2880004F22F00C4A2880067
:1029000014F22F00D4A2880024F22F00E4A2880041
:1029100034322100F4A288004452210004A388002C
:1029200054C2220014A388006482250024A38800D6
:1029300074C2220034A388008442280044A3880083
:102940009402200054A38800A4022C0064A38800F1
:10295000B402200074A38800C402200084A388006D
:10296000D402200094A38800E4022000A4A38800DD
:10297000F4822500B4A3880004032000C4A38800C7
:1029800014032000D4A3880024832500E4A3880036
:1029900034032000F4A3880044A3200004A488008A
:1029A0005403250014A488006403280024A488008C
:1029B0007413200034A488008403280044A48800F1
:1029C0009443240054A48800A453260064A48800DF
:1029D000B453260074A48800C403280084A488008B
:1029E000D403200094A48800E4032000A4A4880059
:1029F000F4032000B4A4880004042000C4A48800C8
:102A000014042400D4A4880024042400E4A488002E
:102A100034042400F4A488004434250004A588006C
:102A200054F4230014A5880064F4230024A588002E
:102A30007404240034A588008404240044A588007C
:102A40009404240054A58800A484200064A5880070
:102A5000B404200074A58800C404200084A5880064
:102A6000D404200094A58800E4042000A4A58800D4
:102A7000F4042000B4A5880004052000C4A5880043
:102A800014052000D4A5880024052000E4A58800B2
:102A900034052000F4A588004405200004A6880021
:102AA0005405200014A688006405200024A6880090
:102AB0007405200034A688008405200044A6880000
:102AC0009405200054A68800A405200064A6880070
:102AD000B405200074A68800C405200084A68800E0
:102AE000D405200094A68800E4052000A4A6880050
:102AF000F4052000B4A6880004062000C4A68800BF
:102B000014062000D4A6880024062000E4A688002D
:102B100034062000F4A688004406200004A788009C
:102B20005406200014A788006406200024A788000B
:102B30007406200034A788008406200044A788007B
:102B40009406200054A78800A406200064A78800EB
:102B5000B406200074A78800C406200084A788005B
:102B6000D406200094A78800E4062000A4A78800CB
:102B7000F4062000B4A7880004972E00C4A788009C
:102B800014A72000D4A7880024172500E4A78800F4
:102B900034772100F4A788004447200004A8880067
:102BA0005457260014A888006407200024A8880031
:102BB0007427200034A888008427230044A88800B4
:102BC0009407200054A88800A4E7200064A8880087
:102BD000B407200074A88800C417200084A88800C7
:102BE00024B8210094A8880034082000A4A88800F4
:102BF00044082000B4A8880054082000C4A8880015
:102C000034102100D4A8880094312000E4A8880062
:102C1000C4012600F4A88800D4F12F0004A988007C
:102C2000E491240014A98800F4612B0024A98800F1
:102C300004F22F0034A9880014F22F0044A9880060
:102C400024F22F0054A988003432210064A988009E
:102C50004452210074A9880054C2220084A988002B
:102C60006482250094A9880074C22200A4A9880067
:102C700084422800B4A9880094022000C4A98800D6
:102C8000A4022C00D4A98800B4022000E4A9880082
:102C9000C4022000F4A98800D402200004AA8800FD
:102CA000E402200014AA8800F482250024AA8800E7
:102CB0000403200034AA88001403200044AA8800DA
:102CC0002483250054AA88003403200064AA8800C5
:102CD0004483200074AA88005483290084AA8800B1
:102CE0006403200094AA880074132000A4AA88001A
:102CF00084132800B4AA880094232400C4AA88005E
:102D0000A4532600D4AA8800B4332300E4AA880080
:102D1000F4042000F4AA880004E7220004AB880031
:102D20001487200014AB88002497290024AB880066
:102D30003467200034AB88004407200044AB88008F
:102D40005407200054AB88006467200064AB8800FF
:102D50007427200074AB88008437230084AB88007C
:102D60009407200094AB8800A4672100A4AB8800DE
:102D7000B4072000B4AB8800C4172000C4AB88009F
:102D800024F82900D4AB88007C35EF0034102100F2
:102D9000F4AB88009431200004AC8800C401260004
:102DA00014AC8800D4F12F0024AC8800E4912400F6
:102DB00034AC8800F4612B0044AC880004F22F008E
:102DC00054AC880014F22F0064AC880024F22F0069
:102DD00074AC88003432210084AC88004452210055
:102DE00094AC880054C22200A4AC880064F22F0086
:102DF000B4AC880074C22200C4AC880084422800AD
:102E0000D4AC880094022000E4AC8800A4022C001A
:102E1000F4AC8800B402200004AD8800C402200095
:102E200014AD8800D402200024AD8800E402200004
:102E300034AD8800F442230044AD88000413200020
:102E400054AD88001403200064AD8800248325005D
:102E500074AD88003403200084AD880044A32000B2
:102E600094AD880054032500A4AD880064032000BD
:102E7000B4AD880074132000C4AD8800841328000A
:102E8000D4AD880094232400E4AD8800A453260028
:102E9000F4AD8800B433230004AE8800F4042000AD
:102EA00014AE880004E7220024AE880014A7200096
:102EB00034AE88002497290044AE8800346720008F
:102EC00054AE88004407200064AE880054072000F8
:102ED00074AE88006467200084AE880074272000E8
:102EE00094AE880084372300A4AE880094072000A5
:102EF000B4AE8800A4872100C4AE8800B4072000C7
:102F0000D4AE8800C4172000E4AE880024F829005D
:102F1000F4AE8800E035EF003410210014AF8800D3
:102F20009431200024AF8800A401200034AF880031
:102F3000B401200044AF8800C401260054AF8800CB
:102F4000D4F12F0064AF8800E491240074AF8800AE
:102F5000F4612B0084AF880004F22F0094AF880046
:102F600014F22F00A4AF880024F22F00B4AF880021
:102F700034322100C4AF880044522100D4AF88000D
:102F800054822200E4AF880064E22600F4AF880097
:102F90007482220004B088008442200014B08800AB
:102FA0009402200024B08800A442200034B088009D
:102FB000B4022C0044B08800C402200054B0880041
:102FC000D402200064B08800E402200074B08800BD
:102FD000F4E2260084B088000403200094B0880046
